:100000000C941F210C944C210C944C210C944C21E9
:100010000C944C210C944C210C944C210C944C21AC
:100020000C944C210C944C210C944C210C944C219C
:100030000C944C210C94CEE60C944C210C944C2145
:100040000C944C210C94FD900C944C210C944C215C
:100050000C944C210C944C210C945C9B0C942EE33E
:100060000C944C210C94753E0C944C210C944C2116
:100070000C944C210C944C210C944C210C944C214C
:100080000C944C210C944C210C944C210C944C213C
:100090000C944C210C944C210C944C210C9406DBB8
:1000A0000C944C210C944C210C944C210C944C211C
:1000B0000C944C210C944C210C944C210C944C210C
:1000C0000C944C210C944C210C944C210C944C21FC
:1000D0000C944C210C944C210C944C210C944C21EC
:1000E0000C944C21084AD73B3BCE016E84BCBFFD2B
:1000F000C12F3D6C74319ABD56833DDA3D00C77FF8
:1001000011BED9E4BB4C3E916BAAAABE0000008090
:100110003F05A84CCDB2D44EB93836A9020C50B91F
:10012000918688083CA6AAAA2ABE000000803F4DFE
:10013000383420582059205A2045006563686F3AAA
:100140000043616E6E6F7420656E74657220737506
:10015000626469723A20004D3234004D32332025FA
:1001600073006175746F25692E67004572726F7236
:100170003A006572726F722077726974696E6720D7
:10018000746F2066696C65004E6F74205344207054
:1001900072696E74696E67002F0053442070726933
:1001A0006E74696E67206279746520002E00446564
:1001B0006C6574696F6E206661696C65642C20469D
:1001C000696C653A200046696C652064656C6574ED
:1001D00065643A002E006F70656E206661696C651B
:1001E000642C2046696C653A200057726974696E08
:1001F0006720746F2066696C653A20002E006F706E
:10020000656E206661696C65642C2046696C653A90
:1002100020002E006F70656E206661696C65642C2D
:100220002046696C653A200046696C652073656CF0
:100230006563746564002053697A653A20004669F5
:100240006C65206F70656E65643A20002E006F70DB
:10025000656E206661696C65642C2046696C653A40
:10026000200053442063617264206F6B006F7065DF
:100270006E526F6F74206661696C656400766F6C96
:10028000756D652E696E6974206661696C656400C0
:10029000534420696E6974206661696C0065636807
:1002A0006F3A0048617264636F64656420446566F8
:1002B00061756C742053657474696E6773204C6F3C
:1002C000616465640053746F72656420736574744F
:1002D000696E677320726574726965766564002063
:1002E00044002049002020204D3330312050005060
:1002F00049442073657474696E67733A00204D69D0
:100300006E757465733A200020486F7572733A20D9
:10031000004C61736572206C69666574696D652057
:1003200075736167653A00205A0020590020204DFE
:10033000323036205800486F6D65206F66667365F1
:100340007420286D6D293A00204500205A0020585D
:100350000020420020540020204D32303520530030
:10036000416476616E636564207661726961626C76
:1003700065733A20533D4D696E2066656564726110
:10038000746520286D6D2F73292C20543D4D696EA6
:100390002074726176656C2066656564726174654F
:1003A00020286D6D2F73292C20423D6D696E696D7B
:1003B000756D207365676D656E742074696D652059
:1003C000286D73292C20583D6D6178696D756D20FD
:1003D0005859206A65726B20286D6D2F73292C2067
:1003E000205A3D6D6178696D756D205A206A65727D
:1003F0006B20286D6D2F73292C2020453D6D617871
:10040000696D756D2045206A65726B20286D6D2FB2
:1004100073290020540020204D32303420530041F5
:100420006363656C65726174696F6E3A20533D61F8
:100430006363656C65726174696F6E2C20543D72E4
:1004400065747261637420616363656C6572617465
:10045000696F6E00204500205A0020590020204D71
:100460003230312058004D6178696D756D204163DF
:1004700063656C65726174696F6E20286D6D2F7392
:1004800032293A00204500205A0020590020204DF2
:100490003230332058004D6178696D756D20666586
:1004A0006564726174657320286D6D2F73293A003D
:1004B000204500205A0020590020204D3932205874
:1004C0000053746570732070657220756E69743A9C
:1004D0000053657474696E67732053746F7265643A
:1004E000006563686F3A004572726F723A00535448
:1004F0004F505045442E20005072696E7465722032
:1005000073746F707065642064756520746F206506
:1005100072726F72732E2046697820746865206548
:1005200072726F7220616E6420757365204D393967
:100530003920746F20726573746172742E20285490
:10054000656D70657261747572652069732072657E
:100550007365742E20536574206974206166746518
:10056000722072657374617274696E6729004B49F9
:100570004C4C45442E20005072696E7465722068A0
:10058000616C7465642E206B696C6C282920636132
:100590006C6C656421006F6B00526573656E643A24
:1005A00020002200556E6B6E6F776E20636F6D6D4D
:1005B000616E643A2022006C636420636F6E747213
:1005C0006173742076616C75653A20007A5F6D61A5
:1005D000783A20007A5F6D696E3A2000795F6D612C
:1005E000783A2000795F6D696E3A2000785F6D611E
:1005F000783A2000785F6D696E3A20005A3A0059C7
:100600003A0020436F756E7420583A2000453A0036
:100610005A3A00593A00583A004649524D57415209
:10062000455F4E414D453A4D61726C696E205631C1
:100630002E312E30687474703A2F2F7777772E6DA5
:10064000656E64656C2D70617274732E636F6D20BE
:1006500050524F544F434F4C5F56455253494F4EA3
:100660003A312E30204D414348494E455F54595050
:10067000453A4C6173657220437574746572204508
:10068000585452554445525F434F554E543A310ADF
:10069000004C6173657220437574746572204F66F7
:1006A000662E004C61736572204375747465722008
:1006B00052656164792E0042656420646F6E652E18
:1006C0000020423A0020453A00543A004265642036
:1006D00048656174696E672E0048656174696E676C
:1006E00020646F6E652E0020573A0020453A005472
:1006F0003A0048656174696E672E2E2E00204240D4
:100700003A0020403A00202F003A00205400202FC9
:100710000020423A00202F006F6B20543A002569D8
:10072000206D696E2C2025692073656300456E6419
:100730002066696C65206C69737400426567696E38
:100740002066696C65206C697374004E6F206D6F54
:1007500076652E00526573756D696E6720707269DB
:100760006E74005761697420666F722075736572CC
:100770002E2E2E00536C6565702E2E2E000080A844
:10078000430000664300009642FFFFFF00000000A8
:100790000000000000000000000000000000000059
:1007A000000000000080A84300006643000096425D
:1007B0000000A0400000A0400000803F25692068A4
:1007C0006F757273202569206D696E75746573008D
:1007D000446F6E65207072696E74696E6720666919
:1007E0006C650053544F505045442E2000507269A0
:1007F0006E7465722073746F7070656420647565C3
:1008000020746F206572726F72732E204669782093
:10081000746865206572726F7220616E64207573F2
:1008200065204D39393920746F2072657374617297
:10083000742E202854656D70657261747572652020
:1008400069732072657365742E2053657420697412
:100850002061667465722072657374617274696E6A
:100860006729006F6B004E6F204C696E65204E75D6
:100870006D626572207769746820636865636B7365
:10088000756D2C204C617374204C696E653A2000A4
:100890004E6F20436865636B73756D20776974686C
:1008A000206C696E65206E756D6265722C204C61DE
:1008B0007374204C696E653A2000636865636B73DE
:1008C000756D206D69736D617463682C204C617364
:1008D00074204C696E653A20004C696E65204E7537
:1008E0006D626572206973206E6F74204C61737441
:1008F000204C696E65204E756D6265722B312C201F
:100900004C617374204C696E653A20004D31313072
:1009100000473700473700473700473700446F6EBE
:100920006520736176696E672066696C652E006F5D
:100930006B004D3239002020506C616E6E65724242
:10094000756666657242797465733A200020467256
:100950006565204D656D6F72793A200046656220AD
:100960003237203230313600436F6D70696C656408
:100970003A200028446F776E756E64657233356D6A
:100980002C204C617365722056312E322900207C58
:1009900020417574686F723A2000466562203237D4
:1009A000203230313632372F30322F32303136204C
:1009B00031353A35346820454153542031353A3584
:1009C000393A353200204C6173742055706461747B
:1009D00065643A2000312E302E30004D61726C6912
:1009E0006E200020536F66747761726520526573C4
:1009F000657400205761746368646F672052657383
:100A00006574002042726F776E206F757420526596
:100A1000736574002045787465726E616C20526550
:100A200073657400506F77657255700073746172EE
:100A300074002200656E717565696E672022002260
:100A400000656E717565696E672022006563686F69
:100A50003A004C6173657220666972696E67206541
:100A60006E61626C6564007C3C3E5E2B3D3F2F5B9B
:100A70005D3B2C2A225C0045313A200045303A206B
:100A8000005A3A2000593A2000583A20004D53317C
:100A90002C4D53322050696E730A00506978656C92
:100AA0003A20004C3A2000593A2000583A200024BD
:100AB000F404D9201BC40C5C0E9804C4095F0265C1
:100AC000077101F405F900FB04B30048048700C175
:100AD0000369005803550003034500BE023A008431
:100AE00002310053022A002902250004022000E4FA
:100AF000011C00C8011900AF0117009801140084FF
:100B0000011300710110006101100051010E00433A
:100B1000010D0036010B002B010B0020010B00150D
:100B20000109000C01090003010800FB000800F3A3
:100B3000000800EB000700E4000600DE000600D815
:100B4000000600D2000600CC000500C7000500C268
:100B5000000500BD000400B9000400B5000400B1A8
:100B6000000400AD000400A9000400A5000300A2D9
:100B70000003009F0004009B000300980003009501
:100B800000020093000300900003008D0002008B20
:100B90000003008800020086000200840003008138
:100BA0000002007F0002007D0002007B000200794D
:100BB000000200770001007600020074000200725B
:100BC000000100710002006F0002006D0001006C66
:100BD0000002006A0001006900020067000100666F
:100BE0000001006500010064000200620001006174
:100BF000000100600001005F0002005D0001005C78
:100C00000001005B0001005A00010059000100587A
:100C1000000100570001005600010055000100547A
:100C20000001005300000053000100520001005178
:100C3000000100500001004F0001004E0000004E76
:100C40000001004D0001004C0001004B0000004B72
:100C50000001004A0001004900010048000000486E
:100C60000001004700010046000000460001004569
:100C70000000004500010044000100430000004363
:100C8000000100420000004200010041000000415C
:100C9000000100400001003F0000003F0001003E55
:100CA0000000003E0001003D0000003D0001003C4E
:100CB0000000003C0000003C0001003B0000003B45
:100CC0000001003A0000003A00010039000000393C
:100CD0000001003800000038000000380001003733
:100CE000000000370001003600000036000000362A
:100CF000000100350000003500000035000100341F
:100D00000000003400000034000100330000003314
:100D10000000003300010032000000320000003209
:100D200000010031000000310000003100010030FE
:100D300000000030000000300001002F0000002FF4
:100D40000000002F0000002F0001002E0000002EE8
:100D50000000002E0001002D0000002D0000002DDD
:100D60000000002D0001002C0000002C0000002CD1
:100D70000000002C0001002B0000002B0000002BC5
:100D80000000002B0001002A0000002A0000002AB9
:100D90000000002A000100290000002900000029AD
:100DA00000000029000000290001002800000028A0
:100DB0000000002800000028000000280001002793
:100DC0000000002700000027000000270000002787
:100DD000000100260000002600000026000000267A
:100DE000000000260001002500000025000000256D
:100DF000000000250000002500000025000100245F
:100E00000000002400000024000000240000002452
:100E10000001002300000023000000230000002345
:100E20000000002300000023000000230001002236
:100E3000000000220000002200000022000000222A
:100E4000000000220001002100000021000000211C
:100E5000000000210000002100000021000000210E
:100E60000001002000000020000000200000002001
:100E700000000020000000200000002000000020F2
:100E80000001001F0000001F0000001F0000001FE5
:100E90000000001F0000001F0000001F0001001ED6
:100EA0000000001E0000001E0000001E00000024C4
:100EB000F4D43050C38E20C2A24017828B7011121E
:100EC0007A910D816CD90AA861E108C7586607615B
:100ED0005143061E4B5D05C145A7041A4111040983
:100EE0003D9803713931034036DB0265339102D4FA
:100EF000305402802E1D02632CEE01752AC501B00C
:100F000028A001102781018F2564012B244B01E0CB
:100F1000223401AC211F018D200D01801FFC0084B3
:100F20001EED00971DDF00B81CD200E61BC6002096
:100F30001BBC00641AB200B219A8000A19A0006A0A
:100F4000189900D117910040178B00B51684003115
:100F5000167E00B31579003A157300C7146F005858
:100F6000146A00EE1366008813630025135E00C741
:100F7000125B006C12570015125400C11151007021
:100F8000114F0021114B00D61049008D104700462B
:100F900010440002104200C00F4000800F3E00428B
:100FA0000F3C00060F3B00CB0E3800930E37005C61
:100FB0000E3500270E3400F30D3200C10D310090C4
:100FC0000D3000600D2E00320D2D00050D2C00D9C6
:100FD0000C2B00AE0C2900850C29005C0C27003579
:100FE0000C27000E0C2600E80B2400C40B2400A0E4
:100FF0000B23007D0B23005A0B2100390B21001815
:101000000B2000F80A1F00D90A1E00BB0A1E009D13
:101010000A1D00800A1D00630A1C00470A1B002CE1
:101020000A1B00110A1A00F7091A00DD091900C489
:10103000091900AB091900920917007B0918006310
:101040000917004C09160036091600200916000A77
:10105000091500F5081500E0081400CC081400B8C4
:10106000081400A4081400900813007D0812006BF7
:101070000813005808120046081200340811002313
:101080000811001208110001081100F0071000E01B
:10109000071000D0071000C0071000B0070F00A114
:1010A00007100091070E0083070F0074070F0065FB
:1010B000070E0057070E0049070E003B070D002ED4
:1010C000070E0020070D0013070D0006070D00F99D
:1010D000060C00ED060D00E0060C00D4060C00C85E
:1010E000060C00BC060C00B0060C00A4060B009910
:1010F000060C008D060B0082060B0077060B006CB9
:10110000060B0061060A0057060B004C060A004257
:10111000060A0038060A002E060A0024060A001AEB
:10112000060A001006090007060A00FD050900F47A
:10113000050900EB050900E2050900D9050900D001
:10114000050900C7050900BE050900B5050800AD81
:10115000050800A50509009C050800940508008CF9
:10116000050800840508007C050800740508006C6B
:10117000050700650508005D050700560508004ED7
:10118000050700470507004005080038050700313E
:101190000507002A050700230507001C05060016A1
:1011A0000507000F0507000805060002050700FBFC
:1011B000040600F5040700EE040600E8040600E259
:1011C000040700DB040600D5040600CF040600C9AE
:1011D000040600C3040600BD040600B7040600B1FF
:1011E000040500AC040600A6040600A00405009B4C
:1011F00004060095040500900406008A0405008595
:10120000040500800406007A0405007504050070DA
:101210000405006B04050066040500610405005C1C
:1012200004050057040500520405004D040500485C
:10123000040500430405003E0404003A040500359B
:10124000040500300404002C0405002704040023D6
:101250000405001E0404001A04040016040500110D
:101260000404000D04040009040500040404000043
:10127000040400FC030400F8030400F4030400F079
:10128000030400EC030400E8030400E4030400E0AA
:10129000030400DC030400D8030400D4030400D0DA
:1012A000030400CC030400C8030300C50303006566
:1012B00063686F3A00656E6473746F707320686959
:1012C000743A205A00205A3A00656E6473746F7045
:1012D00073206869743A20590020593A00656E6499
:1012E00073746F7073206869743A20580020583AFC
:1012F00000656E6473746F7073206869743A2000BF
:101300004572726F723A004572723A204D415854DC
:10131000454D50204245440054656D7065726174BE
:101320007572652068656174656420626564207308
:1013300077697463686564206F66662E204D415836
:1013400054454D5020747269676765726564202149
:1013500021004572723A204D494E54454D50003A95
:101360002045787472756465722073776974636858
:101370006564206F66662E204D494E54454D5020C1
:101380007472696767657265642021004572723AFC
:10139000204D415854454D50003A2045787472759F
:1013A000646572207377697463686564206F66662C
:1013B0002E204D415854454D502074726967676521
:1013C000726564202100202D20496E76616C69646D
:1013D000206578747275646572206E756D626572D1
:1013E000202100504944204175746F74756E65204A
:1013F00066696E697368656421205075742074682D
:1014000065204B702C204B6920616E64204B64205A
:10141000636F6E7374616E747320696E746F2043B2
:101420006F6E66696775726174696F6E2E680050C1
:101430004944204175746F74756E65206661696CEE
:101440006564212074696D656F75740020403A00F1
:101450006F6B20543A006F6B20423A005049442091
:101460004175746F74756E65206661696C65642181
:101470002054656D706572617475726520746F6F4C
:10148000206869676800204B643A2000204B693A65
:101490002000204B703A200020436C617369632068
:1014A00050494420002054753A2000204B753A20C2
:1014B00000206D61783A2000206D696E3A2000208E
:1014C000643A200020626961733A20000006090036
:1014D000FE06018902FE20FFFE07FE06FE00000058
:1014E0000600070106060602008080808000800357
:1014F0000303060103A0A0A00507070600FF505044
:10150000F850F850500509090600FE2070A8A07098
:1015100028A870200608080600FF40A848102048A8
:1015200054080507070600FF6090906098906801D6
:1015300003030602038080800207070602FF408043
:1015400080808080400207070602FF8040404040C4
:1015500040800505050600008850F85088050505FF
:101560000600002020F820200204040602FEC040ED
:101570004080050101060002F8020202060200C0D6
:10158000C0040606060100101020408080040606F4
:1015900006010060909090906003060606010040EE
:1015A000C0404040E0040606060100609010204064
:1015B000F0040606060100F020601010E0050606A3
:1015C00006000010305090F810040606060100F0E6
:1015D00080E01010E00406060601006080E09090B4
:1015E00060040606060100F01010204040040606C4
:1015F000060100609060909060040606060100609D
:101600009090701060020505060200C0C000C0C0C6
:101610000207070602FEC0C000C040408005050565
:101620000600001860806018050303060001F8003A
:10163000F8050505060000C0300830C0040707069D
:101640000100609010604000400506060600007032
:1016500090A8B08070050606060000205088F88823
:1016600088050606060000F088F08888F004060663
:10167000060100609080809060040606060100E08C
:1016800090909090E0040606060100F080E08080D3
:10169000F0040606060100F080E080808004060663
:1016A000060100609080B09060040606060100907C
:1016B00090F0909090030606060100E04040404004
:1016C000E0050606060000381010109060040606BB
:1016D00006010090A0C0A0909004060606010080BC
:1016E00080808080F005060606000088D8A8A888BB
:1016F0008804060606010090D0B09090900506067A
:10170000060000708888888870040606060100E0DC
:101710009090E080800407070601FF609090D0B0B1
:101720006010040606060100E09090E09090040628
:101730000606010060904020906005060606000045
:10174000F8202020202004060606010090909090AA
:101750009060040606060100909090F06060050617
:10176000060600008888A8A8D88805060606000096
:1017700088502020508805060606000088885020E2
:101780002020040606060100F010204080F0030629
:1017900006060100E080808080E004060606010065
:1017A000808040201010030606060100E020202063
:1017B00020E0050303060003205088050101060010
:1017C000FEF802020206020480400404040601003E
:1017D000709090700406060601008080E09090E012
:1017E00004040406010070808070040606060100EF
:1017F00010107090907004040406010060B0C07076
:10180000040606060100205040E04040040606069B
:1018100001FE609090701060040606060100808052
:10182000E09090900306060601004000C04040E0B2
:101830000308080601FE200060202020A0400406C6
:10184000060601008080A0C0A090030606060100E5
:10185000C040404040E0050404060000D0A8A8882D
:10186000040404060100E0909090040404060100C2
:10187000609090600406060601FEE09090E0808093
:101880000406060601FE7090907010100404040611
:101890000100A0D0808004040406010070C030E084
:1018A0000406060601004040E040502004040406FF
:1018B0000100909090700404040601009090606014
:1018C00005040406000088A8A850040404060100CA
:1018D000906060900406060601FE90909070906003
:1018E000040404060100F02040F00307070601008D
:1018F000204040804040200107070602FF80808092
:10190000808080800307070601008040402040401F
:101910008004020206010350A0FFFFFFFFFFFFFF4C
:10192000FFFFFFFFFFFFFFFFFFFFFFFFFFFFFFFFC7
:10193000FFFFFFFFFFFFFFFFFFFF000000060007A4
:1019400001060606020080008080808004060606EC
:1019500001FF2070A0A070200507070600FF304897
:1019600040F04040F8050505060000A8508850A842
:101970000506060600008850F820F8200107070633
:1019800002FF808080008080800407070601FF70CE
:101990008060906010E0030101060105A0060707C2
:1019A000060000788494A494847803050506010158
:1019B00060A06000E00505050600002850A0502842
:1019C000040303060100F01010040101060102F0F7
:1019D0000607070600007884B4A4A48478040101F3
:1019E000060105F004030306010260906005070785
:1019F0000600FF2020F8202000F80305050601015D
:101A000040A02040E0030505060101C0204020C0A1
:101A100002020206020440800405050601FF9090C0
:101A2000B0D08005060606000078E8E8682828019E
:101A30000101060202800202020602FE4080030546
:101A40000506010140C04040E003050506010140D4
:101A5000A04000E0050505060000A0502850A005A4
:101A600008080600FF40C040507030781005080894
:101A70000600FF40C04050680810380508080600FE
:101A8000FFC0204030F03078100407070601002026
:101A9000002060809060050707060000402020506D
:101AA000708888050707060000102020507088887D
:101AB000050707060000205020507088880507079A
:101AC000060000285020507088880507070600008F
:101AD000500020507088880507070600002050201D
:101AE0005070888805060606000078A0F0A0A0B80F
:101AF0000408080601FE6090808090602040040782
:101B0000070601004020F080E080F004070706018E
:101B1000002040F080E080F004070706010020501C
:101B2000F080E080F00407070601005000F080E03C
:101B300080F00307070601008040E0404040E003DA
:101B400007070601002040E0404040E00307070689
:101B5000010040A0E0404040E0030707060100A06C
:101B600000E0404040E00506060600007048E848F6
:101B7000487004070706010050A090D0B090900470
:101B80000707060100402060909090600407070658
:101B9000010020406090909060040707060100203B
:101BA00050609090906004070706010050A060907C
:101BB00090906004070706010050006090909060CC
:101BC0000505050600008850205088040808060115
:101BD000FF1070B0B0D0D0E08004070706010040CD
:101BE000209090909060040707060100204090909C
:101BF000909060040707060100205090909090603C
:101C000004070706010050009090909060050707B8
:101C1000060000102088502020200406060601003F
:101C200080E09090E0800406060601006090A0A08D
:101C300090A00407070601004020007090907004F7
:101C40000707060100204000709090700407070607
:101C500001002050007090907004070706010050AA
:101C6000A00070909070040606060100500070906D
:101C700090700407070601002050207090907005B6
:101C8000040406000070A8B0780406060601FE7081
:101C9000808070204004070706010040200060B0EB
:101CA000C07004070706010020400060B0C0700447
:101CB000070706010020500060B0C0700406060649
:101CC0000100500060B0C0700307070601008040AB
:101CD00000C04040E0030707060100204000C0406C
:101CE00040E003070706010040A000C04040E003B9
:101CF0000606060100A000C04040E00407070601F8
:101D0000003060107090906004070706010050A03A
:101D100000E09090900407070601004020006090CA
:101D20009060040707060100204000609090600466
:101D30000707060100205000609090600407070626
:101D4000010050A00060909060040606060100505B
:101D500000609090600505050600002000F8002056
:101D600004040406010070B0D0E004070706010077
:101D7000402000909090700407070601002040006A
:101D800090909070040707060100205000909090FA
:101D90007004060606010050009090907004090936
:101DA0000601FE20400090909070906004080806A4
:101DB00001FE8080E09090E080800408080601FE2B
:101DC000500090909070906000060900FE07019905
:101DD000032B20FFFE08FE07FE00000006000001A6
:101DE00007070602008080808080008003030306CE
:101DF0000104A0A0A00507070600005050F850F805
:101E000050500507070600002070A07028702005BC
:101E1000070706000048A8502050A89005070706AD
:101E2000000040A0A040A8906801030306020480BF
:101E30008080030707060100204080808040200347
:101E40000707060100804020202040800505050688
:101E500000018850F850880505050600012020F88B
:101E600020200303030601FF6040800501010600F6
:101E700003F80303030601FF40E0400507070600DF
:101E80000008081020408080050707060000205049
:101E900088888850200507070600002060A02020C1
:101EA00020F8050707060000708808304080F80514
:101EB0000707060000F808103008887005070706B5
:101EC000000010305090F81010050707060000F8C9
:101ED00080B0C8088870050707060000304080B051
:101EE000C88870050707060000F808101020404059
:101EF0000507070600007088887088887005070746
:101F0000060000708898680810600307070601FF44
:101F100040E0400040E0400307070601FF40E0408A
:101F20000060408004070706010010204080402028
:101F300010050303060002F800F804070706010075
:101F400080402010204080050707060000708810A0
:101F500020200020050707060000708898A8B080A0
:101F60007005070706000020508888F88888050754
:101F700007060000F04848704848F00507070600CB
:101F80000070888080808870050707060000F04890
:101F900048484848F0050707060000F88080F080B0
:101FA00080F8050707060000F88080F08080800533
:101FB000070706000070888080988870050707066C
:101FC0000000888888F8888888030707060100E0F1
:101FD0004040404040E00507070600003810101060
:101FE0001090600507070600008890A0C0A09088A8
:101FF000050707060000808080808080F8050707BD
:102000000600008888D8A888888805070706000089
:102010008888C8A8988888050707060000708888FF
:1020200088888870050707060000F08888F080809F
:10203000800508080600FF7088888888A870080551
:102040000707060000F08888F0A0908805070706BB
:10205000000070888070088870050707060000F887
:102060002020202020200507070600008888888877
:10207000888870050707060000888888505050201F
:10208000050707060000888888A8A8D888050707DC
:102090000600008888502050888805070706000041
:1020A00088885020202020050707060000F8081027
:1020B000204080F8030707060100E08080808080D0
:1020C000E00507070600008080402010080803078D
:1020D00007060100E02020202020E0050303060081
:1020E000042050880501010600FFF80202020602E2
:1020F0000680400505050600007008788878050709
:10210000070600008080B0C888C8B0050505060035
:102110000070888088700507070600000808689826
:102120008898680505050600007088F88070050726
:1021300007060000304840F0404040050707060011
:10214000FE78888878088870050707060000808078
:10215000B0C88888880307070601004000C04040D7
:1021600040E00409090601FE1000301010109090A4
:102170006005070706000080808890E090880307CC
:1021800007060100C04040404040E005050506004C
:1021900000D0A8A8A888050505060000B0C8888852
:1021A0008805050506000070888888700507070601
:1021B00000FEB0C888C8B080800507070600FE682A
:1021C000988898680808050505060000B0C8808052
:1021D0008005050506000070807008F005070706F9
:1021E00000004040F04040483005050506000088EA
:1021F00088889868050505060000888850502005E5
:1022000005050600008888A8A850050505060000F9
:1022100088502050880507070600FE8888986808BF
:102220008870050505060000F8102040F80407072F
:10223000060100304020C0204030010707060200A0
:1022400080808080808080040707060100C02040D5
:10225000304020C005030306000448A89000000099
:10226000010000000000010000000000010000006B
:10227000000001000000000001000000000001005B
:10228000000000000100000000000100000000004C
:10229000010000000000010000000000010000003B
:1022A000000001000000000001000000000001002B
:1022B000000000000100000000000100000000001C
:1022C000010000000000010000000000010000000B
:1022D00000000100000000000100000000000100FB
:1022E00000000000010000000000010000000000EC
:1022F00001000000000001000000000001000000DB
:1023000000000100000000000100000000000100CA
:1023100000000000010000000000010000000000BB
:10232000010000000000060000010707060200800F
:102330000080808080800507070600FF2078A0A02D
:10234000A07820050707060000304840E04048B06C
:10235000050505060000887050708805080806000D
:10236000FF88885020F820202001070706020080FF
:102370008080008080800508080600FF7080E09063
:1023800048380870030101060107A0050707060089
:10239000007088A8C8A8887004060606010170901D
:1023A000B05000F0060505060000244890482404BB
:1023B0000202060102F010040101060103F0050704
:1023C000070600007088E8C8C8887005010106008B
:1023D00007F803030306010440A0400506060600B3
:1023E000002020F82020F804050506010360902055
:1023F00040F0040505060103E0106010E00202024F
:1024000006020640800506060600FF888888C8B0D8
:102410008005070706000078E8E8682828280101F9
:1024200001060203800202020602FE408003050547
:1024300006010340C04040E004060606010160902A
:10244000906000F0060505060000904824489006BC
:1024500009090600FF40C04040E40C143C04060992
:10246000090600FF40C04040E81404081C050909A3
:102470000600FFC0204020C8182878080507070676
:102480000000200020204088700508080600004059
:1024900020708888F88888050808060000102070D9
:1024A0008888F88888050808060000205070888809
:1024B000F8888805080806000048B0708888F88801
:1024C000880508080600005000708888F88888058C
:1024D00008080600002050708888F88888060707DA
:1024E0000600003C50909CF0909C0509090600FEF7
:1024F00070888080808870204005080806000040B1
:10250000F88080F08080F805080806000010F88048
:1025100080F08080F805080806000020F88080F030
:102520008080F805080806000050F88080F0808060
:10253000F80308080601008040E040404040E00306
:1025400008080601002040E040404040E003080841
:1025500006010040A0E040404040E00308080601BA
:1025600000A000E040404040E0050707060000F002
:102570004848E84848F0050808060000285088C880
:10258000A898888805080806000040207088888878
:1025900088700508080600001020708888888870F8
:1025A0000508080600002050708888888870050893
:1025B000080600002850708888888870050808067A
:1025C00000005000708888888870050505060000A6
:1025D0008850205088050707060000709898A8C802
:1025E000C870050808060000402088888888887020
:1025F000050808060000102088888888887005086B
:1026000008060000205000888888887005080806A1
:102610000000500088888888887005080806000037
:10262000102088885020202005070706000080F031
:1026300088F0808080050707060000708890A090D1
:1026400088B00508080600004020007008788878E7
:102650000508080600001020007008788878050832
:1026600008060000205000700878887805080806E1
:1026700000002850007008788878050707060000D9
:10268000500070087888780508080600002050205F
:10269000700878887806050506000078147C907C20
:1026A0000507070600FE708880887020400508082E
:1026B0000600004020007088F880700508080600B9
:1026C000001020007088F8807005080806000020BF
:1026D00050007088F88070050707060000500070F1
:1026E00088F88070030808060100804000C0404060
:1026F00040E0030808060100408000C0404040E080
:1027000003080806010040A000C0404040E0060A5F
:102710000A0600FEA4A800FC8480808084FC060ACF
:102720000A0600FE549400FC8404040484FC05089A
:1027300008060000285000B0C888888805080806E8
:1027400000004020007088888870040A0A0602FE93
:1027500030408090909090909090040A0A0600FE7D
:10276000C02010909090909090900607070600016E
:10277000448C8C8480403C06070706000188C4C452
:10278000840408F00505050600012000F800200576
:10279000080806000040F0C88888987810050808E6
:1027A000060000E0F88888888888F8050505060096
:1027B000012030F830200508080600002070F820BD
:1027C000202020E00509090600FF2070A8A8B8888D
:1027D0008850200509090600FFE080C0B0A8A83095
:1027E00028280509090600FFF8A88888888888A88D
:1027F000F8050A0A0600FE205050505088A8A88804
:1028000070FFF08F108F109F909F90801086108621
:1028100010C630A6509690AF50FFF0FFF08F108F8B
:10282000109F909F908010801080108010801080EA
:10283000108010FFF059002D2D3A2D2D002D2D2D3B
:10284000250025004E6F2043617264005072696E4E
:10285000742066726F6D2053440053746F70205063
:1028600072696E7400526573756D65205072696E81
:1028700074005061757365205072696E7400436F07
:102880006E74726F6C005072657061726500547581
:102890006E65004C617365722046756E6374696F76
:1028A0006E7300496E666F2073637265656E00F922
:1028B0002E2E004D61696E004D3234004D323320B2
:1028C0002573004D383420582059205A2045005295
:1028D0006573746F7265204661696C73616665002B
:1028E0004C6F6164206D656D6F72790053746F7207
:1028F00065206D656D6F7279004C434420636F6E87
:102900007472617374004D6F74696F6E004D61690C
:102910006E00436F6E7472617374004573746570FA
:10292000732F6D6D004573746570732F6D6D005A54
:1029300073746570732F6D6D005A73746570732FA7
:102940006D6D005973746570732F6D6D00597374DC
:102950006570732F6D6D005873746570732F6D6D96
:10296000005873746570732F6D6D00412D7265741E
:102970007261637400412D72657472616374004109
:102980006D6178206500416D6178206500416D6161
:1029900078207A00416D6178207A00416D6178205D
:1029A0007900416D6178207900416D61782078006F
:1029B000416D61782078005654726176206D696EA1
:1029C000005654726176206D696E00566D696E0016
:1029D000566D696E00566D6178206500566D6178A0
:1029E000206500566D6178207A00566D6178207AF6
:1029F00000566D6178207900566D61782079005617
:102A00006D6178207800566D617820780056652DCC
:102A10006A65726B0056652D6A65726B00567A2D79
:102A20006A65726B00567A2D6A65726B005678790A
:102A30002D6A65726B005678792D6A65726B00415C
:102A40006363656C00416363656C00436F6E747211
:102A50006F6C004D6F76652041786973004D38309A
:102A60000053776974636820506F776572204F6EEA
:102A7000004D38310053776974636820506F776573
:102A800072204F6666004739322058302059302076
:102A90005A3000536574204F726967696E0047327F
:102AA0003820582059204632303030004175746F3C
:102AB00020486F6D65004D313700456E61626C6571
:102AC000205374657070657273004D38340044692A
:102AD0007361626C65205374657070657273004D2C
:102AE00061696E004D6F766520302E316D6D004D41
:102AF0006F766520316D6D004D6F76652031306DDC
:102B00006D0050726570617265004578747275640D
:102B10006572004D6F7665205A004D6F76652059BD
:102B2000004D6F76652058004D6F766520417869BD
:102B300073004578747275646572005A00590058C4
:102B4000005370656564005370656564004D61698C
:102B50006E00546573742046697265005365742075
:102B6000466F637573004D61696E005761726D2D1C
:102B70007570204C6173657220327365630031306B
:102B80003025203130306D73003130302520203534
:102B9000306D730020323025203130306D730020CD
:102BA000323025202035306D73004C617365722002
:102BB00046756E6374696F6E73004D3830004375EF
:102BC00073746F6D00437573746F6D00376D6D00B6
:102BD000366D6D202D20312F34696E00356D6D00FE
:102BE000346D6D00336D6D202D20312F38696E00EE
:102BF000326D6D00316D6D004C61736572204675EC
:102C00006E6374696F6E73004730205A25732046D7
:102C100031353000473238205A20463135300043B4
:102C20006172642072656D6F7665640043617264E1
:102C300020696E73657274656400FFFFFFFFFFFF1C
:102C4000FFF0FFFFFFFFFFFFFFF0FFFFFFF9FFFFB8
:102C5000FFF0FFFFFFF0FFFFFFF0FFFFFFE07FFF50
:102C6000FFF0FFFFFFC03FFFFFF0FFFFFF801FFFF0
:102C7000FFF0FFFFFF000FFFFFF0FFFFFE0007FF69
:102C8000FFF0FFFFFC0003FFFFF0FFFFF80001FF74
:102C9000FFF0FFFFF00000FFFFF0FFFFE000007F0C
:102CA000FFF0FFFFC000003FFFF0FFFF8000003F8C
:102CB000FFF0FFFF0000001FFFF0FFFE0000000F0D
:102CC000FFF0FFFE00000007FFF0FFFC0000000720
:102CD000FFF0FFFC00000003FFF0FFF8000000031E
:102CE000FFF0FFF800000003FFF0FFF80000000114
:102CF000FFF0FFF800000001FFF0FFF80000000106
:102D0000FFF0FFF800000001FFF0FFF800000001F5
:102D1000FFF0FFF800000001FFF0FFF800000001E5
:102D2000FFF0FFF800000001FFF0FFF800000003D3
:102D3000FFF0FFF800000003FFF0FFFC00000003BD
:102D4000FFF0FFFC00000007FFF0FFFE000000079F
:102D5000FFF0FFFE0000000FFFF0FFFF0000001F6C
:102D6000FFF0FFFF8000001FFFF0FFFFC000003FEB
:102D7000FFF0FFFFE000007FFFF0FFFFF00001FF2A
:102D8000FFF0FFFFFC0003FFFFF0FFFFFF001FFF4E
:102D9000FFF0FFFFFFFFFFFFFFF0FFFFFFFFFFFF61
:102DA000FFF0FFFFFFFFFFFFFFF0FFFFFFFFFFFF51
:102DB000FFF0FFFFFFFFFFFFFFF0FFFFFFFFFFFF41
:102DC000FFF0FFFFFFFFFFFFFFF083FFFFFE0FFF9E
:102DD000FFF080FFFFFE03FFFFF0887FFFFE23FF71
:102DE000FFF08C70380E7181C0708C60380E63807B
:102DF000C03080E319C607F8C73080E019C60380E9
:102E0000C7108C6279C6639CC7308C63F8C6711892
:102E1000C6308E30180E7180C0309E38391E79C48D
:102E2000C4F0FFFFF9FFFFFFC7F0FFFFF9FFFFFF4F
:102E3000C7F0FFFFFFFFFFFFFFF0000000000000F2
:102E40000000000000000000000000000000000082
:102E50000000000000000000000000000000000072
:102E60000000000000000000000000000000000062
:102E7000000000000000000001050800FF0601211D
:102E8000023520FFFF07FF06FF090050221656807B
:102E90008080800080153353A0A0A0025757505067
:102EA000F850F850500257572070A0702870201327
:102EB000355580A040A02002475740A0A040A0A0C8
:102EC0005025135380808012265640808080804099
:102ED0001226568040404040800245559060F06088
:102EE000900255552020F820201133536040800473
:102EF0004151F011335340E040024656101020403B
:102F0000808012365640A0A0A0A04012365640C085
:102F1000404040E00246566090106080F002465605
:102F2000F020601090600246562060A0F020200241
:102F30004656F080E01090600246566080E0909027
:102F400060024656F01020204040024656609060D5
:102F5000909060024656609090701060122555C0A7
:102F6000C000C0C011365660600060408012365606
:102F7000204080804020034353F000F012365680FA
:102F8000402020408012365640A02040004001588A
:102F900058304898A8A8904030024656609090F06B
:102FA0009090024656E090E09090E0024656609085
:102FB00080809060024656E090909090E0024656E5
:102FC000F080E08080F0024656F080E08080800251
:102FD0004656609080B090600246569090F0909077
:102FE00090123656E040404040E0024656702020A5
:102FF00020A04002465690A0C0A0A0900246568055
:1030000080808080F002465690F0F09090900246CA
:103010005690D0F0B0B0900246566090909090607C
:10302000024656E09090E08080014757609090D033
:10303000B06010024656E09090E0909002465660D4
:103040009040209060123656E0404040404002469A
:10305000569090909090600246569090909060604C
:10306000024656909090F0F0900246569090606024
:103070009090025656888850202020024656F01024
:10308000204080F0123656E080808080E002465674
:10309000808040201010123656E020202020E016BC
:1030A000325240A0014151F0162252804002445455
:1030B000709090700246568080E09090E0123454F8
:1030C00060808060024656101070909070024454E8
:1030D00060B0C060024656205040E0404001455577
:1030E00060907010600246568080E090909012369A
:1030F000564000C04040E01137572000202020A05B
:1031000040024656808090E09090123656C0404073
:103110004040E0025454D0A8A8A8024454E0909043
:103120009002445460909060014555E090E08080AA
:103130000145557090701010024454A0D080801248
:10314000345460C020C00246564040E04050200247
:10315000445490909070123454A0A0A04002545453
:1031600088A8A85002445490606090014555909002
:10317000709060024454F02040F0024757304020E5
:10318000C0204030221656808080808080024757C1
:10319000C02040304020C006425250A0FFFFFFFF39
:1031A000FFFFFFFFFFFFFFFFFFFFFFFFFFFFFFFF2F
:1031B000FFFFFFFFFFFFFFFFFFFFFFFFFF090050C3
:1031C0002216568000808080800146562070A0A084
:1031D00070200246562050E04050A002555588709D
:1031E0005070880256568850F820F82022175780D1
:1031F0008080008080800247577080E0907010E0EF
:10320000173151A002565670A8C8C8A87014355579
:1032100060A06000E003435350A050123353E020FD
:1032200020143151E002565670E8D8E8D8701731B2
:1032300051E015335340A04012355540E04000E0C6
:1032400014355540A02040E0143555C020C020C0A2
:103250001622524080014555909090E080025656CB
:1032600078E8E868282824115180112252408014FF
:10327000355540C04040E014355540A04000E003C3
:103280004353A050A0024757808080A060F02002E6
:1032900047578080A0D01020700247578040806040
:1032A000A0F02012365640004080A0400247574010
:1032B000206090F0909002475720406090F09090EE
:1032C00002475760906090F0909002475750A0607E
:1032D00090F0909002475790006090F090900247D5
:1032E0005760906090F0909002465670A0A0F0A0B9
:1032F000B00147576090808090604002475740205F
:10330000F080E080F00247572040F080E080F0023B
:1033100047576090F080E080F00247579000F080BF
:10332000E080F01237578040E0404040E0123757CD
:103330002040E0404040E012375740A0E04040408D
:10334000E0123757A000E0404040E0025656704877
:10335000E848487002475750A090D0B0909002477C
:1033600057402060909090600247572040609090B6
:10337000906002475760906090909060024757506D
:10338000A06090909060024757900060909090608D
:10339000123353A040A002465670B0B0D0D0E00225
:1033A000475740209090909060024757204090905F
:1033B00090906002475760909090909060024757BD
:1033C00090009090909060025757102088502020D5
:1033D0002002465680E09090E0800246566090A021
:1033E000A090A0024757402000709090700247576D
:1033F00020400070909070024757205000709090CD
:103400007002475750A000709090700246565000CE
:103410007090907002475760906070909070025466
:1034200054F068B07811355560808060400247578D
:1034300040200060B0C06002475720400060B0C02C
:103440006002475760900060B0C06002465650006E
:1034500060B0C060123757804000C04040E0123773
:1034600057204000C04040E012375740A000C04005
:1034700040E0123656A000C04040E0024757A0404E
:10348000A01070906002475750A000E0909090020A
:1034900047574020006090906002475720400060EE
:1034A000909060024757609000609090600247578C
:1034B00050A000609090600246569000609090602E
:1034C0001235554000E0004002445470B0D0E00294
:1034D000475740200090909070024757204000903E
:1034E00090907002475760900090909070024656FE
:1034F00090009090907001485820400090907090FB
:10350000600147578080E090E0808001475790003D
:10351000909070906000091200FC0A01E803D72027
:10352000FFFD0EFD0BFD00000009000E010B0B0955
:1035300004008080808080808000008080040404FB
:1035400009030790909090080A0A09000024242497
:10355000FF2424FF242424070B0B0901FF107C9275
:103560009050381412927C10070A0A09010042A4F4
:10357000A4481010244A4A84070A0A0901006090EE
:10358000909060629488946201040409040780802A
:103590008080030C0C0903FF2040408080808080E5
:1035A00080404020030C0C0903FF80404020202075
:1035B000202020404080070707090103109254385B
:1035C000549210070707090101101010FE10101087
:1035D0000204040904FEC0C040800701010901047F
:1035E000FE020202090400C0C0070A0A0901000223
:1035F000040408101020404080070A0A090100381E
:10360000448282828282824438070A0A09010010B9
:103610003050901010101010FE070A0A09010038EF
:103620004482020408102040FE070A0A090100FE35
:10363000020408180402028478070A0A0901000437
:103640000C14244484FE040404070A0A090100FE41
:10365000808080F80402028478070A0A0901003C8D
:10366000408080B8C482824438070A0A090100FEFB
:10367000020404080810101010070A0A0901003893
:10368000448244384482824438070A0A09010038D7
:10369000448282463A02020478020707090400C005
:1036A000C0000000C0C00209090904FEC0C000003B
:1036B00000C0C040800509090902000810204080B0
:1036C00040201008070404090102FE0000FE05095D
:1036D00009090200804020100810204080070A0AD3
:1036E00009010038448202040810100010070A0A79
:1036F00009010038449AAAAAAAAA9C403C070A0ACF
:1037000009010010282828447C44828282070A0A82
:10371000090100F8848284F884828284F8070A0A06
:103720000901003C42808080808080423C070A0A78
:10373000090100F88482828282828284F8070A0A60
:10374000090100FE808080F880808080FE070A0AE0
:10375000090100FE808080F88080808080070A0A4E
:1037600009010038448280808E82824438070A0A28
:1037700009010082828282FE8282828282050A0A96
:10378000090200F82020202020202020F8070A0A23
:103790000901003E080808080808888870070A0A16
:1037A00009010082848890A0D088848282070A0A56
:1037B000090100808080808080808080FE070A0A66
:1037C0000901008282C6AA928282828282070A0A44
:1037D0000901008282C2A2928A86828282070A0A34
:1037E0000901007C82828282828282827C070A0AAC
:1037F000090100F884828284F880808080080B0BA5
:103800000901FF384482828282828A443A01070A8F
:103810000A090100F884828284F890888482070A69
:103820000A0901007C8280807C020202827C070AF5
:103830000A090100FE101010101010101010070AD5
:103840000A09010082828282828282824438070AC7
:103850000A09010082828244444428282810070A69
:103860000A0901008282828292929292AA44070AF5
:103870000A09010082824428101028448282070A23
:103880000A09010082824428101010101010070A43
:103890000A090100FE0204081020408080FE040C8A
:1038A0000C0903FFF080808080808080808080F021
:1038B000070A0A0901008040402010100804040291
:1038C000040C0C0902FFF010101010101010101052
:1038D00010F00704040901061028448208010109B8
:1038E00000FFFF03030309030A80402007070709BD
:1038F00001007C02027E82867A070A0A09010080A2
:103900008080BCC2828282C2BC0707070901007C9A
:1039100082808080827C070A0A0901000202027A02
:1039200086828282867A0707070901007C8282FEEE
:1039300080827C070A0A0901001C22222020F8202C
:10394000202020070A0A0901FD7A84848478807C7B
:1039500082827C070A0A090100808080BCC28282C0
:10396000828282050A0A090200600000E02020200D
:103970002020F8050D0D0902FD1800003808080880
:10398000080808888870070A0A0901008080808476
:103990008890B0C88482050A0A090200E02020202D
:1039A0002020202020F8070707090100EC929292BE
:1039B000929282070707090100BCC282828282823A
:1039C0000707070901007C82828282827C070A0A3B
:1039D0000901FDB8C4828282C4B8808080070A0AC7
:1039E0000901FD3A46828282463A0202020707072F
:1039F0000901009C6242404040400707070901005E
:103A00007C82807C02827C0709090901002020FC5D
:103A100020202020221C07070709010082828282C1
:103A200082867A0707070901008282444428281009
:103A30000707070901008282929292AA44070707AA
:103A400009010082442810284482070A0A0901FD5E
:103A50004242242424181810906007070709010027
:103A6000FE0408102040FE060B0B0902001C20205B
:103A70002020C0202020201C010C0C0904FF808085
:103A800080808080808080808080060B0B09010010
:103A9000E0101010100C10101010E00703030901C3
:103AA0000762928CFFFFFFFFFFFFFFFFFFFFFFFF9B
:103AB000FFFFFFFFFFFFFFFFFFFFFFFFFFFFFFFF16
:103AC000FFFFFFFFFF00000009000E010B0B0904C0
:103AD0000080800000808080808080800608080947
:103AE000010008789490A0A47840070A0A09010010
:103AF0001C222020F8202060A25C07060609010392
:103B0000827C44447C82070A0A090100828244289C
:103B10007C107C101010010B0B0904FF808080804A
:103B200080008080808080040B0B0902FF60908001
:103B3000609090906010906003020209030BA0A0B7
:103B40000809090900013C4299A5A1A599423C0533
:103B50000707090103609070907800F807080809CA
:103B6000010112244890904824120604040901021D
:103B7000FC040404050101090204F808090909000C
:103B8000013C42B9A5BDA9A5423C060101090109B4
:103B9000FC04040409030660909060070909090108
:103BA00001101010FE10101000FE0406060901049A
:103BB0006090106080F004060609010460902010F7
:103BC000906003030309030A2040800709090901E3
:103BD000FE8282828282C6BA8080070A0A090100B8
:103BE0007E8A8A8A7A0A0A0A0A0A020202090404F6
:103BF000C0C00403030902FD20906003060609010A
:103C00000440C0404040E005060609010470888871
:103C10007000F8070808090101904824121224488E
:103C200090070A0A09010040C0404042E60A121A01
:103C300006070A0A09010040C040404CF2020C107D
:103C40001E070A0A0901006090201092660A121AE3
:103C500006070A0A09010010001010204080828225
:103C60007C070E0E090100201008001028282844A7
:103C70007C44828282070E0E090100081020001089
:103C8000282828447C44828282070E0E09010010F5
:103C900028440010282828447C44828282070D0D85
:103CA00009010034580010282828447C448282826C
:103CB000070D0D09010028280010282828447C44FD
:103CC000828282070E0E0901001028281010282871
:103CD00028447C44828282070A0A0901001E28289F
:103CE000284E784888888E070D0D0901FD3C4280DA
:103CF0008080808080423C082418070E0E09010055
:103D000020100800FE808080F880808080FE070EF2
:103D10000E09010008102000FE808080F88080805D
:103D200080FE070E0E09010010284400FE808080EE
:103D3000F880808080FE070D0D090100282800FE14
:103D4000808080F880808080FE050E0E0902004091
:103D5000201000F82020202020202020F8050E0E22
:103D600009020010204000F82020202020202020E0
:103D7000F8050E0E09020020508800F820202020AF
:103D800020202020F8050D0D090200505000F820D9
:103D900020202020202020F8070A0A09010078446A
:103DA0004242F24242424478070D0D090100345864
:103DB000008282C2A2928A86828282070E0E090146
:103DC00000201008007C82828282828282827C07AC
:103DD0000E0E090100081020007C828282828282FD
:103DE00082827C070E0E090100102844007C82822A
:103DF0008282828282827C070D0D09010034580084
:103E00007C82828282828282827C070D0D0901007F
:103E10002828007C82828282828282827C07070735
:103E200009010182442810284482070C0C0901FF73
:103E3000027C868A8A9292A2A2C27C80070E0E0918
:103E400001002010080082828282828282824438AD
:103E5000070E0E09010008102000828282828282F1
:103E600082824438070E0E09010010284400828225
:103E70008282828282824438070D0D09010028283F
:103E80000082828282828282824438070E0E090179
:103E90000008102000828244281010101010100713
:103EA0000A0A0901008080FC828282FC80808006F0
:103EB0000A0A09010038444448D048444444580799
:103EC0000B0B090100201008007C02027E82867A1A
:103ED000070B0B090100081020007C02027E82867D
:103EE0007A070B0B090100102844007C02027E8235
:103EF000867A070A0A0901003458007C02027E8291
:103F0000867A070A0A0901002828007C02027E82BC
:103F1000867A070C0C09010010282810007C020288
:103F20007E82867A0707070901006C12127E909242
:103F30006C070A0A0901FD7C82808080827C10481F
:103F400030070B0B090100201008007C8282FE80E4
:103F5000827C070B0B090100081020007C8282FE86
:103F600080827C070B0B090100102844007C8282B0
:103F7000FE80827C070A0A0901002828007C8282D0
:103F8000FE80827C050C0C0902008040200000E0CD
:103F90002020202020F8050C0C09020010204000F1
:103FA00000E02020202020F8050C0C090200205001
:103FB000880000E02020202020F8050B0B090200DB
:103FC00050500000E02020202020F8070B0B0901B2
:103FD00000483050083C448282824438070A0A096B
:103FE0000100345800BCC28282828282070B0B0916
:103FF0000100201008007C82828282827C070B0BE9
:10400000090100081020007C82828282827C070BDA
:104010000B090100102844007C82828282827C0786
:104020000A0A0901003458007C82828282827C075D
:104030000A0A0901002828007C82828282827C0789
:10404000090909010010381000FE00103810070996
:10405000090901FF027C8A8A92A2A27C80070B0BCD
:10406000090100402010008282828282867A070B3A
:104070000B090100081020008282828282867A0762
:104080000B0B090100102844008282828282867A0A
:10409000070A0A0901002828008282828282867A21
:1040A000070E0E0901FD04081000424224242418C2
:1040B00018109060070B0B0901FE8080B8C4828243
:1040C00082C4B88080070D0D0901FD2424004242FE
:1040D00024242418181090600000210024002700D8
:1040E0002A002D0030003300010100000401070107
:1040F0000A0100002200250028002B002E003100BC
:10410000340002010000050108010B01000020003D
:104110002300260029002C002F003200000100009F
:10412000030106010901050505050705080808083A
:10413000020202020A0A080804040404010101013F
:10414000010101010303030303030303040707073A
:104150000C0C0C0C0C0C0C0C0202020206060606DF
:10416000060606060B0B0B0B0B0B0B0B01021020AC
:10417000200808102040102040800201020108049D
:104180000201010204081020408080402010080431
:10419000020180040201804020100804020108048A
:1041A00002010102040810204080010204081020CE
:1041B00040800000090A02080B0C0D0706030401E9
:1041C00000000000000000000000000000000000EF
:1041D00000000000000000000000000000001110BE
:1041E0000F000000000000000000000000000000C0
:1041F000000000000000000002494E46494E4954AC
:10420000594E414ECDCCCC3D0AD7233C17B7D138BF
:1042100077CC2B329595E6241FB14F0A0000204140
:104220000000C84200401C4620BCBE4CCA1B0E5AAF
:10423000AEC59D74093F744116D775DA6F411124DC
:104240001FBECFEFD1E2DEBFCDBF00E00CBF15E057
:10425000A0E0B2E0ECE0FFED01E00BBF02C0079090
:104260000D92A239B107D9F71BBE1BE1A2E9B5E057
:1042700001C01D92A835B107E1F712E4CCE3D2E406
:1042800004C02297FE010E942CEFC433D107C9F766
:104290000E9428E60C947AEF0C940000A0E0B0E0B5
:1042A000E4E5F1E20C9449EFEC015B016115710565
:1042B00019F0FB0191838083F9908F2D90E00E948B
:1042C00030EF892BC9F7FDE2FF1621F4F990EE24B7
:1042D000E39405C02BE2F21609F4F990EE248E0166
:1042E00001501040C80169EF71E443E050E069D229
:1042F000892BF9F48E010E5F1F4FC8016CEF71E43A
:1043000045E050E05ED2892B19F48E01095F1F4F02
:10431000A114B10419F0F50111830083E0FC04C07D
:1043200070E090E080E813C070E090E080E86FEF0C
:1043300007C1C80161E072E443E050E042D2892B3A
:1043400069F4A114B10429F470E090E080EC6FE707
:10435000F7C02296F501D183C083F6CF8824992433
:1043600040E050E060E070E0EF2DE053EA30A0F56F
:10437000F2E0EF2A8E2D90E09C0128703070E2FE72
:1043800006C0232B79F50894811C911C2BC0232B8C
:1043900019F0089481089108DB01CA0112E0880F26
:1043A000991FAA1FBB1F1A95D1F7480F591F6A1FE3
:1043B0007B1F440F551F661F771F4E0F511D611D38
:1043C000711D483929E9520729E9620729E1720775
:1043D00048F084E0E82A06C0EE3F31F4E3FC39C03F
:1043E00098E0E92AF990C0CFE53311F0E53189F57D
:1043F00029912D3219F4E0E1EE2A05C02B3219F093
:1044000081E090E003C0299182E090E0E22FE05348
:10441000EA3018F0C81BD90B1CC020E030E0FCE0EB
:1044200020383F075CF4C901880F991F880F991F36
:10443000280F391F220F331F2E0F311DE991E05332
:10444000EA3068F3E4FE03C0309521953F4F820EB9
:10445000931ECE2CDD24E1FE07C0A114B10421F08F
:104460002197F501D183C083CB01BA010E9495EB5E
:104470007B018C01F3E0CF22DD2423E0C216D104BE
:1044800021F417FB109517F9109557016801C80121
:10449000B70120E030E040E050E00E94F5EA8823D8
:1044A00009F44AC097FE0DC028E1E22E22E4F22E64
:1044B0009094819491089394C0E2D0E000E010E0E1
:1044C00012C090E3E92E92E4F92EF6CFF701259180
:1044D000359145915491C601B5010E94D5ED5B011E
:1044E0006C018C1A9D0A8C169D0684F7D595C7958C
:1044F0000F5F1F4F0630110529F08CEF9FEFE80E7C
:10450000F91EF1CFC501D6017C018D018C2D880FDC
:104510008D2D881F8F3F51F0C601B50120E030E09E
:1045200040E050E00E94F5EA882331F482E290E016
:104530009093571B8093561B7E2D9F2D802F612FAC
:10454000272F392F482F562FB901CA01CDB7DEB713
:10455000ECE00C9465EF2F923F925F926F927F9206
:104560008F929F92AF92BF92CF92DF92EF92FF9283
:104570000F931F93CF93DF938C011B01EA01611509
:10458000710519F0FB0191838083209749F0CE01DA
:104590000297839728F020E030E040E050E0F6C03A
:1045A000F801A1908F018A2D90E00E9430EF892BB5
:1045B000B9F7FDE2AF1631F4F801A1908F0155244F
:1045C000539407C0FBE2AF1619F4F801A1908F01D4
:1045D0005524209719F0C031D105C1F4F0E3AF168E
:1045E00079F4F8018081883711F0883549F4F801B1
:1045F000A1800E5F1F4FF2E05F2AC0E1D0E006C04D
:10460000209721F480E3A816E9F427C0C830D1052B
:1046100031F1C930D10524F4C230D10531F50CC0D7
:10462000CA30D10589F0C031D105F9F4C12CD12CA3
:10463000E12CB8E0FB2E28C0C12CD12CE12CA0E449
:10464000FA2E22C0CAE0D0E0FCECCF2EFCECDF2E2C
:10465000FCECEF2EFCE0FF2E17C0C8E0D0E0C12C30
:10466000D12CE12CE0E1FE2E0FC09E01442737FD46
:104670004095542F60E070E080E090E80E94EDEEFD
:10468000C901DA016C017D0120E030E040E050E03A
:1046900060E03E01882477FC8094982C70EDB72E62
:1046A000BA0CE9E0EB1570F48A2D81548A3118F4C4
:1046B00099ECB92E06C08A2D81568A3150F589EAC7
:1046C000B82EBA0C8B2D90E08C179D0714F56F3F18
:1046D000E1F0C216D306E406F506B0F0CA01B9014E
:1046E000A40193010E94A7EE9B01AC012B0D311D8B
:1046F000411D511D2130F0E03F07F0E04F07F0E889
:104700005F0710F461E001C06FEFF801A1908F0125
:10471000C5CF2114310481F0662331F001501040DF
:10472000F1011183008308C051FE1AC002501040ED
:10473000F1011183008314C067FF12C050FC05C053
:104740002FEF3FEF4FEF5FE704C020E030E040E0A5
:1047500050E882E290E09093571B8093561B16C05E
:1047600050FE08C050954095309521953F4F4F4FD2
:104770005F4F0CC057FF0AC082E290E09093571B36
:104780008093561B2FEF3FEF4FEF5FE7B901CA0150
:10479000DF91CF911F910F91FF90EF90DF90CF901D
:1047A000BF90AF909F908F907F906F905F903F9061
:1047B0002F900895FB01DC0105900D920020E1F798
:1047C0000895FB01DC014150504088F08D91813407
:1047D0001CF08B350CF4805E659161341CF06B35F8
:1047E0000CF4605E861B611171F3990B0895881BB0
:1047F000FCCFFB01DC014150504048F005900D9288
:104800000020C9F701C01D9241505040E0F70895C3
:10481000FB0155915523A9F0BF01DC014D914517CE
:104820004111E1F759F4CD010590002049F04D9177
:1048300040154111C9F3FB014111EFCF81E090E038
:1048400001970895FB01DC0104C08D91019080194E
:1048500021F441505040C8F7881B990B0895FB0183
:10486000DC0102C001900D9241505040D8F70895EC
:10487000FB01DC010D900020E9F7119701900D92EA
:104880000020E1F70895FC018191861721F088232B
:10489000D9F7992708953197CF010895FB01DC01DD
:1048A00001900D920020E1F70895FB01DC014150D9
:1048B000504030F08D910190801919F40020B9F723
:1048C000881B990B0895FB01DC014150504048F0D2
:1048D00001900D920020C9F701C01D924150504037
:1048E000E0F70895AEE0B0E0E8E7F4E20C9451EFB1
:1048F0000E891F898EE08C831A8309838FEF9FE7CF
:104900009E838D839E01265E3F4FCE010196688D6A
:10491000798DA9010AD02F813885020F131FF80164
:1049200010822E96E4E00C946DEFABE0B0E0EBE982
:10493000F4E20C9443EF3C012B015A01FC01178275
:104940001682838181FD03C06FEF7FEFB9C19AE0CA
:10495000892E1E010894211C311CF3012381F201D0
:1049600023FD859123FF81912F01882309F4A5C19F
:10497000853239F423FD859123FF81912F01853202
:1049800021F490E0B301B7D1E8CF982FFF24EE24B3
:104990009924FFE1FF15D0F09B3269F09C3228F496
:1049A000903259F0933291F40EC09D3249F0903319
:1049B00069F441E024C052E0F52A84E0F82A28C0D6
:1049C00098E0F92A25C0E0E1FE2A22C0F7FC29C0C0
:1049D000892F80538A3070F4F6FE05C0989C902C85
:1049E0001124980E15C0E89CE02C1124E80EF0E28A
:1049F000FF2A0EC09E3229F4F6FC5FC140E4F42A7F
:104A000007C09C3619F450E8F52A02C0983649F4DC
:104A1000F20123FD959123FF91912F01992309F034
:104A2000B8CF892F8554833018F08052833038F402
:104A300044E050E0A40EB51E5FE359830FC09336E7
:104A400031F0933779F0933509F052C01FC0F5016A
:104A50008081898342E050E0A40EB51E610101E02F
:104A600010E011C0F501C080D180F6FC03C06FEFEB
:104A70007FEF02C0692D70E042E050E0A40EB51E49
:104A8000C6012ED18C015FE7F52213C0F501C0806D
:104A9000D180F6FC03C06FEF7FEF02C0692D70E09C
:104AA00042E050E0A40EB51EC6010FD18C0150E8C3
:104AB000F52AF3FE06C018C080E290E0B3011BD1D6
:104AC000EA948E2D90E008171907B0F30DC0F60197
:104AD000F7FC8591F7FE81916F0190E0B3010BD156
:104AE000E110EA94015010400115110581F7E2C070
:104AF000943611F0993661F5F7FE08C0F501208172
:104B000031814281538184E090E00AC0F5018081C7
:104B100091819C01442737FD4095542F82E090E01D
:104B2000A80EB91E9FE6F92257FF09C0509540957F
:104B3000309521953F4F4F4F5F4FE0E8FE2ACA0165
:104B4000B901A1012AE030E002D1D82ED2183FC02D
:104B5000953729F41F2D1F7E2AE030E01DC01F2D40
:104B6000197F9F3661F0903720F4983509F0A5C081
:104B70000FC0903739F0983709F09FC004C028E083
:104B800030E00AC0106114FD146020E130E004C080
:104B900014FD166020E132E017FF08C0F5016081C6
:104BA00071818281938144E050E008C0F5018081E9
:104BB0009181BC0180E090E042E050E0A40EB51E7F
:104BC000A101C5D0D82ED2188FE7F82EF122F6FE1B
:104BD0000BC05EEFF522D91438F4F4FE07C0F2FCE6
:104BE00005C08FEEF82202C01D2D01C0192DF4FE64
:104BF0000DC0FE01ED0DF11D8081803319F499EE99
:104C0000F92208C01F5FF2FE05C003C08F2D867811
:104C100009F01F5F0F2DF3FC13C0F0FE0EC01E1530
:104C200010F09D2C0AC09D2C9E0C911A1E2D05C0C3
:104C300080E290E0B3015FD01F5F1E15C8F304C08F
:104C40001E1510F4E11A01C0EE2404FF0EC080E32B
:104C500090E0B30150D002FF1BC001FD03C088E704
:104C600090E00EC088E590E00BC0802F867881F040
:104C700001FF02C08BE201C080E2F7FC8DE290E010
:104C8000B30139D005C080E390E0B30134D09A94E9
:104C9000D914C8F3DA94F101ED0DF11D808190E093
:104CA000B30129D0DD20B1F705C080E290E0B30167
:104CB00022D0EA94EE20C9F750CEF30166817781C5
:104CC000CB012B96E2E10C945FEFFC010590615063
:104CD00070400110D8F7809590958E0F9F1F089512
:104CE000FC016150704001900110D8F780959095BB
:104CF0008E0F9F1F08950F931F93CF93DF938C0107
:104D0000EB018B8181FF1BC082FF0DC02E813F8193
:104D10008C819D812817390764F4E881F98101931A
:104D2000F983E88306C0E885F985802F1995892BDA
:104D300031F48E819F8101969F838E8302C00FEF95
:104D40001FEFC801DF91CF911F910F910895FA01D4
:104D5000AA27283051F1203181F1E8946F936E7FBA
:104D60006E5F7F4F8F4F9F4FAF4FB1E03ED0B4E0AB
:104D70003CD0670F781F891F9A1FA11D680F791FEC
:104D80008A1F911DA11D6A0F711D811D911DA11DFD
:104D900020D009F468943F912AE0269F112430190D
:104DA000305D3193DEF6CF010895462F4770405DA8
:104DB0004193B3E00FD0C9F7F6CF462F4F70405D57
:104DC0004A3318F0495D31FD4052419302D0A9F7B2
:104DD000EACFB4E0A6959795879577956795BA95AC
:104DE000C9F700976105710508959B01AC010A2E72
:104DF00006945795479537952795BA95C9F7620F49
:104E0000731F841F951FA01D08958F929F92AF92CC
:104E1000BF92CF92DF92EF92FF920F931F93DF9397
:104E2000CF93CDB7DEB727970FB6F894DEBF0FBE8E
:104E3000CDBF6C017B018A0160E070E0A0E0B0E0D2
:104E400084E0A82EB12CAC0EBD1EF4E08F2E912C68
:104E50008A0C9B1C66C0F70180818D3309F465C004
:104E6000F501E60FF71F80836F5F7F4F6430710598
:104E700009F052C0F5019081892F81548A31A0F048
:104E800080528A3110F4865E0FC0892F80538A3099
:104E900010F48C5C09C09B3211F48EE305C09F3284
:104EA00011F08FEF01C08FE38193E815F90519F731
:104EB0002D8130E0C90180739070E4E0959587956D
:104EC000EA95E1F76C81660F660F680F69838E8142
:104ED00090E0AC014C7350705595479555954795AA
:104EE00054E0220F331F5A95E1F7420F4A8326E020
:104EF000880F991F2A95E1F72F81280F2B83F60140
:104F0000EA0FFB1F60831196F601EA0FFB1F408337
:104F10002183129660E070E00894E11CF11C0150BE
:104F200010400115110509F096CF6115710509F4BE
:104F30006CC0FE013496E60FF71FCB0102C0119240
:104F4000019684309105DCF3FE0134969F012C5FBD
:104F50003F4F9081892F81548A31A0F080528A314D
:104F600010F4865E0FC0892F80538A3010F48C5C59
:104F700009C09B3211F48EE305C09F3211F08FEF10
:104F800001C08FE38193E217F30719F74D8150E0D9
:104F9000CA0180739070F4E095958795FA95E1F7D2
:104FA0002C81220F220F280F29832E8130E0C90186
:104FB0008C739070959587959595879594E0440F9F
:104FC000551F9A95E1F7840F8A8386E0220F331FDD
:104FD0008A95E1F78F81820F8B83A6014A0F5B1FB1
:104FE00020E030E0615070408E010F5F1F4F0AC01B
:104FF000F801E20FF31F8081FA018193AF0111964E
:105000002F5F3F4F261737079CF3CA0EDB1EF601B2
:105010001082CD0127960FB6F894DEBF0FBECDBF2C
:10502000CF91DF911F910F91FF90EF90DF90CF9084
:10503000BF90AF909F908F900895FC0112821382D1
:105040000895FC018381882311F081E08283089513
:10505000FC018281811112820895CF93DF93DC01DC
:10506000FC01EB55FE4F808191810097C9F10197BA
:1050700091838083ED01CC5ADF4FFD01ED58FF4F46
:105080008BE1019009928150E1F7FD01EE5AFF4F4B
:10509000AF58BF4F8D919C911197A157B04091830C
:1050A0008083FD01ED58FF4F20E030E0AD014B550E
:1050B0005E4F10C02F5F3F4FEF01DF015F968BE126
:1050C0000D9009928150E1F7858D968D32979183ED
:1050D0008083B196DA018D919C912817390750F39E
:1050E000DF91CF910895FC018AE695E0918380835A
:1050F0008781882321F0CF0104960C9418830895AA
:105100000F931F93CF93DF938C010E94DE900E9438
:10511000BB90C80182539E4F0E941883F8011282EF
:105120008FE291E00E94F6668091080B882301F1DE
:105130001092080B8091B508C82FD0E0CC0FDD1F6E
:10514000CF56D84E68817981882777FD8095982F32
:105150000E9497EB2091B7043091B8044091B904B4
:105160005091BA040E9403ED181614F419821882A3
:10517000DF91CF911F910F910895CF92DF92EF921F
:10518000FF920F931F93DF93CF93CDB7DEB76F9747
:105190000FB6F894DEBF0FBECDBF8C016B01095A6C
:1051A0001F4FD8018C9107551040882321F43FE20E
:1051B000E32EF12C03C020E5E22EF12CE00EF11ECF
:1051C0008AE695E09A8389831C821B8218861D8259
:1051D000B7016C5F7F4FCE010596A60121E00E94CA
:1051E000048A882391F5EBE3F1E0949108C0809163
:1051F000C00085FFFCCF9093C6003196949199230F
:10520000B1F7E1E4F1E0949108C08091C00085FF1E
:10521000FCCF9093C600319694919923B1F709C0C1
:105220008091C00085FFFCCF0894C11CD11C9093D5
:10523000C600F6019081992399F78091C00085FFFF
:10524000FCCF8AE08093C6005AC0F801EB55FE4FB0
:10525000208131812A30310508F040C02F5F3F4F57
:105260003183208321503040F90195E0EE0FFF1F7C
:105270009A95E1F7E21BF30BED58FF4FE00FF11F9A
:1052800013C0AF01415E5F4FBF018BE1DB010D90A9
:10529000BD01DA010D92AD018150C1F79291829169
:1052A0003296968F858F7F9721503040BFEF2E3FEB
:1052B0003B0739F7D801AD58BF4FF70134968BE162
:1052C00001900D928150E1F70F581F4FF701828135
:1052D0009381D8018D939C9301571040D801AC5A0B
:1052E000BF4FFE0135968BE101900D928150E1F7A1
:1052F0000E5A1F4F8B819C81F80191838083CE01D0
:105300000196F1DE6F960FB6F894DEBF0FBECDBFEB
:10531000CF91DF911F910F91FF90EF90DF90CF9091
:105320000895EF92FF920F931F938C014EECE42EA1
:1053300041E0F42EE80EF91EC7010E94C982C701A0
:105340000E941883F801108211821F910F91FF9023
:10535000EF900895CF92DF92EF92FF920F931F93F9
:10536000CF93DF937C016B01DB010D900020E9F707
:105370008D0101501040061B170BEEECF1E0EE0E14
:10538000FF1ED7011C92E2E3FEEFEE0EFF1ECB01E3
:105390006EE470E078DAEC01009731F4F8013197AF
:1053A000EC0DFD1D86010CC060E270E06CDA8C0132
:1053B0000F5F1F4FCE016AE270E065DAFC013197A2
:1053C0008DE081838AE082831382C70186539E4FDA
:1053D000B8010E94FD8A8EEC91E0E80EF91ED7011B
:1053E0008C91882319F1EBE6F1E0949108C080914B
:1053F000C00085FFFCCF9093C6003196949199230D
:10540000B1F7E2E7F1E0949108C08091C00085FF18
:10541000FCCF9093C600319694919923B1F7809177
:10542000C00085FFFCCF8AE08093C600DF91CF915A
:105430001F910F91FF90EF90DF90CF900895CF9341
:10544000DF93EC018B81882309F43BC0EAE9F1E0AA
:10545000949108C08091C00085FFFCCF9093C60056
:10546000319694919923B1F7CF50DE4F48815981FD
:105470006A817B81C15FD14086E896E02AE030E016
:105480000E94A23FE8E9F1E0949108C08091C00039
:1054900085FFFCCF9093C600319694919923B1F784
:1054A000C751DE4F488159816A817B8186E896E049
:1054B0002AE030E00E94A23F8091C00085FFFCCF2F
:1054C00012C0E8E8F1E0949108C08091C00085FF27
:1054D000FCCF9093C600319694919923B1F78091B7
:1054E000C00085FFFCCF8AE08093C600DF91CF919A
:1054F00008952F923F924F925F926F927F928F9278
:105500009F92AF92BF92CF92DF92EF92FF920F9352
:105510001F93DF93CF93CDB7DEB7AC970FB6F89458
:10552000DEBF0FBECDBF5C014B01FC018381882330
:1055300009F434C1C50182539E4F0E941883F501BE
:1055400012821A8A1D8A198A188A8AE695E09F872C
:105550008E876EE4C62ED12CCA0CDB1C2FE230E005
:10556000A20EB31EF601B182A08221ED3FEFA20E82
:10557000B31EF40180818F3209F08DC0C4016FE247
:1055800070E081D97C010894E11CF11C3E01089473
:10559000611C711C260152E1252E312C2C0E3D1E62
:1055A00075C0C7016FE270E06ED96C01009709F415
:1055B00080C0E816F90608F07CC08C010E191F099E
:1055C000C301B701A8017FD9060D171DF80110828C
:1055D000F30107C08091C00085FFFCCF3196909306
:1055E000C60090819923B1F78091C00085FFFCCF60
:1055F000FAE0F093C600F2016081718161157105D6
:1056000019F460E070E002C06C5F7F4FC101A3013C
:1056100021E00E94048A882371F5E6EDF1E094917F
:1056200008C08091C00085FFFCCF9093C6003196E2
:1056300094919923B1F7FE01319607C08091C00083
:1056400085FFFCCF31969093C60090819923B1F7E6
:10565000E4EDF1E0949108C08091C00085FFFCCF9B
:105660009093C600319694919923B1F78091C00030
:1056700085FFFCCF8DC02EE030E02C0F3D1FF201E6
:105680003183208376010894E11CF11CE114F104BC
:1056900009F087CF0BC080E590E0A80EB91EF60197
:1056A000B182A08220EB3FEFA20EB31ED82C092DB1
:1056B00002C0DE2C0F2D8EE490E0A80EB91EF5017D
:1056C0008081918122EB3FEFA20EB31E009719F467
:1056D00080E090E001C004966D2D702F0E94D08A6A
:1056E000882339F1E6ECF1E0949108C08091C00084
:1056F00085FFFCCF9093C600319694919923B1F722
:105700008D2D902F9C01F90107C08091C00085FF6D
:10571000FCCF31969093C60090819923B1F781EF29
:1057200091E0A80EB91EF501108211821282138237
:1057300032C0EEEAF1E0949108C08091C00085FF8C
:10574000FCCF9093C600319694919923B1F78D2D9B
:10575000902F9C01F90107C08091C00085FFFCCF0C
:1057600031969093C60090819923B1F7ECEAF1E06D
:10577000949108C08091C00085FFFCCF9093C60033
:10578000319694919923B1F78091C00085FFFCCFA9
:105790008AE08093C600CE010E96A5DCAC960FB6CB
:1057A000F894DEBF0FBECDBFCF91DF911F910F9157
:1057B000FF90EF90DF90CF90BF90AF909F908F9031
:1057C0007F906F905F904F903F902F9008952F9211
:1057D0003F924F925F926F927F928F929F92AF9281
:1057E000BF92CF92DF92EF92FF920F931F93DF93BE
:1057F000CF93CDB7DEB7AD970FB6F894DEBF0FBE2F
:10580000CDBF5C014B014DA7FC018381882309F4C6
:10581000E5C1EEEC4E2EE1E05E2E4A0C5B1CC201AF
:105820000E941883F50112821A8A1D8A198A188A21
:105830008AE695E09F878E877EE4C72ED12CCA0C1E
:10584000DB1C8FE290E0A80EB91EF601B182A082A7
:1058500081ED9FEFA80EB91EF40180818F3209F00F
:1058600089C0C4016FE270E00ED87C010894E11C8D
:10587000F11C3E010894611C711C160176C0C70121
:105880006FE270E000D86C01009709F481C0E8165F
:10589000F90608F07DC08C010E191F09C301B7017C
:1058A000A80111D8060D171DF8011082F30107C0D9
:1058B0008091C00085FFFCCF31969093C600908107
:1058C0009923B1F78091C00085FFFCCFFAE0F093F7
:1058D000C600F101608171816115710519F460E004
:1058E00070E002C06C5F7F4FCE014296A30121E0C1
:1058F0000E94048A882371F5EEE4F2E0949108C0D6
:105900008091C00085FFFCCF9093C60031969491A2
:105910009923B1F7FE01319607C08091C00085FF41
:10592000FCCF31969093C60090819923B1F7ECE4B7
:10593000F2E0949108C08091C00085FFFCCF909365
:10594000C600319694919923B1F78091C00085FFEC
:10595000FCCF15C18EE090E08C0F9D1FF10191836B
:10596000808376010894E11CF11CE114F10409F034
:1059700086CF0BC0E0E5F0E0AE0EBF1EF601B182AF
:10598000A08280EB9FEFA80EB91E082DF92C01C054
:105990000E2DF501E25BFF4F9DA5992309F4ADC0E3
:1059A000608171816115710519F460E070E002C0D9
:1059B0006C5F7F4FC201402F5F2D21E00E94048A5F
:1059C000882309F46AC0EFEDF1E0AE0EBF1EF501C9
:1059D00040815181628173818AE090E0A80EB91EF6
:1059E000F501408351836283738387E19EEFA80EA4
:1059F000B91EEEE3F2E0949108C08091C00085FFEB
:105A0000FCCF9093C600319694919923B1F7802FE3
:105A10009F2D9C01F90107C08091C00085FFFCCF3C
:105A200031969093C60090819923B1F7E6E3F2E0B6
:105A3000949108C08091C00085FFFCCF9093C60070
:105A4000319694919923B1F786E896E02AE030E008
:105A50000E94A23F8091C00085FFFCCF8AE0809326
:105A6000C600E1EFF1E0AE0EBF1EF501108211821B
:105A700012821382E8E2F2E0949108C08091C000A3
:105A800085FFFCCF9093C600319694919923B1F78E
:105A90008091C00085FFFCCF97C0E4E1F2E09491D3
:105AA00008C08091C00085FFFCCF9093C60031965E
:105AB00094919923B1F7802F9F2D9C01F90107C084
:105AC0008091C00085FFFCCF31969093C6009081F5
:105AD0009923B1F7E2E1F2E0949108C08091C0000F
:105AE00085FFFCCF9093C600319694919923B1F72E
:105AF0008091C00085FFFCCF42C06081718161153B
:105B0000710519F460E070E002C06C5F7F4FC20164
:105B1000402F5F2D26E50E94048A882309F033C0B8
:105B2000EEEFF1E0949108C08091C00085FFFCCFBA
:105B30009093C600319694919923B1F7802F9F2DB1
:105B40009C01F90107C08091C00085FFFCCF319610
:105B50009093C60090819923B1F7ECEFF1E0949116
:105B600008C08091C00085FFFCCF9093C60031969D
:105B700094919923B1F78091C00085FFFCCF8AE012
:105B80008093C60028C081E0F5018083EAEEF1E051
:105B9000949108C08091C00085FFFCCF9093C6000F
:105BA000319694919923B1F7F40107C08091C00018
:105BB00085FFFCCF31969093C60090819923B1F771
:105BC0008091C00085FFFCCF8AE08093C600802FC3
:105BD0009F2D0E9459D7CE010E9685DAAD960FB64D
:105BE000F894DEBF0FBECDBFCF91DF911F910F9113
:105BF000FF90EF90DF90CF90BF90AF909F908F90ED
:105C00007F906F905F904F903F902F900895FC0190
:105C100081E08183CF0140E0DACDEF92FF920F93D4
:105C20001F93CF93DF938C01FC01138286A98823F5
:105C300021F0C801C3960E941883F7EAEF2EF1E025
:105C4000FF2EE00EF11EC70160E045E30E94C58013
:105C5000882309F5EBE3F1E0949108C08091C0003E
:105C600085FFFCCF9093C600319694919923B1F7AC
:105C7000E0E9F2E0949108C08091C00085FFFCCF7C
:105C80009093C600319694919923B1F78091C0000A
:105C900085FFFCCF7DC0E801C455DE4FCE01B701C2
:105CA00041E00E948E8B882341F5CE01B70140E090
:105CB0000E948E8B882309F5EBE6F1E0949108C0F1
:105CC0008091C00085FFFCCF9093C60031969491DF
:105CD0009923B1F7EDE7F2E0949108C08091C000FC
:105CE00085FFFCCF9093C600319694919923B1F72C
:105CF0008091C00085FFFCCF4BC0C801C396BE0198
:105D00000E940A86882309F5EBE6F1E0949108C029
:105D10008091C00085FFFCCF9093C600319694918E
:105D20009923B1F7EDE6F2E0949108C08091C000AC
:105D300085FFFCCF9093C600319694919923B1F7DB
:105D40008091C00085FFFCCF23C081E0F8018383F0
:105D5000EBE3F1E0949108C08091C00085FFFCCF97
:105D60009093C600319694919923B1F7E2E6F2E060
:105D7000949108C08091C00085FFFCCF9093C6002D
:105D8000319694919923B1F78091C00085FFFCCFA3
:105D90008AE08093C600D801AC5ABF4FF801F39651
:105DA0008BE101900D928150E1F7F80181A992A950
:105DB0000E5A1F4FF8019183808302551040C8018D
:105DC0008F96025B1F4FF80191838083DF91CF9103
:105DD0001F910F91FF90EF9008952F923F924F9255
:105DE0005F926F927F929F92AF92BF92CF92DF921B
:105DF000EF92FF920F931F93DF93CF93CDB7DEB750
:105E0000CC55D0400FB6F894DEBF0FBECDBF6C01AD
:105E1000662311F525EF31E0C20ED31ED6018C9119
:105E2000EBE0FEEFCE0EDF1E882309F4E3C02DEE7B
:105E300031E0C20ED31ED601ED90FD900D911C9164
:105E4000E3E1FEEFCE0EDF1E0E9476E3E616F706D4
:105E50000807190708F4CEC025EF31E0C20ED31EA3
:105E6000D6011C92EBE0FEEFCE0EDF1ED60113969C
:105E70008C91882339F4C601D0DEF6018381882312
:105E800009F4B8C000D000D0EDB7FEB731967E015E
:105E90000894E11CF11CADB7BEB71296FC92EE92CD
:105EA000119782E691E093838283D6019D968D912E
:105EB0009C919E97958384830E9472248701EDB7FD
:105EC000FEB736960FB6F894FEBF0FBEEDBF570172
:105ED0000AC0D8018C91992787FD90950E9438EFD0
:105EE000F80181938F01F50101900020E9F73197C6
:105EF000EA19FB09802F8E198E175CF303E3A02E9D
:105F0000B12CAC0CBD1CC50140E050E060E070E07D
:105F10000E94FF8199241DE3E12EF12CEC0EFD1E61
:105F20002E010894411C511CBFE16B2E712C6C0E8C
:105F30007D1EABE52A2EA1E03A2E42C0D8018C91FD
:105F400090E00E9438EFF80181938F01D7010D9006
:105F50000020E9F71197AE19BF09802F8E198A1713
:105F60006CF327968FAD27978E3751F1C701B20199
:105F700045E050E00E945524009711F500D000D074
:105F8000EDB7FEB73196ADB7BEB712967C926E9262
:105F9000119733822282558244820E947224EDB787
:105FA000FEB736960FB6F894FEBF0FBEEDBFC30125
:105FB0000E946F6787E591E00E94F66699249394AA
:105FC000C501B70140E050E00E942985181614F47D
:105FD0008701BCCF992041F48FEF9FEFD6019E96A9
:105FE0009C938E939D9706C0F60185A596A5019674
:105FF00096A785A7C45ADF4F0FB6F894DEBF0FBE31
:10600000CDBFCF91DF911F910F91FF90EF90DF9067
:10601000CF90BF90AF909F907F906F905F904F9088
:106020003F902F9008952F923F924F925F926F92E0
:106030007F928F929F92AF92BF92CF92DF92EF9218
:10604000FF920F931F93DF93CF93CDB7DEB7CF5857
:10605000D0400FB6F894DEBF0FBECDBF8C013B0120
:106060006A0184E090E0C80ED91EF8017196C75706
:10607000DF4FF983E883C958D040C8010496CA5756
:10608000DF4F99838883C658D040C857DF4F1882A6
:10609000C858D04046E6E42EF12CEC0EFD1EF70168
:1060A0003B96C557DF4FF983E883CB58D04036EF96
:1060B000832E31E0932E800E911E28EFA22E21E038
:1060C000B22EA00EB11E9EE0292E312C2C0E3D1EAC
:1060D00087E4482E512C4C0E5D1EC2010496C35716
:1060E000DF4F99838883CD58D040EBE3F1E0949162
:1060F000C157DF4F9883CF58D0404EC1F7018385F9
:10610000482F50E0BA01687170706031710509F074
:1061100051C1F401208131812130310509F44AC196
:106120002230310509F446C1F701DE011196908154
:10613000903239F08E2F8E19883011F48EE28D93C3
:106140009D933196C557DF4F88819981CB58D040B8
:10615000E817F90761F71C921E86F30180818823F6
:1061600029F4C10160E072E00E943824C101B3014A
:106170000E943824C101BE016F5F7F4F0E94382406
:10618000C10160E072E00E9438241CA61FA61BA675
:106190001AA68AE695E099A788A7CE018C96B60143
:1061A000AE014F5F5F4F21E00E94048A882309F00F
:1061B0003FC0F40180819181892BD1F5C157DF4F18
:1061C0009881CF58D040EBE3F1E008C08091C00047
:1061D00085FFFCCF9093C600319694919923B1F737
:1061E000E2E0F2E007C08091C00085FFFCCF31966D
:1061F0009093C60090819923B1F78091C00085FFEC
:10620000FCCFFAE0F093C600FE01319607C0809102
:10621000C00085FFFCCF31969093C60090819923F2
:10622000B1F78091C00085FFFCCF8AE08093C60063
:10623000C357DF4FA881B981CD58D040FE01BC962D
:106240008BE101900D928150E1F78AA59BA5F201A7
:10625000938382838AE695E091838083C801B101AC
:10626000A201E1DEC2010E947328CE0188960E943D
:10627000732892C0953E09F48FC09E3209F48CC0F9
:106280009F3509F489C0F8019189992331F09E3234
:1062900009F482C09F3509F47FC043FD7DC080E0D2
:1062A0006031710509F481E0F80184A7882349F47D
:1062B000F7018085873409F06FC081858E3709F436
:1062C0006BC0CA57DF4FA881B981C658D040F701CB
:1062D0008081803241F08E2F8E19883011F48EE249
:1062E0008D9380818D933196C557DF4F8881998139
:1062F000CB58D040E817F90759F71C92F401808178
:106300009181009729F5F30107C08091C00085FFB6
:10631000FCCF31969093C60090819923B1F7CA576C
:10632000DF4FE881F981C658D04007C08091C00096
:1063300085FFFCCF31969093C60090819923B1F7E9
:106340008091C00085FFFCCFFAE0F093C60024C026
:106350008130910539F4F501808191810196918315
:1063600080831AC00297C1F4C857DF4FF881C8581C
:10637000D0402F2F30E0F501808191812817390717
:10638000F1F0C857DF4FF881C858D040FF5FC857B9
:10639000DF4FF883C858D040C601B701C757DF4F59
:1063A00048815981C958D0400E94298518160CF49B
:1063B000A5CE05C0F7019081992309F05BCFC157A5
:1063C000DF4F0FB6F894DEBF0FBECDBFCF91DF9188
:1063D0001F910F91FF90EF90DF90CF90BF90AF9003
:1063E0009F908F907F906F905F904F903F902F90F5
:1063F0000895EF92FF920F931F93DF93CF93CDB742
:10640000DEB76F970FB6F894DEBF0FBECDBF7C012D
:106410008C01025B1F4F805B9F4FF801918380834B
:1064200026EF31E0E20EF31E21E030E0F701219388
:1064300031937F011182108228E03EEFE20EF31EBD
:10644000049640E050E060E070E00E94FF81F801B7
:1064500020813181DE011596F90134968BE101909E
:106460000D928150E1F7F901828193819C838B83A6
:106470008AE695E09A838983C70165E172E08E011F
:106480000F5F1F4FA801CFDDC8010E947328F701DD
:10649000E850FE4F808191816F960FB6F894DEBF71
:1064A0000FBECDBFCF91DF911F910F91FF90EF9065
:1064B0000895EF92FF920F931F93DF93CF93CDB781
:1064C000DEB76F970FB6F894DEBF0FBECDBF7C016D
:1064D0008C01025B1F4F805B9F4FF801918380838B
:1064E00026EF31E0E20EF31E22E030E0F7013183C7
:1064F00020832AE03EEFE20EF31EF701E850FE4F44
:1065000060831182049640E050E060E070E00E94F9
:10651000FF81F80120813181DE011596F901349661
:106520008BE101900D928150E1F7F9018281938115
:106530009C838B838AE695E09A838983C70165E112
:1065400072E08E010F5F1F4FA8016DDDC8010E9430
:1065500073286F960FB6F894DEBF0FBECDBFCF91F4
:10656000DF911F910F91FF90EF900895EF92FF92AE
:106570000F931F93DF93CF93CDB7DEB76F970FB60F
:10658000F894DEBF0FBECDBF7C0186EF91E0E80E30
:10659000F91EF701118210828AE09EEFE80EF91EC3
:1065A00087010D5C1F4FC80140E050E060E070E0E3
:1065B0000E94FF81DE011596F8018BE101900D929A
:1065C0008150E1F7F70181A992A99C838B838AE628
:1065D00095E09A838983C70165E172E08E010F5FC0
:1065E0001F4FA80120DDC8010E9473286F960FB6C7
:1065F000F894DEBF0FBECDBFCF91DF911F910F91F9
:10660000FF90EF9008950F931F93CF93DF93DC01DA
:10661000D3961C92D397D6961C92D697D2961C925C
:106620001E92D1978AE695E0D0969C938E939F9781
:10663000AC5ABF4F1C9213961C92A755B040FD0157
:10664000E05BFF4FAE5ABF4F11961C921E92A255AF
:10665000B04091838083ED01C159DF4FFE0120E0FE
:1066600030E0482F14821782138212824083918374
:10667000215E3F4F7F9681E02633380799F7A85572
:10668000BE4F89E18C9313961C9258961C921B96D0
:106690001C9213961C92A15DB140FD01E653FE4F82
:1066A000A453BE4F11961C921E92408391835D9617
:1066B0001D921D921D921C92139718961D921D9269
:1066C0001D921C921397A15FB14012961C921297D3
:1066D00013961C9213971C9211961C9211978D0180
:1066E00003511E4FF8011082118212821382AB55A2
:1066F000BE4F11961C921E92FE01C9011192019784
:10670000E9F7A05BBF4F81E08C93A55FB1409E96F7
:106710001C921E929D970E9476E368577C4E8F4F85
:106720009F4FF8016083718382839383DF91CF91C0
:106730001F910F910895DF93CF93CDB7DEB72897C0
:106740000FB6F894DEBF0FBECDBF809116029091B8
:106750001702A0911802B091190289839A83AB8322
:10676000BC83FE01319684E690E02081F999FECF4A
:106770001FBA92BD81BD20BD0FB6F894FA9AF99A5E
:106780000FBE01968836910511F03196EECFECEAF6
:10679000FAE02081F999FECF1FBA92BD81BD20BDDC
:1067A0000FB6F894FA9AF99A0FBE019688379105B8
:1067B00011F03196EECFECE9FAE02081F999FECFA5
:1067C0001FBA92BD81BD20BD0FB6F894FA9AF99A0E
:1067D0000FBE01968838910511F03196EECFECEBA3
:1067E000FAE02081F999FECF1FBA92BD81BD20BD8C
:1067F0000FB6F894FA9AF99A0FBE01968839910566
:1068000011F03196EECFE0EDFAE02081F999FECF5C
:106810001FBA92BD81BD20BD0FB6F894FA9AF99ABD
:106820000FBE01968C39910511F03196EECFE4ED53
:10683000FAE02081F999FECF1FBA92BD81BD20BD3B
:106840000FB6F894FA9AF99A0FBE0196803A91051C
:1068500011F03196EECFECECFAE02081F999FECF01
:106860001FBA92BD81BD20BD0FB6F894FA9AF99A6D
:106870000FBE0196843A910511F03196EECFE4EE09
:10688000FAE02081F999FECF1FBA92BD81BD20BDEB
:106890000FB6F894FA9AF99A0FBE0196883A9105C4
:1068A00011F03196EECFE8E9FAE02081F999FECFB8
:1068B0001FBA92BD81BD20BD0FB6F894FA9AF99A1D
:1068C0000FBE01968C3A910511F03196EECFE8EDAE
:1068D000FAE02081F999FECF1FBA92BD81BD20BD9B
:1068E0000FB6F894FA9AF99A0FBE0196803B91057B
:1068F00011F03196EECFECEDFAE02081F999FECF60
:106900001FBA92BD81BD20BD0FB6F894FA9AF99ACC
:106910000FBE0196843B910511F03196EECFE0EE6B
:10692000FAE02081F999FECF1FBA92BD81BD20BD4A
:106930000FB6F894FA9AF99A0FBE0196883B910522
:1069400011F03196EECFEDE9F8E02081F999FECF14
:106950001FBA92BD81BD20BD0FB6F894FA9AF99A7C
:106960000FBE0196843C910511F03196EECFEEEA10
:10697000F5E02081F999FECF1FBA92BD81BD20BDFF
:106980000FB6F894FA9AF99A0FBE0196863C9105D3
:1069900011F03196EECFEDEDF7E12081F999FECFC0
:1069A0001FBA92BD81BD20BD0FB6F894FA9AF99A2C
:1069B0000FBE0196883C910511F03196EECFEFEDB8
:1069C000F7E12081F999FECF1FBA92BD81BD20BDAC
:1069D0000FB6F894FA9AF99A0FBE01968A3C91057F
:1069E00011F03196EECFE1EEF7E12081F999FECF7B
:1069F0001FBA92BD81BD20BD0FB6F894FA9AF99ADC
:106A00000FBE01968C3C910511F03196EECFE3EE6E
:106A1000F7E12081F999FECF1FBA92BD81BD20BD5B
:106A20000FB6F894FA9AF99A0FBE01968E3C91052A
:106A300011F03196EECFE5EEF7E12081F999FECF26
:106A40001FBA92BD81BD20BD0FB6F894FA9AF99A8B
:106A50000FBE0196803D910511F03196EECFE7EE25
:106A6000F7E12081F999FECF1FBA92BD81BD20BD0B
:106A70000FB6F894FA9AF99A0FBE0196823D9105E5
:106A800011F03196EECFE4ECF4E02081F999FECFDD
:106A90001FBA92BD81BD20BD0FB6F894FA9AF99A3B
:106AA0000FBE0196863D910511F03196EECFE8ECD0
:106AB000F4E02081F999FECF1FBA92BD81BD20BDBF
:106AC0000FB6F894FA9AF99A0FBE01968A3D91058D
:106AD00011F03196EECFECECF4E02081F999FECF85
:106AE0001FBA92BD81BD20BD0FB6F894FA9AF99AEB
:106AF0000FBE01968E3D910511F03196EECFEAEE74
:106B0000F9E12081F999FECF1FBA92BD81BD20BD68
:106B10000FB6F894FA9AF99A0FBE8F3D910521F0BD
:106B200031968FED90E0EDCF80911A0290911B028B
:106B3000A0911C02B0911D028D839E83AF83B88704
:106B4000FE01359684E690E02081F999FECF1FBAC8
:106B500092BD81BD20BD0FB6F894FA9AF99A0FBE86
:106B60008736910519F001963196EECFEDE9F2E006
:106B7000949108C08091C00085FFFCCF9093C6001F
:106B8000319694919923B1F7E1EDF4E0949108C026
:106B90008091C00085FFFCCF9093C6003196949100
:106BA0009923B1F78091C00085FFFCCF8AE08093E4
:106BB000C60028960FB6F894DEBF0FBECDBFCF91AA
:106BC000DF910895DF93CF93CDB7DEB7AC970FB6C3
:106BD000F894DEBF0FBECDBFDE011196EEE1F5E009
:106BE0008CE001900D928150E1F7DE011D96EEE000
:106BF000F5E080E101900D928150E1F7DE015D96B4
:106C0000EEEFF4E080E101900D928150E1F789818F
:106C10009A81AB81BC818093AC0A9093AD0AA0931A
:106C2000AE0AB093AF0A2D853E854F8558892093D3
:106C30009C0A30939D0A40939E0A50939F0A8D8D23
:106C40009E8DAF8DB8A18093BC0A9093BD0AA0938E
:106C5000BE0AB093BF0A8D819E81AF81B8858093B3
:106C6000B00A9093B10AA093B20AB093B30A89898B
:106C70009A89AB89BC898093A00A9093A10AA093BA
:106C8000A20AB093A30A89A19AA1ABA1BCA1809347
:106C9000C00A9093C10AA093C20AB093C30A89851F
:106CA0009A85AB85BC858093B40A9093B50AA0936E
:106CB000B60AB093B70A8D899E89AF89B88D809343
:106CC000A40A9093A50AA093A60AB093A70A8DA13F
:106CD0009EA1AFA1B8A58093C40A9093C50AA093C2
:106CE000C60AB093C70A2093B80A3093B90A4093F2
:106CF000BA0A5093BB0A898D9A8DAB8DBC8D809357
:106D0000A80A9093A90AA093AA0AB093AB0A89A5EE
:106D10009AA5ABA5BCA58093C80A9093C90AA09375
:106D2000CA0AB093CB0A0E948A6C80E090E0A6E188
:106D3000B4E48093D00A9093D10AA093D20AB0937E
:106D4000D30A8093D40A9093D50AA093D60AB0931D
:106D5000D70A20E030E040E050E02093CC0A3093A6
:106D6000CD0A4093CE0A5093CF0A80E29EE4A0E081
:106D7000B0E08093980A9093990AA0939A0AB093EE
:106D80009B0A2093E40A3093E50A4093E60A509365
:106D9000E70A80E090E0A0EAB1E48093D80A9093FB
:106DA000D90AA093DA0AB093DB0A8DEC9CECACEC28
:106DB000BEE38093DC0A9093DD0AA093DE0AB093D1
:106DC000DF0A80E090E0A0EAB0E48093E00A9093CC
:106DD000E10AA093E20AB093E30A2093A508309356
:106DE000A6084093A7085093A8082093A1083093C1
:106DF000A2084093A3085093A40820939D083093C1
:106E00009E0840939F085093A00884EB90E09093D5
:106E1000DE178093DD1786E490E09093E01780936F
:106E2000DF172FEF30E03093E2172093E11780EF68
:106E300090E09093E4178093E31784E690E09093BA
:106E4000E6178093E5173093E8172093E7178FE054
:106E500090E09093EB198093EA198AE999E9A1EB04
:106E6000B1E48093C4049093C504A093C604B09386
:106E7000C70461E77DE38AE89FE30E94C09A6093BC
:106E8000C8047093C9048093CA049093CB0460E053
:106E900070E084EE92E40E94CC9A6093CC047093EC
:106EA000CD048093CE049093CF040E947A9A80E020
:106EB00090E0A0E8BFE38093D0049093D104A09326
:106EC000D204B093D304EDE9F2E0949108C080912C
:106ED000C00085FFFCCF9093C60031969491992312
:106EE000B1F7E3EAF2E0949108C08091C00085FF19
:106EF000FCCF9093C600319694919923B1F780917D
:106F0000C00085FFFCCF8AE08093C600AC960FB628
:106F1000F894DEBF0FBECDBFCF91DF910895CF9320
:106F2000DF93CDE9D2E0FE01949108C08091C000CA
:106F300085FFFCCF9093C600319694919923B1F7C9
:106F4000E1ECF4E0949108C08091C00085FFFCCF93
:106F50009093C600319694919923B1F78091C00027
:106F600085FFFCCF8AE08093C600FE019491EDE995
:106F7000F2E008C08091C00085FFFCCF9093C6006E
:106F8000319694919923B1F74091AC0A5091AD0A92
:106F90006091AE0A7091AF0A89EB94E00E94374786
:106FA0004091B00A5091B10A6091B20A7091B30A4F
:106FB00086EB94E00E9437474091B40A5091B50A9D
:106FC0006091B60A7091B70A83EB94E00E9437474C
:106FD0004091B80A5091B90A6091BA0A7091BB0AFF
:106FE00080EB94E00E943747EEE1F2E007C0809129
:106FF000C00085FFFCCF31969093C6009081992305
:10700000B1F78091C00085FFFCCF8AE08093C60075
:10701000FE019491EDE9F2E008C08091C00085FF87
:10702000FCCF9093C600319694919923B1F7E6E98D
:10703000F4E0949108C08091C00085FFFCCF90934C
:10704000C600319694919923B1F78091C00085FFD5
:10705000FCCF8AE08093C600FE019491EDE9F2E056
:1070600008C08091C00085FFFCCF9093C600319688
:1070700094919923B1F740919C0A50919D0A609197
:107080009E0A70919F0A8DE894E00E9437474091D4
:10709000A00A5091A10A6091A20A7091A30A8AE8FD
:1070A00094E00E9437474091A40A5091A50A60914C
:1070B000A60A7091A70A87E894E00E94374740919A
:1070C000A80A5091A90A6091AA0A7091AB0A84E8B3
:1070D00094E00E943747EEE1F2E007C08091C000E3
:1070E00085FFFCCF31969093C60090819923B1F72C
:1070F0008091C00085FFFCCF8AE08093C600FE012E
:107100009491EDE9F2E008C08091C00085FFFCCFCA
:107110009093C600319694919923B1F7E6E6F4E096
:10712000949108C08091C00085FFFCCF9093C60069
:10713000319694919923B1F78091C00085FFFCCFDF
:107140008AE08093C600FE019491EDE9F2E008C068
:107150008091C00085FFFCCF9093C600319694913A
:107160009923B1F74091BC0A5091BD0A6091BE0AC3
:107170007091BF0A8DE594E00E9449474091C00A92
:107180005091C10A6091C20A7091C30A8AE594E0E5
:107190000E9449474091C40A5091C50A6091C60AAD
:1071A0007091C70A87E594E00E9449474091C80A58
:1071B0005091C90A6091CA0A7091CB0A84E594E0A3
:1071C0000E944947EEE1F2E007C08091C00085FFD0
:1071D000FCCF31969093C60090819923B1F78091AE
:1071E000C00085FFFCCF8AE08093C600FE01949129
:1071F000EDE9F2E008C08091C00085FFFCCF9093DC
:10720000C600319694919923B1F7EFE1F4E094919F
:1072100008C08091C00085FFFCCF9093C6003196D6
:1072200094919923B1F78091C00085FFFCCF8AE04B
:107230008093C600FE019491EDE9F2E008C08091D0
:10724000C00085FFFCCF9093C6003196949199239E
:10725000B1F74091D00A5091D10A6091D20A709151
:10726000D30A86E194E00E9437474091D40A5091B6
:10727000D50A6091D60A7091D70A83E194E00E9402
:107280003747EEE1F2E007C08091C00085FFFCCFF8
:1072900031969093C60090819923B1F78091C000F8
:1072A00085FFFCCF8AE08093C600FE019491EDE952
:1072B000F2E008C08091C00085FFFCCF9093C6002B
:1072C000319694919923B1F7E0E6F3E0949108C0E8
:1072D0008091C00085FFFCCF9093C60031969491B9
:1072E0009923B1F78091C00085FFFCCF8AE080939D
:1072F000C600FE019491EDE9F2E008C08091C00063
:1073000085FFFCCF9093C600319694919923B1F7F5
:107310004091CC0A5091CD0A6091CE0A7091CF0A6B
:1073200087E593E00E9437474091E40A5091E50ACF
:107330006091E60A7091E70A84E593E00E9437477E
:107340004091980A5091990A60919A0A70919B0A0B
:1073500081E593E00E9449474091D80A5091D90AAB
:107360006091DA0A7091DB0A8EE493E00E9437475D
:107370004091DC0A5091DD0A6091DE0A7091DF0ACB
:107380008BE493E00E9437474091E00A5091E10A74
:107390006091E20A7091E30A88E493E00E94374723
:1073A000EEE1F2E007C08091C00085FFFCCF31968E
:1073B0009093C60090819923B1F78091C00085FF1A
:1073C000FCCF8AE08093C600FE019491EDE9F2E0E3
:1073D00008C08091C00085FFFCCF9093C600319615
:1073E00094919923B1F7E6E3F3E0949108C080917A
:1073F000C00085FFFCCF9093C600319694919923ED
:10740000B1F78091C00085FFFCCF8AE08093C60071
:10741000FE019491EDE9F2E008C08091C00085FF83
:10742000FCCF9093C600319694919923B1F7409187
:107430009D0850919E0860919F087091A0088DE270
:1074400093E00E9437474091A1085091A2086091B3
:10745000A3087091A4088AE293E00E943747409104
:10746000A5085091A6086091A7087091A80887E226
:1074700093E00E943747EEE1F2E007C08091C00040
:1074800085FFFCCF31969093C60090819923B1F788
:107490008091C00085FFFCCF8AE08093C600FE018A
:1074A0009491EDE9F2E008C08091C00085FFFCCF27
:1074B0009093C600319694919923B1F7E1E1F3E0FE
:1074C000949108C08091C00085FFFCCF9093C600C6
:1074D000319694919923B1F78091C00085FFFCCF3C
:1074E0008AE08093C600FE019491EDE9F2E008C0C5
:1074F0008091C00085FFFCCF9093C6003196949197
:107500009923B1F78091AE059091AF056CE370E0DF
:107510000E94C6EEAB0160E070E088E093E00E945C
:107520004947EEE1F2E007C08091C00085FFFCCF43
:1075300031969093C60090819923B1F78091C00055
:1075400085FFFCCF8AE08093C6008091AE059091C4
:10755000AF056CE370E00E94C6EEAC0160E070E045
:107560008DEF92E00E944947EEE1F2E007C0809182
:10757000C00085FFFCCF31969093C600908199237F
:10758000B1F78091C00085FFFCCF8AE08093C600F0
:10759000FE019491EDE9F2E008C08091C00085FF02
:1075A000FCCF9093C600319694919923B1F7EFEEFA
:1075B000F2E0949108C08091C00085FFFCCF9093C9
:1075C000C600319694919923B1F78091C00085FF50
:1075D000FCCF8AE08093C600FE019491EDE9F2E0D1
:1075E00008C08091C00085FFFCCF9093C600319603
:1075F00094919923B1F74091C4045091C5046091CE
:10760000C6047091C70485EE92E00E9437476091EE
:10761000C8047091C9048091CA049091CB040E945F
:10762000C69AAB01BC0182EE92E00E94374760919E
:10763000CC047091CD048091CE049091CF040E942F
:10764000D29AAB01BC018FED92E00E943747EEE188
:10765000F2E007C08091C00085FFFCCF3196909387
:10766000C60090819923B1F78091C00085FFFCCFBF
:107670008AE08093C600DF91CF9108950F931F9306
:10768000DF93CF93CDB7DEB728970FB6F894DEBF60
:107690000FBECDBF80911A0290911B02A0911C02D7
:1076A000B0911D028D839E83AF83B887FE01319612
:1076B00004E610E0F999FECF12BD01BDF89A80B53D
:1076C00080830F5F1F4F0836110511F03196F2CFFE
:1076D000CE010596BE016F5F7F4F43E050E00E94F0
:1076E0005524009709F098C1ECEAFAE0F999FECF29
:1076F00012BD01BDF89A80B580830F5F1F4F083718
:10770000110511F03196F2CFECE9FAE0F999FECFCC
:1077100012BD01BDF89A80B580830F5F1F4F0838F6
:10772000110511F03196F2CFECEBFAE0F999FECFAA
:1077300012BD01BDF89A80B580830F5F1F4F0839D5
:10774000110511F03196F2CF0E948A6CE0EDFAE05B
:10775000F999FECF12BD01BDF89A80B580830F5F05
:107760001F4F0C39110511F03196F2CFE4EDFAE01C
:10777000F999FECF12BD01BDF89A80B580830F5FE5
:107780001F4F003A110511F03196F2CFECECFAE000
:10779000F999FECF12BD01BDF89A80B580830F5FC5
:1077A0001F4F043A110511F03196F2CFE4EEFAE0E2
:1077B000F999FECF12BD01BDF89A80B580830F5FA5
:1077C0001F4F083A110511F03196F2CFE8E9FAE0BF
:1077D000F999FECF12BD01BDF89A80B580830F5F85
:1077E0001F4F0C3A110511F03196F2CFE8EDFAE097
:1077F000F999FECF12BD01BDF89A80B580830F5F65
:107800001F4F003B110511F03196F2CFECEDFAE07D
:10781000F999FECF12BD01BDF89A80B580830F5F44
:107820001F4F043B110511F03196F2CFE0EEFAE064
:10783000F999FECF12BD01BDF89A80B580830F5F24
:107840001F4F083B110511F03196F2CFEDE9F8E03A
:10785000F999FECF12BD01BDF89A80B580830F5F04
:107860001F4F043C110511F03196F2CFEEEAF5E01E
:10787000F999FECF12BD01BDF89A80B580830F5FE4
:107880001F4F063C110511F03196F2CFEDEDF7E1F7
:10789000F999FECF12BD01BDF89A80B580830F5FC4
:1078A0001F4F083C110511F03196F2CFEFEDF7E1D3
:1078B000F999FECF12BD01BDF89A80B580830F5FA4
:1078C0001F4F0A3C110511F03196F2CFE1EEF7E1BE
:1078D000F999FECF12BD01BDF89A80B580830F5F84
:1078E0001F4F0C3C110511F03196F2CFE3EEF7E19A
:1078F000F999FECF12BD01BDF89A80B580830F5F64
:107900001F4F0E3C110511F03196F2CFE5EEF7E175
:10791000F999FECF12BD01BDF89A80B580830F5F43
:107920001F4F003D110511F03196F2CFE7EEF7E160
:10793000F999FECF12BD01BDF89A80B580830F5F23
:107940001F4F023D110511F03196F2CFE4ECF4E047
:10795000F999FECF12BD01BDF89A80B580830F5F03
:107960001F4F063D110511F03196F2CFE8ECF4E01F
:10797000F999FECF12BD01BDF89A80B580830F5FE3
:107980001F4F0A3D110511F03196F2CFECECF4E0F7
:10799000F999FECF12BD01BDF89A80B580830F5FC3
:1079A0001F4F0E3D110511F03196F2CFEAEEF9E1CD
:1079B000F999FECF12BD01BDF89A80B580830F3DC5
:1079C000110521F031960FED10E0F2CF0E947A9A66
:1079D000EDE9F2E0949108C08091C00085FFFCCFF2
:1079E0009093C600319694919923B1F7E5ECF2E0BB
:1079F000949108C08091C00085FFFCCF9093C60091
:107A0000319694919923B1F78091C00085FFFCCF06
:107A10008AE08093C60001C0D5D881DA28960FB6D7
:107A2000F894DEBF0FBECDBFCF91DF911F910F91B4
:107A300008958130910541F08230910549F0892BFC
:107A400051F41092A605089581E08093A60508954B
:107A500082E08093A6050895CF92DF92EF92FF9285
:107A60000F931F938091A5058823E1F11092A5053E
:107A700085E061E00E94F6E50091AC051091AD054E
:107A80000E9476E36B017C016091A7057091A805C7
:107A90008091A9059091AA0528EE33E040E050E0DE
:107AA0000E94EDEE021B130B0C0D1D1D1093AD0576
:107AB0000093AC058091AB058823A1F0EFE1F2E0E3
:107AC00007C08091C00085FFFCCF31969093C6001F
:107AD00090819923B1F78091C00085FFFCCF8AE0A7
:107AE0008093C6001F910F91FF90EF90DF90CF9091
:107AF0000895CF93DF93EC0181E08093A5050E9468
:107B000084E36093A7057093A8058093A9059093DB
:107B1000AA05BE01882777FD8095982F0E9497EBD4
:107B200020E030E44CE156E40E9403ED18161CF40A
:107B3000C0E1D7E204C0D7FF02C0C0E0D0E085E0DA
:107B400061E00E9443E5BE01882777FD8095982F6C
:107B50000E9497EB20E030E44CE156E40E94FCEAFE
:107B600020E030E040EA53E40E94D5ED0E9464EB4F
:107B70009B01AC0197FF07C050954095309521952A
:107B80003F4F4F4F5F4F86E0B9010E9465E485E0AB
:107B900060E00E94F6E58091AB058823A1F0E2E366
:107BA000F2E007C08091C00085FFFCCF3196909332
:107BB000C60090819923B1F78091C00085FFFCCF6A
:107BC0008AE08093C600DF91CF9108951F93182F0C
:107BD00061E00E9443E5812F61E070E00E9465E46E
:107BE000E1EAF0E0108282E88093A00080E491E076
:107BF0009093A7008093A6008FE391E09093A90053
:107C00008093A80089E18083F894E1EAF0E0808124
:107C1000887F808380E491E09093A5008093A40006
:107C20009093A7008093A6008081816080837894E0
:107C30001F91089586E090E0C9DF85E061E00E9431
:107C4000F6E585E061E00E9443E580E090E4ACE188
:107C5000B6E48093940590939505A0939605B09310
:107C6000970580E090E0A0E0B0E0809398059093C5
:107C70009905A0939A05B0939B0510929C051092CC
:107C80009D0510929E0510929F051092A4051092DA
:107C9000A5051092A6051092A7051092A8051092AE
:107CA000A9051092AA051092AB051092AD0510928D
:107CB000AC0580E090E0A0E8BFE38093F5059093E9
:107CC000F605A093F705B093F8058DEC9CECACE4B9
:107CD000BEE38093F9059093FA05A093FB05B0935A
:107CE000FC0581E080930106B7CE1F920F920FB67C
:107CF0000F920BB60F9211242F933F934F938F93B4
:107D00009F93EF93FF934091C600E0918206F0911C
:107D1000830631969F012F773070319780918406CA
:107D2000909185062817390739F0EE5FF94F4083A7
:107D30003093830620938206FF91EF919F918F915C
:107D40004F913F912F910F900BBE0F900FBE0F9050
:107D50001F9018959A01AB01203081EE380780E022
:107D6000480780E0580749F182E08093C00060E056
:107D700079E08DE390E00E940FEF215030404040C9
:107D80005040CA01B90122E030E040E050E00E94DA
:107D90000FEF3093C5002093C4008091C100806133
:107DA0008093C1008091C10088608093C100809160
:107DB000C10080688093C10008951092C00020E146
:107DC00030E0E7CF209184063091850680918206CD
:107DD000909183068217930719F42FEF3FEF0EC09F
:107DE000F901EE5FF94F80812F5F3F4F2F773070A1
:107DF0003093850620938406282F30E0C90108952A
:107E000080918406909185069093830680938206E4
:107E1000089508952F923F924F925F926F927F92B2
:107E20008F929F92AF92BF92CF92DF92EF92FF928A
:107E30000F931F93DF93CF93CDB7DEB7A0970FB605
:107E4000F894DEBF0FBECDBF1C016A017B01411556
:107E500051056105710541F440E350E060E070E0D8
:107E600020E030E08BD055C0882499245401422E64
:107E700055246624772401E010E00C0F1D1F080D27
:107E8000191DC701B601A30192010E94EDEEF80190
:107E900060830894811C911CA11CB11CC701B60110
:107EA000A30192010E94EDEEC901DA016C017D018E
:107EB000C114D104E104F104F1F681E0E82EF12CC3
:107EC000EC0EFD1EE80CF91C3E010894611C711CAF
:107ED000D501C4010197A109B1096C01C818D908DD
:107EE00015C0F601EE0DFF1D40814A3010F4405DD3
:107EF00001C0495C552747FD5095652F752FC1017D
:107F000020E030E03BD00894E108F1086E147F04D3
:107F100041F7A0960FB6F894DEBF0FBECDBFCF914C
:107F2000DF911F910F91FF90EF90DF90CF90BF9066
:107F3000AF909F908F907F906F905F904F903F9009
:107F40002F9008952115310539F48091C00085FFE7
:107F5000FCCF4093C60008955DCFEF92FF920F9340
:107F60001F939A01E62EFF2400E010E0B801A7015C
:107F7000E9DF1F910F91FF90EF900895EF92FF922C
:107F80000F931F93CF93DF93EC017A018B0121159F
:107F9000310539F48091C00085FFFCCFE092C60026
:107FA00019C02A303105A9F477FF0FC04DE250E027
:107FB00060E070E020E030E0E1DF10950095F094A3
:107FC000E094E11CF11C011D111DCE01B801A701B7
:107FD0002AE020DFDF91CF911F910F91FF90EF906A
:107FE0000895EF92FF920F931F937B019A01002750
:107FF000F7FC0095102FB801A701C0DF1F910F916A
:10800000FF90EF9008950F931F938C014DE050E087
:1080100060E070E020E030E0B1DFC8014AE050E00D
:1080200060E070E020E030E0A9DF1F910F9108953B
:10803000CF92DF92EF92FF920F931F938C019A01E0
:108040006B01EE24FF24B701A6017CDFC801DBDF52
:108050001F910F91FF90EF90DF90CF9008959F9226
:10806000AF92BF92CF92DF92EF92FF920F931F9346
:10807000CF93DF93EC017A018B01922ECB01BA01F1
:1080800020E030E040E050E00E94F5EA882364F40C
:10809000CE014DE250E060E070E020E030E06EDFC5
:1080A00017FB109517F9109520E030E040E05FE3F2
:1080B000AA240BC0CA01B90120E030E040E251E43B
:1080C0000E94FCEA9B01AC01A394A91498F3C80197
:1080D000B7010E941CEA7B018C010E9469EB5B01E5
:1080E0006C010E9495EB9B01AC01C801B7010E9495
:1080F0001BEA7B018C01CE01B601A5012AE030E02C
:1081000021DF992099F1EEE3F2E007C08091C000F1
:1081100085FFFCCF31969093C60090819923B1F7EB
:1081200025C0C801B70120E030E040E251E40E94E0
:10813000D5ED7B018C010E9464EB5B016C01CC24CA
:10814000B7FCC094DC2CCE01B601A5012AE030E0DA
:1081500015DFC601B5010E9497EB9B01AC01C80178
:10816000B7010E941BEA7B018C019A949920C9F601
:10817000DF91CF911F910F91FF90EF90DF90CF9003
:10818000BF90AF909F9008956ACF0895EF92FF92AD
:108190000F931F93CF93DF93EC01E090A004F09036
:1081A000A1040091A2041091A304688179818A81BD
:1081B0009B81A80197010E9403ED181624F4E88220
:1081C000F9820A831B83E090A404F090A504009137
:1081D000A6041091A7046C817D818E819F81A801E6
:1081E00097010E9403ED181624F4EC82FD820E83A1
:1081F0001F83E090A804F090A9040091AA041091B4
:10820000AB04688579858A859B85A80197010E94C2
:1082100003ED181624F4E886F9860A871B87DF9198
:10822000CF911F910F91FF90EF9008958091C0081A
:1082300008950F931F93CF93DF938130910549F4F5
:108240006F5F7F4F09F046C087E896E00E940333D6
:1082500041C0892B09F03EC06F5F7F4FD9F58AE698
:1082600095E0909352088093510880915808882394
:1082700021F085E598E00E941883CDE0D8E00AE679
:1082800015E005C06F9786E0C73DD80751F0198308
:1082900008838F818823B1F3CE0104960E9418834E
:1082A000F1CF8AE695E0998388838F81882321F036
:1082B000CE0104960E9418838AE695E09093B70653
:1082C0008093B6068091BD06882321F08AEB96E064
:1082D0000E941883DF91CF911F910F91089580E044
:1082E00090E06FEF7FEFA5CF81E090E06FEF7FEF41
:1082F000A0CF0E949D9A8091AB058823A1F0E0E475
:10830000F2E007C08091C00085FFFCCF31969093CA
:10831000C60090819923B1F78091C00085FFFCCF02
:108320008AE08093C60098DB8091C008882309F01A
:108330003AC081E08093C0088091CB089091CC082E
:10834000A091CD08B091CE088093CF089093D0082B
:10835000A093D108B093D208E7EEF4E0949108C05E
:108360008091C00085FFFCCF9093C6003196949118
:108370009923B1F7E8EFF4E0949108C08091C00030
:1083800085FFFCCF9093C600319694919923B1F765
:108390008091C00085FFFCCF8AE08093C6008EEEFE
:1083A00094E00C9437D7089589E260E00E9443E599
:1083B000A09A0895F8940E949D9A5F9A8A9A8FB71E
:1083C000F894909108019160909308018FBF129AE0
:1083D00031DC8CE060E00E9443E5E7EEF4E094914C
:1083E00008C08091C00085FFFCCF9093C6003196F5
:1083F00094919923B1F7E7E7F5E0949108C0809153
:10840000C00085FFFCCF9093C600319694919923CC
:10841000B1F78091C00085FFFCCF8AE08093C60051
:108420008EE695E00E9446D7FFCF0E9476E36093E8
:10843000D3087093D4088093D5089093D608E09120
:108440000009F0910109EE5FF64F80818823A9F4BD
:10845000E6E9F5E0949108C08091C00085FFFCCF6B
:108460009093C600319694919923B1F78091C00002
:1084700085FFFCCF8AE08093C60008950E9476E3D2
:108480002091C6083091C7084091C8085091C9088A
:10849000621B730B840B950B645C794080409040A9
:1084A00008F448C00E9476E36093C6087093C7083A
:1084B0008093C8089093C9084F9B08C07A9B06C058
:1084C0008091060180FF02C002990AC00E9476E3F3
:1084D0006093C2087093C3088093C4089093C50842
:1084E0000E9476E32091C2083091C3084091C408ED
:1084F0005091C508621B730B840B950B60567A4E26
:108500008040904028F4211531054105510549F47A
:108510008AE060E00E94F6E58AE060E070E00C949A
:1085200065E48AE06FEF0E94F6E58AE06FEF70E0A5
:108530000C9465E40895EF92FF920F931F930E94AD
:1085400076E3E090D708F090D8080091D908109110
:10855000DA082091D3083091D4084091D508509181
:10856000D608621B730B840B950BE616F7060807FB
:10857000190730F4E114F1040105110509F01ADFBF
:108580008091DB089091DC08A091DD08B091DE08B5
:108590000097A105B10509F447C00E9476E3209138
:1085A000D3083091D4084091D5085091D608621B69
:1085B000730B840B950B2091DB083091DC08409104
:1085C000DD085091DE08261737074807590760F580
:1085D0009091191580911A15981731F55F9A8A9A1A
:1085E0008FB7F894909108019160909308018FBF24
:1085F0001092990810929A08129A8091AC05909165
:10860000AD0580569A4E78F08091AE059091AF05F9
:1086100001969093AF058093AE051092AD05109230
:10862000AC050E949B3306DB909901C0C3DE26DFB8
:108630000E94F76E1F910F91FF90EF9008956F9237
:108640007F928F929F92AF92BF92CF92DF92EF92E2
:10865000FF920F931F93F82E6091DF087091E0084E
:108660008091E1089091E2082091E3083091E408BC
:108670004091E5085091E6080E9410ED3B014C0145
:1086800000D000D00DB71EB70F5F1F4F60919C0444
:1086900070919D04882777FD8095982F0E9497EB15
:1086A0002091AE043091AF044091B0045091B104D8
:1086B0000E94D5ED20E030E040E752E40E94FCEA61
:1086C00020E030E048EC52E40E94FCEA5B016C01DF
:1086D000F8016082718282829382F4828091B5086F
:1086E000858389E898E06BEE78E04FED58E020E074
:1086F00001E032E0E32E0E94E8678091EB08909160
:10870000EC08A091ED08B091EE0880938908909351
:108710008A08A0938B08B0938C088091EF08909101
:10872000F008A091F108B091F20880938D08909321
:108730008E08A0938F08B09390088091F3089091D1
:10874000F408A091F508B091F608809391089093F1
:108750009208A0939308B09394088091F7089091A1
:10876000F808A091F908B091FA08809395089093C1
:108770009608A0939708B09398088DB79EB7069671
:108780000FB6F8949EBF0FBE8DBF0E9476E3609334
:10879000D3087093D4088093D5089093D6081F917E
:1087A0000F91FF90EF90DF90CF90BF90AF909F9090
:1087B0008F907F906F900895AF92BF92CF92DF928B
:1087C000EF92FF920F931F93E090A004F090A1040A
:1087D0000091A2041091A3046091EB087091EC0841
:1087E0008091ED089091EE08A80197010E9403ED99
:1087F000181644F4E092EB08F092EC080093ED08B0
:108800001093EE08E090A404F090A5040091A60453
:108810001091A7046091EF087091F0088091F10821
:108820009091F208A80197010E9403ED181644F4F4
:10883000E092EF08F092F0080093F1081093F2082C
:10884000E090A804F090A9040091AA041091AB0450
:108850006091F3087091F4088091F5089091F60802
:10886000A80197010E9403ED181644F4E092F30862
:10887000F092F4080093F5081093F6080E9476E34E
:108880006093D3087093D4088093D5089093D6084A
:10889000A0909508B0909608C0909708D09098083E
:1088A000E090F708F090F8080091F9081091FA08A4
:1088B000C601B501A80197010E94F5EA882389F154
:1088C0006091890870918A0880918B0890918C083A
:1088D0002091EB083091EC084091ED085091EE08A2
:1088E0000E94F5EA8823A1F460918D0870918E08AA
:1088F00080918F08909190082091EF083091F008B6
:108900004091F1085091F2080E94F5EA882349F05D
:1089100081E08093A4058CE090E090939305809390
:108920009205C601B501A80197010E94F5EA8823C6
:1089300041F480919205909193050C9711F4109257
:10894000A4056091890870918A0880918B089091A4
:108950008C082091EB083091EC084091ED08509183
:10896000EE080E94F5EA882309F07CC060918D082A
:1089700070918E0880918F08909190082091EF0857
:108980003091F0084091F1085091F2080E94F5EA08
:10899000882309F067C06091AE047091AF048091A4
:1089A000B0049091B10420E030E040E752E40E942E
:1089B000FCEA7B018C018BEE98E06FEE78E043EFF0
:1089C00058E027EF38E0E5EBCE2EE8E0DE2E0E94FF
:1089D0001C728091EB089091EC08A091ED08B09189
:1089E000EE088093890890938A08A0938B08B0932F
:1089F0008C088091EF089091F008A091F108B09157
:108A0000F20880938D0890938E08A0938F08B093FE
:108A100090088091F3089091F408A091F508B09126
:108A2000F6088093910890939208A0939308B093CE
:108A300094088091F7089091F808A091F908B091F6
:108A4000FA088093950890939608A0939708B0939E
:108A500098081F910F91FF90EF90DF90CF90BF90FB
:108A6000AF90089560919C0470919D04882777FDD4
:108A70008095982F0E9497EB2091AE043091AF041F
:108A80004091B0045091B1040E94D5ED20E030E057
:108A900040E752E40E94FCEA20E030E048EC52E477
:108AA00086CF86E896E0ACD9E9E9F5E0949108C074
:108AB0008091C00085FFFCCF9093C60031969491C1
:108AC0009923B1F74091CB085091CC086091CD0823
:108AD0007091CE084F5F5F4F6F4F7F4F86E896E0F3
:108AE0002AE030E04BDA8091C00085FFFCCF8AE0BD
:108AF0008093C6009ACCFC01949108C08091C0007C
:108B000085FFFCCF9093C600319694919923B1F7DD
:108B100086E896E02AE030E031CA2F923F924F92E9
:108B20005F926F927F928F929F92AF92BF92CF92FD
:108B3000DF92EF92FF920F931F93DF93CF9300D0BA
:108B400000D0CDB7DEB79C018330910508F055C148
:108B5000FC01E757F84FD490FC01E756F74F81E04E
:108B600080833901660C771C660C771C93012757AC
:108B7000374F3A83298380E090E0A0E0B0E0F9012C
:108B800080839183A283B38389E898E06DE878E0DD
:108B900041E958E025E938E00E94D26CF301E3583E
:108BA000F84FE590F590059114916D2D772767FDAD
:108BB0007095882777FD8095982F0E9497EB1B0171
:108BC0002C0193012551374F3E832D83C801B701F6
:108BD00020E030E040EC5FE30E94D5EDA20191017E
:108BE0000E94D5EDAD81BE816D937D938D939C9355
:108BF0001397F301E457FB4FFC83EB836081718192
:108C0000828193816093AE047093AF048093B0042B
:108C10009093B10420E030E040E752E40E94FCEA87
:108C20007B018C018BEE98E06FEE78E043EF58E02B
:108C300027EF38E0A5EBCA2EA8E0DA2E0E941C72BE
:108C40000E94DE9080E090E0A0E0B0E0E981FA814F
:108C500080839183A283B38389E898E06DE878E00C
:108C600041E958E025E938E00E94D26CF301E05573
:108C7000F84F85909590A590B490C501B401905897
:108C8000A20191010E94D5EDAD81BE816D937D93CE
:108C90008D939C9313976091AE047091AF04809173
:108CA000B0049091B10420E030E040E752E40E942B
:108CB000FCEA7B018C018BEE98E06FEE78E043EFED
:108CC00058E027EF38E00E941C720E94DE90C50138
:108CD000B401A50194010E941CEAA20191010E9425
:108CE000D5EDED81FE816083718382839383AB81B7
:108CF000BC816D917D918D919C9120E030E040E0B0
:108D00005FE30E94D5ED6093AE047093AF0480934F
:108D1000B0049093B10420E030E040E752E40E94B8
:108D2000FCEA7B018C018BEE98E06FEE78E043EF7C
:108D300058E027EF38E00E941C720E94DE90F30199
:108D4000E457F84F6591759185919491F301E3563D
:108D5000F74FA080B180C280D380A60195010E9408
:108D60001CEA7B018C01CB01D801E981FA81808367
:108D70009183A283B383F301E856F84F659175910F
:108D800085919491F9EA8F2EF8E09F2E860C971C1E
:108D9000A60195010E941CEAD4016D937D938D93E9
:108DA0009C931397F301EC55F84F6591759185915C
:108DB0009491E0EAF4E06E0E7F1EA60195010E94F8
:108DC0001CEAD3016D937D938D939C931397C701F8
:108DD000D801ED81FE8180839183A283B38380E0FB
:108DE00090E0A0E0B0E08093AE049093AF04A09335
:108DF000B004B093B1040E94C08F26960FB6F894C9
:108E0000DEBF0FBECDBFCF91DF911F910F91FF90BD
:108E1000EF90DF90CF90BF90AF909F908F907F901A
:108E20006F905F904F903F902F9008954091000970
:108E30005091010920E630E0B901469F9001479F1B
:108E4000300D569F300D1124682F772767FD7095E0
:108E5000C901885F964F0E9443249C0190930709A3
:108E60008093060980E0232B09F081E00895FC013E
:108E7000949108C08091C00085FFFCCF9093C600FC
:108E8000319694919923B1F786E896E022E030E09C
:108E90007BC9FC01949108C08091C00085FFFCCF84
:108EA0009093C600319694919923B1F786E896E0A5
:108EB0002AE030E047C880910609909107090196A1
:108EC00060E070E04AE050E00C94AB22809106092B
:108ED00090910709019660E070E00C944E21CF93C9
:108EE000DF93EC018091B5088093CA0884E59EDF8A
:108EF000882309F46EC0EADF0E9469EB262F609395
:108F0000CA08662309F465C0E1EEF4E0949108C054
:108F10008091C00085FFFCCF9093C600319694915C
:108F20009923B1F7C936D10599F0CA36D10524F491
:108F3000C836D105F1F50FC0CD36D10531F0CA3DA7
:108F4000D105B9F5E0E6F2E031C0E7E7F2E023C091
:108F5000EEE8F2E015C0E5EAF2E007C08091C0005B
:108F600085FFFCCF31969093C60090819923B1F78D
:108F700020C08091C00085FFFCCF31969093C60041
:108F800090819923B1F715C08091C00085FFFCCF77
:108F900031969093C60090819923B1F70AC08091D1
:108FA000C00085FFFCCF31969093C6009081992335
:108FB000B1F786E896E0622F40E050E00E94AD3FB6
:108FC0008091C00085FFFCCF8AE08093C60081E0DD
:108FD00001C080E0DF91CF910895AF92BF92CF9210
:108FE000DF92EF92FF920F931F93CF93DF9319E8D5
:108FF000E12E18E0F12ECBEED8E000E010E0F80111
:10900000E65DFA4F808112DF882331F15FDF5B017B
:109010006C01F801ED57F74F8081882311F061E072
:1090200002C06091FB0870E0882777FD8095982F3B
:109030000E9497EBF70120813181428153810E9488
:10904000D5ED9B01AC01C601B5010E941CEA688305
:1090500079838A839B8309C0F70180819181A281F2
:10906000B38188839983AA83BB830F5F1F4F84E0FA
:1090700090E0E80EF91E24960430110509F0BFCFE8
:1090800086E4D4DE8823D9F021DF7B018C01609354
:10909000FC087093FD088093FE089093FF0820E081
:1090A00030E040E050E00E9403ED181644F4E092F6
:1090B000AE04F092AF040093B0041093B104DF91BA
:1090C000CF911F910F91FF90EF90DF90CF90BF90C5
:1090D000AF90089582DF89E4A9DE882351F0F6DE9F
:1090E0006093DF087093E0088093E1089093E208B2
:1090F0000CC080E090E0A0E0B0E08093DF089093A7
:10910000E008A093E108B093E2088AE48FDE8823A8
:1091100051F0DCDE6093E3087093E4088093E50887
:109120009093E608089580E090E0A0E0B0E080939E
:10913000E3089093E408A093E508B093E608089547
:109140002F923F924F925F926F927F928F929F9257
:10915000AF92BF92CF92DF92EF92FF920F931F9345
:10916000DF93CF93CDB7DEB76E970FB6F894DEBF1F
:109170000FBECDBF87E45ADE882309F4ABC6A6DE56
:109180000E9464EB6430710509F4B8C16530710563
:10919000A4F461307105A1F16230710524F4672BEC
:1091A00039F10C943F606230710509F4A7C0633057
:1091B000710511F00C943F601FC16A35710509F407
:1091C00036C66B35710554F46730710509F4DAC1A0
:1091D0006C31710511F00C943F6019C36B3571054A
:1091E00009F429C66C35710511F00C943F6028C64E
:1091F0008091C008882321F4F0DEDEDA0C946460EC
:109200008091C008882309F079C0E7DE83E50EDE8F
:10921000882369F08091C008882349F457DE609361
:1092200094057093950580939605909397058CE42B
:10923000FDDD882311F18091C0088823F1F446DE1A
:109240000E9464EB9B01AC0160939C0570939D05AB
:1092500080939E0590939F0597FF0FC088279927BD
:10926000DC01821B930BA40BB50B80939C059093A0
:109270009D05A0939E05B0939F0580E5D7DD8823CB
:1092800069F08091C008882349F420DE6093980536
:109290007093990580939A0590939B0584E4C6DDAD
:1092A000882391F08091C008882371F40FDE10921A
:1092B000AB0520E030E040E050E00E94F5EA882372
:1092C00019F081E08093AB0582E4B0DD882359F08A
:1092D0008091C008882339F4F9DD0E9464EBDC0139
:1092E000CB010E94193D81E08093A4058AE090E0C3
:1092F00090939305809392055FDAFCC08091C0083B
:10930000882309F079C0E6DE83E590DD882369F0E3
:109310008091C008882349F4D9DD60939405709347
:10932000950580939605909397058CE47FDD8823BF
:1093300011F18091C0088823F1F4C8DD0E9464EB2C
:109340009B01AC0160939C0570939D0580939E05E5
:1093500090939F0597FF0FC088279927DC01821BF8
:10936000930BA40BB50B80939C0590939D05A09344
:109370009E05B0939F0580E559DD882369F08091B3
:10938000C008882349F4A2DD60939805709399057D
:1093900080939A0590939B0584E448DD882391F09F
:1093A0008091C008882371F491DD1092AB0520E014
:1093B00030E040E050E00E94F5EA882319F081E0B7
:1093C0008093AB0582E432DD882359F08091C00898
:1093D000882339F47BDD0E9464EBDC01CB010E9421
:1093E000193D81E08093A4058AE090E09093930575
:1093F0008093920581E07DC08091C008882309F0A8
:109400007DC068DE83E512DD882369F08091C008A5
:10941000882349F45BDD60939405709395058093F0
:109420009605909397058CE401DD882311F18091D6
:10943000C0088823F1F44ADD0E9464EB9B01AC0173
:1094400060939C0570939D0580939E0590939F0566
:1094500097FF0FC088279927DC01821B930BA40B71
:10946000B50B80939C0590939D05A0939E05B093AA
:109470009F0580E5DBDC882369F08091C0088823A4
:1094800049F424DD609398057093990580939A05BB
:1094900090939B0584E4CADC882391F08091C008F6
:1094A000882371F413DD1092AB0520E030E040E03A
:1094B00050E00E94F5EA882319F081E08093AB0523
:1094C00082E4B4DC882359F08091C008882339F401
:1094D000FDDC0E9464EBDC01CB010E94193D81E0C0
:1094E0008093A4058AE090E0909393058093920581
:1094F00080E0A5D81092A4050C94646084E797E0FE
:109500000E9437D780E592DC882321F4EE24FF24E3
:10951000870105C0DBDC0E9469EB7B018C0183E5E0
:1095200085DC882359F0D2DC20E030E04AE754E4BF
:109530000E94D5ED0E9469EB7B018C010E94DE90B8
:109540000E9476E35B016C01AE0CBF1CC01ED11EF5
:109550000E9476E36093D3087093D4088093D50873
:109560009093D60806C00E94129E0E949B420E94C1
:1095700017D80E9476E36A157B058C059D0598F344
:109580000C943F608CE452DC882339F09FDC0E940D
:1095900064EB7093FE056093FD0584E247DC88234D
:1095A000A1F194DC1092010620E030E040E050E0B0
:1095B0000E94F5EA882319F081E08093010660910A
:1095C000F9057091FA058091FB059091FC052091B9
:1095D000F5053091F6054091F7055091F8050E9488
:1095E000D5ED9B01AC0160918D0870918E08809142
:1095F0008F08909190080E941CEA6093EF08709386
:10960000F0088093F1089093F20884E40FDC88233B
:1096100091F060910609709107096F5F7F4F40914B
:10962000FD055091FE0580EB95E00E940527909383
:1096300000068093FF0580910106882309F04DC044
:109640006091FF0570910006882777FD8095982F1F
:109650000E9497EB2091F9053091FA054091FB05A6
:109660005091FC050E94D5ED9B01AC0160918908E9
:1096700070918A0880918B0890918C080E941BEA57
:109680006093EB087093EC088093ED089093EE08DC
:109690008091AB05882309F46EC0E1EEF4E094916B
:1096A00008C08091C00085FFFCCF9093C600319622
:1096B00094919923B1F7ECEBF2E007C08091C000E0
:1096C00085FFFCCF31969093C60090819923B1F726
:1096D0008091C00085FFFCCF4BC06091FF05709169
:1096E0000006882777FD8095982F0E9497EB2091A0
:1096F000F9053091FA054091FB055091FC050E9457
:10970000D5ED9B01AC016091890870918A08809128
:109710008B0890918C080E941CEA6093EB08709370
:10972000EC088093ED089093EE088091AB058823B8
:1097300011F1E1EEF4E0949108C08091C00085FF42
:10974000FCCF9093C600319694919923B1F7E1ED47
:10975000F2E007C08091C00085FFFCCF3196909366
:10976000C60090819923B1F78091C00085FFFCCF9E
:109770008AE08093C60060E070E080E89FE320917B
:10978000F9053091FA054091FB055091FC050E94C6
:10979000FCEA7B018C016093980570939905809396
:1097A0009A0590939B056091AE047091AF048091EF
:1097B000B0049091B10420E030E040E752E40E9410
:1097C000FCEA9B01AC0160E074E284E799E40E944A
:1097D000FCEAA80197010E94FCEA0E9469EB6093F1
:1097E0009C0570939D0580939E0590939F0582E054
:1097F0008093A60581E08093A40582E090E0909399
:109800009305809392050E94DC430C943F60809105
:10981000AE049091AF04A091B004B091B1048093D4
:10982000880A9093890AA0938A0AB0938B0A809140
:109830009C0490919D04909388088093870884E607
:1098400090E090939D0480939C040E9476E3609343
:10985000D3087093D4088093D5089093D60881E0FC
:109860000E94C78F8091890890918A08A0918B08E7
:10987000B0918C088093EB089093EC08A093ED08CE
:10988000B093EE0880918D0890918E08A0918F087A
:10989000B09190088093EF089093F008A093F1089E
:1098A000B093F2088091910890919208A09193084A
:1098B000B09194088093F3089093F408A093F5086E
:1098C000B093F6088091950890919608A09197081A
:1098D000B09198088093F7089093F808A093F9083E
:1098E000B093FA0880E090E0A0E0B0E08093AE048E
:1098F0009093AF04A093B004B093B10488E596DAD6
:10990000882351F489E592DA882331F48AE58EDAE6
:10991000882311F481E001C080E08093B2048823A1
:1099200051F488E583DA882309F4D3C189E57EDA26
:10993000882309F4CEC180E090E0A0E0B0E08093FD
:10994000890890938A08A0938B08B0938C08809321
:109950008D0890938E08A0938F08B0939008F9E833
:109960008F2EF7E09F2EF401E49089E898E06DE8EF
:1099700078E041E958E025E938E00E94D26CEDE753
:10998000F7E0659175918591949120E030E040EC8D
:109990005FE30E94D5ED5B016C01FF24E7FCF094CE
:1099A0000027F7FC0095102FC801B7010E9497EB24
:1099B0009B01AC01C601B5010E94D5ED6093EB0897
:1099C0007093EC088093ED089093EE08E1E8F7E0DF
:1099D00065917591859194910894811C911CF40175
:1099E000D49020E030E040EC5FE30E94D5ED7B01B5
:1099F0008C016D2D772767FD7095872F972F0E941B
:109A000097EB9B01AC01C801B7010E94D5ED6093B3
:109A1000EF087093F0088093F1089093F20820917A
:109A20008C0430918D0440918E0450918F042093CA
:109A3000AE043093AF044093B0045093B104E0906F
:109A40009004F09091040091920410919304C80145
:109A5000B7010E94F5EA882344F4E092AE04F09244
:109A6000AF040093B0041093B1046091AE04709100
:109A7000AF048091B0049091B10420E030E040E761
:109A800052E40E94FCEA7B018C018BEE98E06FEEC1
:109A900078E043EF58E027EF38E0E5EBCE2EE8E042
:109AA000DE2E0E941C720E94DE90ECE8F7E06591C9
:109AB00075918591949120919D0830919E084091D7
:109AC0009F085091A0080E941CEA60938908709337
:109AD0008A0880938B0890938C08E8E9F7E06591F9
:109AE00075918591949120919D0830919E084091A7
:109AF0009F085091A0080E941CEA6093A9087093E7
:109B0000AA088093AB089093AC08E4EAF7E065916B
:109B100075918591949120919D0830919E08409176
:109B20009F085091A0080E941CEA6093A0047093C3
:109B3000A1048093A2049093A304E0E9F7E0659167
:109B40007591859194912091A1083091A20840913E
:109B5000A3085091A4080E941CEA60938D0870939A
:109B60008E0880938F0890939008ECE9F7E0659158
:109B70007591859194912091A1083091A20840910E
:109B8000A3085091A4080E941CEA6093AD0870934A
:109B9000AE088093AF089093B008E8EAF7E06591CB
:109BA0007591859194912091A1083091A2084091DE
:109BB000A3085091A4080E941CEA6093A404709327
:109BC000A5048093A6049093A70489E898E06DE823
:109BD00078E041E958E025E938E00E94D26C8091B4
:109BE000890890918A08A0918B08B0918C08809385
:109BF000EB089093EC08A093ED08B093EE088091E9
:109C00008D0890918E08A0918F08B0919008809354
:109C1000EF089093F008A093F108B093F2086091D8
:109C2000AE047091AF048091B0049091B10420E033
:109C300030E040E752E40E94FCEA7B018C018BEEAD
:109C400098E06FEE78E043EF58E027EF38E00E94AD
:109C50001C7280E090E0A0E0B0E08093AE049093AE
:109C6000AF04A093B004B093B1040E94DE900E94B0
:109C7000C08F8091EB089091EC08A091ED08B09115
:109C8000EE088093890890938A08A0938B08B0937C
:109C90008C088091EF089091F008A091F108B091A4
:109CA000F20880938D0890938E08A0938F08B0934C
:109CB00090088091F3089091F408A091F508B09174
:109CC000F6088093910890939208A0939308B0931C
:109CD00094088091B204882321F488E5A7D88823CA
:109CE00021F080E090E00E948D458091B2048823AD
:109CF00021F489E59BD8882321F081E090E00E943F
:109D00008D458091B204882321F48AE58FD8882379
:109D100021F082E090E00E948D4588E587D8882375
:109D2000C9F0C9D8611571058105910599F0CED8A2
:109D300020919D0830919E0840919F085091A00865
:109D40000E941CEA6093890870938A0880938B08AC
:109D500090938C0889E56AD88823C9F0ACD861153E
:109D600071058105910599F0B1D82091A108309134
:109D7000A2084091A3085091A4080E941CEA609395
:109D80008D0870938E0880938F08909390088AE5D1
:109D90004DD88823C9F08FD86115710581059105CB
:109DA00099F094D82091A5083091A6084091A70871
:109DB0005091A8080E941CEA609391087093920841
:109DC000809393089093940889E898E06DE878E090
:109DD00041E958E025E938E00E94D26C80E00E9419
:109DE000C78F8091880A9091890AA0918A0AB091C0
:109DF0008B0A8093AE049093AF04A093B004B09309
:109E0000B104809187089091880890939D04809375
:109E10009C040E9476E36093D3087093D4088093E7
:109E2000D5089093D6080E94C08F0C943F60109282
:109E3000FB080C943F6081E08093FB080C943F602A
:109E400085E40E941647882311F40E94DE9059E8A9
:109E5000E52E58E0F52E4DE9C42E48E0D42E00E062
:109E600010E0F801E65DFA4F80810E9416478823D2
:109E700021F1033059F42AD8F7016083718382837A
:109E8000938385E998E00E94B56C17C01FD8F6014E
:109E900020813181428153810E941CEAF701608355
:109EA00071838283938389E898E06DE878E041E9E3
:109EB00058E025E938E00E94D26C0F5F1F4F24E084
:109EC00030E0E20EF31EC20ED31E0430110549F637
:109ED0000C943F608DE40E941647882311F40C9483
:109EE000615F0E9466470E9464EB6A36710511F457
:109EF0000C9490586B3671050CF08FC06B31710566
:109F000009F4D5C26C317105ECF56431710509F4C1
:109F100042C265317105E4F46330710509F49CC1F6
:109F20006430710534F46230710510F00C943F60B8
:109F300034C16131710509F41DC26231710511F43A
:109F40000C94F3586530710511F00C943F600AC20F
:109F50006731710509F45BC26831710554F46531EC
:109F6000710509F448C26631710511F00C943F6027
:109F700048C26931710509F475C26A3171050CF086
:109F800077C260C26135710511F40C94D058623506
:109F9000710504F56F31710509F480C360327105F4
:109FA00054F46C31710509F488C26E31710511F0F9
:109FB0000C943F60BEC26A32710509F41EC460355C
:109FC000710511F40C94C4586032710511F00C94B1
:109FD0003F60F4C26535710511F40C94495966353A
:109FE000710564F46335710511F40C94EF58643510
:109FF000710514F00C94F3580C94EC586836710504
:10A0000009F445C4693671050CF072C46C357105EC
:10A0100011F00C943F600C945F596E3C710511F483
:10A020000C94C35C6F3C71050CF053C0683771052C
:10A0300011F40C94FD5A693771051CF562377105EE
:10A0400011F40C94095A633771055CF46B36710591
:10A0500011F40C94BF586D36710511F00C943F60EB
:10A060006BC56537710511F40C94F35967377105A9
:10A0700009F48FC06337710511F00C943F600C94A4
:10A08000E459693C710511F40C94055C6A3C710556
:10A090007CF46C38710509F41AC46E3B710509F43F
:10A0A0002DC76937710511F00C943F600C94015B6A
:10A0B0006C3C710511F40C94455C6D3C710514F019
:10A0C0000C94655C6B3C710511F00C943F600C9432
:10A0D000275C31E06039730711F40C94895E41E02C
:10A0E000613974073CF56A3F710511F40C940E5EFA
:10A0F0006B3F710564F46C3D710511F40C94E15CE7
:10A100006D3D710511F00C943F600C94F05C51E0D2
:10A110006D32750711F40C94365D81E06F3278076B
:10A1200011F40C94495E6C52714011F00C943F6034
:10A130000C94FF5CE1E0673F7E0711F40C94955EA0
:10A14000F1E0683F7F079CF421E0653F720711F45E
:10A150000C948F5E31E0663F730714F00C94925EAE
:10A16000645F714011F00C943F600C948C5E53E07E
:10A17000603A750709F457C283E0673E780711F427
:10A180000C944A5F6958724011F00C943F600C9433
:10A19000985EE6EEF2E00C940C5B83E697E00E949A
:10A1A00037D780E50E941647882321F4EE24FF2448
:10A1B000870106C00E9466470E9469EB7B018C0103
:10A1C00083E50E941647882361F00E94664720E0DD
:10A1D00030E04AE754E40E94D5ED0E9469EB7B0130
:10A1E0008C010E94DE900E9476E36093D308709306
:10A1F000D4088093D5089093D608E114F1040105A2
:10A20000110501F10E9476E35B016C01AE0CBF1CED
:10A21000C01ED11E0E9476E36A157B058C059D0544
:10A22000A8F40E946BA4882389F40E94129E0E94C5
:10A230009B420E9417D8EECF0E94129E0E949B4222
:10A240000E9417D80E946BA48823B1F384E597E09D
:10A250000E9437D70C943F6083E50E9416478823FD
:10A2600071F08091C008882351F40E946647609382
:10A2700094057093950580939605909397058CE4CB
:10A280000E941647882319F18091C0088823F9F4A9
:10A290000E9466470E9464EB9B01AC0160939C05A1
:10A2A00070939D0580939E0590939F0597FF0FC027
:10A2B00088279927DC01821B930BA40BB50B809395
:10A2C0009C0590939D05A0939E05B0939F0580E506
:10A2D0000E941647882371F08091C008882351F4AA
:10A2E0000E946647609398057093990580939A053C
:10A2F00090939B0584E40E941647882399F08091EF
:10A30000C008882379F40E9466471092AB0520E0CC
:10A3100030E040E050E00E94F5EA882319F081E047
:10A320008093AB0582E40E941647882361F08091F8
:10A33000C008882341F40E9466470E9464EBDC0158
:10A34000CB010E94193D81E08093A4058BE090E051
:10A3500090939305809392050E9417D80E94DC4346
:10A360000C943F601092A4050E9417D80E94DC4311
:10A370000C943F608BE497E00E9437D75F988A98EF
:10A380009FB7F894809108018E7F809308019FBF4A
:10A3900012980C943F60EBE3F7E0949108C0809131
:10A3A000C00085FFFCCF9093C6003196949199230D
:10A3B000B1F78091C00085FFFCCF8AE08093C60092
:10A3C00087E896E00E94B632EDE2F7E0949108C08B
:10A3D0008091C00085FFFCCF9093C6003196949188
:10A3E0009923B1F78091C00085FFFCCF8AE080936C
:10A3F000C6000C943F6087E896E00E940D2E0C94F6
:10A400003F6087E896E00E941D280C943F60809191
:10A4100006099091070904966AE270E00E944324BD
:10A42000FC01009711F0319710826091060970913C
:10A4300007096C5F7F4F87E896E041E00E94E72BB9
:10A440000C943F6087E896E00E9421280E9476E302
:10A450006093B8087093B9088093BA089093BB08CA
:10A460000C943F6087E896E00E9428280C943F6097
:10A4700080918A06882311F40C943F6083E50E9442
:10A480001647882311F40C943F600E945B47AB0190
:10A49000BC01409378085093790880937A087093B0
:10A4A0007B0885E598E00E94FF810C943F6087E877
:10A4B00096E00E941F2A0C943F60809106099091BB
:10A4C000070904966AE270E00E9443248C01009719
:10A4D00019F1209100093091010980E690E0FC011A
:10A4E0002E9FC0012F9F900D3E9F900D1124885FDD
:10A4F000964F6EE470E00E94432460E270E00E9498
:10A5000043249C012F5F3F4F309307092093060996
:10A5100001501040F80110826091060970910709FE
:10A520006C5F7F4F87E896E040E00E94E72B0C9439
:10A530003F6080918A06882311F40C943F6087E87D
:10A5400096E00E949129809106099091070904964E
:10A550006AE270E00E9443248C01009719F1209177
:10A5600000093091010980E690E0AC01249FC00110
:10A57000259F900D349F900D1124885F964F6EE4B7
:10A5800070E00E94432460E270E00E9443249C013A
:10A590002F5F3F4F30930709209306090150104069
:10A5A000F801108260910609709107096C5F7F4F76
:10A5B00087E896E00E94792A0C943F608091890692
:10A5C000882341F00E94DE9087E896E00E9491295E
:10A5D00010928906809106099091070904966AE213
:10A5E00070E00E944324FC01009711F03197108223
:10A5F00060910609709107096C5F7F4F87E896E0CC
:10A6000041E00E94E72B87E896E00E9421280E9403
:10A6100076E36093B8087093B9088093BA08909372
:10A62000BB080C943F60809106099091070905963C
:10A630006AE270E00E9443248C01009719F1209196
:10A6400000093091010980E690E0AC01249FC0012F
:10A65000259F900D349F900D1124885F964F6EE4D6
:10A6600070E00E94432460E270E00E9443249C0159
:10A670002F5F3F4F30930709209306090150104088
:10A68000F801108260910609709107096B5F7F4F96
:10A6900087E896E00E94072E0C943F600E9476E3C4
:10A6A0006093BC087093BD088093BE089093BF0868
:10A6B0002091B8083091B9084091BA085091BB0870
:10A6C000621B730B840B950B28EE33E040E050E0E7
:10A6D0000E94EDEEF22EE32ED42EC52E2DB73EB7FE
:10A6E000285030400FB6F8943EBF0FBE2DBF0DB7B7
:10A6F0001EB70F5F1F4FCE010196EDB7FEB79283D5
:10A7000081838EE197E0F801938382836F2D7E2D04
:10A71000842F952F2CE330E040E050E00E94EDEED6
:10A72000F801358324836F2D7E2D8D2D9C2D2CE3F8
:10A7300030E040E050E00E94EDEEF8017783668360
:10A740000E947224E1EEF4E094912DB73EB7285FA9
:10A750003F4F0FB6F8943EBF0FBE2DBF08C080918B
:10A76000C00085FFFCCF9093C60031969491992349
:10A77000B1F7FE01319607C08091C00085FFFCCF84
:10A7800031969093C60090819923B1F78091C000D3
:10A7900085FFFCCF8AE08093C600CE0101960E941F
:10A7A00059D78091080B882311F40C943F601092C4
:10A7B000080B8091B508082F10E0000F111F0F56ED
:10A7C000184EF80160817181882777FD8095982F58
:10A7D0000E9497EB2091B7043091B8044091B904DE
:10A7E0005091BA040E9403ED181614F00C943F60C7
:10A7F000F801118210820C943F6083E50E94164795
:10A80000882311F40C943F600E9466470E9464EB19
:10A810007B018C016B0180E50E941647882369F05B
:10A82000F7FC0BC0FFEFEF16F10409F034F40E94BF
:10A8300066470E9464EB8B0102C00DE010E0EEE27F
:10A84000F5E0808191818017910711F40C943F60AD
:10A85000329625E0EE39F207A1F70930110529F407
:10A86000D092B708C092B60804C017FF02C00C947B
:10A870003F60802F61E00E9443E5802F6C2D0E9495
:10A88000F6E5802FB6010E9465E40C943F6088E6EF
:10A8900090E00E946F47882311F00C943F6083E59D
:10A8A0000E941647882379F00E9466472091CA08C3
:10A8B000022F10E0000F111F0F56184E0E9464EB7C
:10A8C000F801718360830E949C9A0C943F6083E539
:10A8D0000E941647882311F40C943F600E9466473B
:10A8E0000E9464EB70939417609393170C943F60ED
:10A8F00089E690E00E946F47882311F00C943F6036
:10A90000E8E1F7E0949108C08091C00085FFFCCF9A
:10A910009093C600319694919923B1F7E091CA08BB
:10A92000F0E0EE0FFF1FEE0FFF1FE956F84E4081DB
:10A9300051816281738186E896E021E030E00E94D7
:10A94000C440E5E1F7E0949108C08091C00085FF24
:10A95000FCCF9093C600319694919923B1F7E09182
:10A96000CA08F0E0EE0FFF1FEF56F84E60817181CC
:10A97000882777FD8095982F0E9497EBAB01BC014B
:10A9800086E896E021E030E00E94C440E1E1F7E093
:10A99000949108C08091C00085FFFCCF9093C600C1
:10A9A000319694919923B1F740919D1750919E173C
:10A9B00060919F177091A01786E896E021E030E043
:10A9C0000E94C440EEE0F7E0949108C08091C0007E
:10A9D00085FFFCCF9093C600319694919923B1F7EF
:10A9E0006091931770919417882777FD8095982F21
:10A9F0000E9497EBAB01BC0186E896E021E030E0D5
:10AA00000E94C440EBE0F7E0949108C08091C00040
:10AA100085FFFCCF9093C600319694919923B1F7AE
:10AA200086E896E060E070E04AE050E00E94F13F86
:10AA3000E9E0F7E0949108C08091C00085FFFCCF69
:10AA40009093C600319694919923B1F7409197174E
:10AA5000509198176091991770919A1786E896E02F
:10AA600021E030E00E94C440E6E0F7E0949108C0A5
:10AA70008091C00085FFFCCF9093C60031969491E1
:10AA80009923B1F76091911770919217882777FDFC
:10AA90008095982F0E9497EBAB01BC0186E896E069
:10AAA00021E030E00E94C440E2E0F7E0949108C069
:10AAB0008091C00085FFFCCF9093C60031969491A1
:10AAC0009923B1F78091CA080E94919ABC0186E847
:10AAD00096E04AE050E00E94F13FEDEFF6E09491FD
:10AAE00008C08091C00085FFFCCF9093C6003196CE
:10AAF00094919923B1F78FEF9FEF0E94919ABC0137
:10AB000086E896E04AE050E00E94F13FEFEFF2E085
:10AB100007C08091C00085FFFCCF31969093C6009E
:10AB200090819923B1F78091C00085FFFCCF8AE026
:10AB30008093C6000C9464608DE690E00E946F479D
:10AB4000882311F00C943F6082EF96E00E9437D783
:10AB50001092080B83E50E941647882399F00E9403
:10AB600066472091CA08022F10E0000F111F0F56F0
:10AB7000184E0E9464EBF8017183608381E080933A
:10AB8000AD0416C082E50E941647882389F00E9412
:10AB900066472091CA08022F10E0000F111F0F56C0
:10ABA000184E0E9464EBF801718360831092AD042B
:10ABB00083E50E941647882351F00E946647609300
:10ABC000B7047093B8048093B9049093BA0482E4F4
:10ABD0000E941647882351F00E9466476093B30491
:10ABE0007093B4048093B5049093B60486E40E94F5
:10ABF0001647882369F00E9466476093BB047093F0
:10AC0000BC048093BD049093BE0481E08093080B44
:10AC10000E949C9A0E9476E34B015C012091CA0835
:10AC2000022F10E01092C108000F111FF801EF561B
:10AC3000F84E60817181882777FD8095982F0E945A
:10AC400097EB000F111F0956184EF8012081318132
:10AC5000428153810E9403ED18161CF481E0809319
:10AC6000C108CC24CA94DC2C7601EFEEF6E05490B7
:10AC7000EBEEF6E06490E7EEF6E074905AE0452ED5
:10AC800030C1952DEFEEF6E008C08091C00085FF41
:10AC9000FCCF9093C600319694919923B1F7E0913F
:10ACA000CA08F0E0EE0FFF1FEE0FFF1FE956F84E47
:10ACB000408151816281738186E896E021E030E035
:10ACC0000E94C440962DEBEEF6E008C08091C000D3
:10ACD00085FFFCCF9093C600319694919923B1F7EC
:10ACE0006091CA0886E896E070E04AE050E00E9471
:10ACF000F13F972DE7EEF6E008C08091C00085FF98
:10AD0000FCCF9093C600319694919923B1F7F7FE4A
:10AD100003C0E0E0F3E028C00E9476E3A7019601BB
:10AD2000205F384D4F4F5F4F261B370B480B590B99
:10AD3000CA01B90128EE33E040E050E00E94EDEE98
:10AD400086E896E0BA01A9012AE030E00E94A23F1D
:10AD50008091C00085FFFCCF0EC08091C00085FFB0
:10AD6000FCCF31969093C60090819923B1F78091E2
:10AD7000C00085FFFCCF4092C6000E9476E34B01E5
:10AD80005C010E94129E0E949B420E9417D8FFEF16
:10AD9000CF16FFEFDF06FFEFEF06FFEFFF0609F02C
:10ADA00052C08091C108E091CA08882331F1F0E0D7
:10ADB0008F01000F111F000F111F0956184EEE0FC3
:10ADC000FF1FEF56F84E60817181882777FD8095CF
:10ADD000982F0E9497EB20E030E040E85FE30E946C
:10ADE0001BEA9B01AC01F801608171818281938132
:10ADF0000E9403ED87FF58C05EC0F0E08F01000F96
:10AE0000111F000F111F0956184EEE0FFF1FEF56AE
:10AE1000F84E60817181882777FD8095982F0E9478
:10AE200097EB20E030E040E85FE30E941CEA9B01E2
:10AE3000AC01F80160817181828193810E94F5EA01
:10AE4000181694F538C0F7FC36C0E091CA08F0E057
:10AE50008F01000F111F000F111F0956184EEE0F22
:10AE6000FF1FEF56F84E60817181882777FD80952E
:10AE7000982F0E9497EB9B01AC01F80160817181D2
:10AE8000828193810E941BEA0E9464EB97FF07C0B6
:10AE900090958095709561957F4F8F4F9F4F64304F
:10AEA0007105810591053CF00E9476E3AC01CB0170
:10AEB000DA016C017D01FFEFCF16FFEFDF06FFEF38
:10AEC000EF06FFEFFF0669F0F7FE02C00C94426048
:10AED0000E9476E36C197D096051774210F00C9462
:10AEE00042600E9476E3681979098A099B09695EC4
:10AEF00073408040904008F0C4CE43CF8CEC96E085
:10AF00000E9437D783E50E941647882361F00E948C
:10AF100066470E9464EB709394176093931781E0E7
:10AF20008093AD040FC082E50E941647882351F03C
:10AF30000E9466470E9464EB709394176093931786
:10AF40001092AD040E9476E37B018C011092C1083F
:10AF50006091931770919417882777FD8095982FAB
:10AF60000E9497EB20919D1730919E1740919F175B
:10AF70005091A0170E9403ED18160CF082C081E0DA
:10AF80008093C1087EC00E9476E36E197F09800B12
:10AF9000910B695E73408040904008F46BC0E09173
:10AFA000B508F0E0EE0FFF1FEE0FFF1FE956F84E59
:10AFB00040815181628173819B2DE9ECF6E008C0EC
:10AFC0008091C00085FFFCCF9093C600319694918C
:10AFD0009923B1F786E896E022E030E00E94C44071
:10AFE0009C2DE5ECF6E008C08091C00085FFFCCF09
:10AFF0009093C600319694919923B1F76091B5086A
:10B0000086E896E070E04AE050E00E94F13F9D2D16
:10B01000E1ECF6E008C08091C00085FFFCCF909382
:10B02000C600319694919923B1F740919D175091A4
:10B030009E1760919F177091A01786E896E021E017
:10B0400030E00E94C440EFEFF2E007C08091C00002
:10B0500085FFFCCF31969093C60090819923B1F77C
:10B060008091C00085FFFCCFA092C6000E9476E3CD
:10B070007B018C010E94129E0E949B420E9417D865
:10B080000BC0E9ECF6E0B490E5ECF6E0C490E1EC3E
:10B09000F6E0D4906AE0A62E8091C1082091931723
:10B0A000309194178823A9F0B901882777FD8095FE
:10B0B000982F0E9497EB20919D1730919E174091F9
:10B0C0009F175091A0170E9403ED18160CF45BCF48
:10B0D00018C0B901882777FD8095982F0E9497EBBB
:10B0E00020919D1730919E1740919F175091A01766
:10B0F0000E94F5EA88232CF48091AD04882309F49A
:10B1000042CF87EB96E00E9437D70E9476E36093A8
:10B11000D3087093D4088093D5089093D608AFC70E
:10B1200083E50E941647882319F10E94664720E0B4
:10B1300030E040E050E00E94F5EA88231CF460E033
:10B1400070E011C00E94664720E030E04FE753E412
:10B150000E9403ED18161CF46FEF70E004C00E940B
:10B1600066470E9464EB7093B7086093B60887C780
:10B170008FEF90E09093B7088093B60880C7109245
:10B18000B7081092B6087BC7269A2E9881E0809364
:10B19000AC0483EA96E00E9437D70E9417D86FC7A5
:10B1A0000E949D9A0E94DE90129A0E94EC9010924A
:10B1B000B7081092B60868EE73E080E090E00E9455
:10B1C000AAE3269A2E9A1092AC0481E996E00E9496
:10B1D00037D70E9417D853C71092860850C781E00E
:10B1E000809386084CC783E50E941647882399F010
:10B1F0000E94664720E030E04AE754E40E94D5ED23
:10B200000E9469EB6093DB087093DC088093DD0893
:10B210009093DE0834C788E50E941647882309F01A
:10B220004AC789E50E941647882309F044C78AE582
:10B230000E941647882309F03EC785E40E941647FE
:10B24000882309F038C70E94DE90129A0E94EC9081
:10B2500016C7109299085F9A89E50E9416478823BD
:10B2600019F010929A088A9A8AE50E941647882354
:10B2700041F09FB7F89480910801816080930801A4
:10B280009FBF85E40E941647882309F4F8C6129AE6
:10B29000F6C683E50E9416470E94664720E030E02C
:10B2A0004AE754E40E94D5ED0E9469EB6093D70809
:10B2B0007093D8088093D9089093DA08E0C65CEAC6
:10B2C000652E5AE0752E4CE9242E4AE0342E38EED5
:10B2D000432E3AE0532E88249924F401E65DFA4F78
:10B2E00080810E941647882309F45DC053E08516CB
:10B2F00009F052C00E9466475B016C0120E030E01B
:10B3000040EA51E40E94F5EA88230CF03FC0F301C3
:10B310006081718182819381A60195010E94FCEA7E
:10B320007B018C016091E00A7091E10A8091E20A50
:10B330009091E30AA80197010E94D5ED6093E00A7D
:10B340007093E10A8093E20A9093E30AF10160812D
:10B35000718182819381A80197010E94D5EDF1014D
:10B360006083718382839383F20160817181828122
:10B3700093810E9495EBA80197010E94D5ED0E9450
:10B3800069EBF2016083718382839383F301A0826E
:10B39000B182C282D38207C00E946647F3016083F4
:10B3A0007183828393830894811C911C24E030E094
:10B3B000620E731E220E331E420E531E34E083169D
:10B3C000910409F08ACF5BC6E9E1F6E0949108C0E8
:10B3D0008091C00085FFFCCF9093C6003196949178
:10B3E0009923B1F74CC680910609909107090596FB
:10B3F0006AE270E00E944324FC01009711F031974B
:10B400001082809106099091070905960E9459D7EC
:10B4100036C6E6E1F6E0949108C08091C00085FF51
:10B42000FCCF9093C600319694919923B1F7409147
:10B43000890850918A0860918B0870918C0886E881
:10B4400096E022E030E00E94C440E3E1F6E094910F
:10B4500008C08091C00085FFFCCF9093C600319654
:10B4600094919923B1F740918D0850918E08609185
:10B470008F087091900886E896E022E030E00E9404
:10B48000C440E0E1F6E0949108C08091C00085FFDF
:10B49000FCCF9093C600319694919923B1F74091D7
:10B4A000910850919208609193087091940886E8F1
:10B4B00096E022E030E00E94C440EDE0F6E0949196
:10B4C00008C08091C00085FFFCCF9093C6003196E4
:10B4D00094919923B1F74091950850919608609105
:10B4E00097087091980886E896E022E030E00E9484
:10B4F000C440E2E0F6E0949108C08091C00085FF6E
:10B50000FCCF9093C600319694919923B1F780E0D7
:10B510000E94A9900E9497EB2091AC0A3091AD0A4D
:10B520004091AE0A5091AF0A0E94FCEAAB01BC0107
:10B5300086E896E022E030E00E94C440EFEFF5E0BC
:10B54000949108C08091C00085FFFCCF9093C60005
:10B55000319694919923B1F781E00E94A9900E94BD
:10B5600097EB2091B00A3091B10A4091B20A509104
:10B57000B30A0E94FCEAAB01BC0186E896E022E037
:10B5800030E00E94C440ECEFF5E0949108C0809157
:10B59000C00085FFFCCF9093C6003196949199230B
:10B5A000B1F782E00E94A9900E9497EB2091B40A23
:10B5B0003091B50A4091B60A5091B70A0E94FCEA50
:10B5C000AB01BC0186E896E022E030E00E94C44076
:10B5D000EFEFF2E007C08091C00085FFFCCF31960D
:10B5E0009093C60090819923B1F78091C00085FFA8
:10B5F000FCCF8AE08093C60042C580E00E94C78FDE
:10B600003EC581E00E94C78F3AC58091C00085FF8A
:10B61000FCCF31969093C60090819923B1F7809129
:10B62000C00085FFFCCF8AE08093C600E4EFF5E020
:10B63000949108C08091C00085FFFCCF9093C60014
:10B64000319694919923B1F7659903C0E2E0F3E054
:10B650000AC0E7E0F3E007C08091C00085FFFCCF9F
:10B6600031969093C60090819923B1F78091C000E4
:10B6700085FFFCCF8AE08093C600ECEEF5E0949164
:10B6800008C08091C00085FFFCCF9093C600319622
:10B6900094919923B1F7649B03C0E2E0F3E00AC000
:10B6A000E7E0F3E007C08091C00085FFFCCF319652
:10B6B0009093C60090819923B1F78091C00085FFD7
:10B6C000FCCF8AE08093C600E4EEF5E0949108C0D8
:10B6D0008091C00085FFFCCF9093C6003196949175
:10B6E0009923B1F78091030181FD03C0E2E0F3E00B
:10B6F0000AC0E7E0F3E007C08091C00085FFFCCFFF
:10B7000031969093C60090819923B1F78091C00043
:10B7100085FFFCCF8AE08093C600ECEDF5E09491C4
:10B7200008C08091C00085FFFCCF9093C600319681
:10B7300094919923B1F78091030180FF03C0E2E067
:10B74000F3E00AC0E7E0F3E007C08091C00085FFA6
:10B75000FCCF31969093C60090819923B1F78091E8
:10B76000C00085FFFCCF8AE08093C600E4EDF5E0E1
:10B77000949108C08091C00085FFFCCF9093C600D3
:10B78000319694919923B1F74B9903C0E2E0F3E02D
:10B790000AC0E7E0F3E007C08091C00085FFFCCF5E
:10B7A00031969093C60090819923B1F78091C000A3
:10B7B00085FFFCCF8AE08093C600ECECF5E0949125
:10B7C00008C08091C00085FFFCCF9093C6003196E1
:10B7D00094919923B1F74A9B03C0E2E0F3E00AC0D9
:10B7E000E7E0F3E007C08091C00085FFFCCF319611
:10B7F0009093C60090819923B1F78091C00085FF96
:10B80000FCCF8AE08093C6003AC40AE215E02CEB34
:10B81000E22E2AE0F22EF80180810E94164788234A
:10B8200049F00E9466470E9469EBF70160837183CB
:10B83000828393830F5F1F4F24E030E0E20EF31EFC
:10B8400035E00E32130739F70E948A6C18C40AE2F9
:10B8500015E09CE9E92E9AE0F92EF80180810E941A
:10B860001647882339F00E946647F7016083718389
:10B87000828393830F5F1F4F24E030E0E20EF31EBC
:10B8800035E00E32130749F7FAC383E50E941647E5
:10B89000882351F00E9466476093D00A7093D10AC2
:10B8A0008093D20A9093D30A84E50E941647882396
:10B8B00009F4E5C30E9466476093D40A7093D50AE1
:10B8C0008093D60A9093D70ADAC383E50E9416477D
:10B8D000882351F00E9466476093CC0A7093CD0A8A
:10B8E0008093CE0A9093CF0A84E50E94164788235E
:10B8F00051F00E9466476093E40A7093E50A8093D2
:10B90000E60A9093E70A82E40E941647882361F0D2
:10B910000E9466470E9469EB6093980A7093990AA7
:10B9200080939A0A90939B0A88E50E941647882381
:10B9300051F00E9466476093D80A7093D90A8093A9
:10B94000DA0A9093DB0A8AE50E941647882351F0B1
:10B950000E9466476093DC0A7093DD0A8093DE0ADA
:10B960009093DF0A85E40E941647882309F487C371
:10B970000E9466476093E00A7093E10A8093E20AAE
:10B980009093E30A7CC30AE215E08DE9E82E88E093
:10B99000F82EF80180810E941647882339F00E9412
:10B9A0006647F70160837183828393830F5F1F4F24
:10B9B00024E030E0E20EF31E35E00D32130749F7C4
:10B9C0005EC383E50E941647882309F458C30E948A
:10B9D00066470E9464EB70939D0460939C044FC380
:10B9E00083E50E941647882309F449C30E946647ED
:10B9F0000E9464EB70939F0460939E0440C383E5B0
:10BA00000E941647882321F40EE6C02ED12C05C0D3
:10BA10000E9466470E9464EB6B0180E50E94164716
:10BA2000882319F468EE73E004C00E9466470E9400
:10BA300064EB7B010027F7FC0095102F1C141D04FC
:10BA400084F485E2B60120E030E040E050E00E945E
:10BA50002DE7C801B7010E94AAE385E20E94B9E67A
:10BA60000EC3C801B7010E94AAE309C380E50E9482
:10BA70001647882351F00E9466476093C404709370
:10BA8000C5048093C6049093C70489E40E941647B6
:10BA9000882361F00E9466470E94C09A6093C804A0
:10BAA0007093C9048093CA049093CB0484E40E94E9
:10BAB0001647882361F00E9466470E94CC9A6093E3
:10BAC000CC047093CD048093CE049093CF0483E490
:10BAD0000E941647882351F00E9466476093D00465
:10BAE0007093D1048093D2049093D3040E947A9AE5
:10BAF000E1E1F3E007C08091C00085FFFCCF319603
:10BB00009093C60090819923B1F7E4E1F3E007C078
:10BB10008091C00085FFFCCF31969093C600908144
:10BB20009923B1F74091C4045091C5046091C604B3
:10BB30007091C70486E896E022E030E00E94C4409D
:10BB4000E8E1F3E007C08091C00085FFFCCF3196AB
:10BB50009093C60090819923B1F76091C8047091C9
:10BB6000C9048091CA049091CB040E94C69AAB018B
:10BB7000BC0186E896E022E030E00E94C440ECE19F
:10BB8000F3E007C08091C00085FFFCCF3196909311
:10BB9000C60090819923B1F76091CC047091CD04D7
:10BBA0008091CE049091CF040E94D29AAB01BC0147
:10BBB00086E896E022E030E00E94C440E0E2F3E054
:10BBC00007C08091C00085FFFCCF31969093C600DE
:10BBD00090819923B1F74091D0045091D1046091A4
:10BBE000D2047091D30486E896E022E030E00E940F
:10BBF000C440EFEFF2E007C08091C00085FFFCCFAA
:10BC000031969093C60090819923B1F78091C0003E
:10BC100085FFFCCF8AE08093C60031C283E40E9496
:10BC20001647882349F00E9466470E9464EBDC01B6
:10BC3000CB018F730E9458BCE7EBF5E0949108C0EC
:10BC40008091C00085FFFCCF9093C60031969491FF
:10BC50009923B1F76091EA197091EB1986E896E0A3
:10BC60004AE050E00E94F13FEFEFF2E007C0809120
:10BC7000C00085FFFCCF31969093C6009081992338
:10BC8000B1F78091C00085FFFCCF8AE08093C600A9
:10BC9000F6C185E40E941647882319F4CC24DD24DC
:10BCA00012C00E9466470E9464EB6B0177FF0BC0D5
:10BCB0000F2EF0E0EF2EF0E0FF2EFCE80F2FF2E465
:10BCC0001F2FF02D0AC00F2EF0E0EF2EF0E0FF2E18
:10BCD000F6E10F2FF3E41F2FF02D83E50E941647A6
:10BCE000882321F00E9466477B018C0183E40E9437
:10BCF0001647882319F425E030E005C00E94664706
:10BD00000E9464EB9B01C801B701A6010E94BD9F80
:10BD1000B6C10E94DE90B3C10E949B33B0C10E94A5
:10BD20003E3BADC10E94E235AAC10E948F37A7C138
:10BD300083E50E941647882391F08091C0088823EC
:10BD400071F40E9466476093940570939505809303
:10BD50009605909397050E9469EB6093F4058CE437
:10BD60000E941647882319F18091C0088823F9F4AE
:10BD70000E9466470E9464EB9B01AC0160939C05A6
:10BD800070939D0580939E0590939F0597FF0FC02C
:10BD900088279927DC01821B930BA40BB50B80939A
:10BDA0009C0590939D05A0939E05B0939F0580E50B
:10BDB0000E941647882371F08091C008882351F4AF
:10BDC0000E946647609398057093990580939A0541
:10BDD00090939B0584E40E941647882399F08091F4
:10BDE000C008882379F40E9466471092AB0520E0D2
:10BDF00030E040E050E00E94F5EA882319F081E04D
:10BE00008093AB0582E40E941647882361F08091FD
:10BE1000C008882341F40E9466470E9464EBDC015D
:10BE2000CB010E94193D82E50E941647882371F0DC
:10BE30008091C008882351F40E9466476093F905F9
:10BE40007093FA058093FB059093FC0586E40E94AD
:10BE50001647882309F413C10E9466477B018C01B1
:10BE60006093FC087093FD088093FE089093FF0890
:10BE700020E030E040E050E00E9403ED18160CF0A6
:10BE8000FEC0E092AE04F092AF040093B0041093B1
:10BE9000B104F5C01092C0080E9468A48091CF0838
:10BEA0009091D008A091D108B091D2088093CB088E
:10BEB0009093CC08A093CD08B093CE080E94514532
:10BEC000DEC084E50E941647882309F48DC00E94D5
:10BED00066470E9469EB262F6093CA086623B9F172
:10BEE000E1EEF4E0949108C08091C00085FFFCCFA2
:10BEF0009093C600319694919923B1F7E4E2F3E070
:10BF000007C08091C00085FFFCCF31969093C6009A
:10BF100090819923B1F786E896E0622F40E050E0E7
:10BF20000E94AD3FE6E2F3E007C08091C00085FFCC
:10BF3000FCCF31969093C60090819923B1F7809100
:10BF4000C00085FFFCCF8AE08093C60098C086E4DD
:10BF50000E9416478823E1F00E9466477B018C010E
:10BF60006093FC087093FD088093FE089093FF088F
:10BF700020E030E040E050E00E9403ED181644F469
:10BF8000E092AE04F092AF040093B0041093B104B9
:10BF9000E1EEF4E0949108C08091C00085FFFCCFF1
:10BFA0009093C600319694919923B1F7E7E3F3E0BB
:10BFB00007C08091C00085FFFCCF31969093C600EA
:10BFC00090819923B1F76091B50886E896E070E01A
:10BFD0004AE050E00E94F13F8091C00085FFFCCF15
:10BFE0008AE08093C6004BC0E1EEF4E0949108C073
:10BFF0008091C00085FFFCCF9093C600319694914C
:10C000009923B1F7E4EAF5E0949108C08091C0006B
:10C0100085FFFCCF9093C600319694919923B1F798
:10C02000209100093091010980E690E0289FF001FD
:10C03000299FF00D389FF00D1124E85FF64F07C0DF
:10C040008091C00085FFFCCF31969093C60090810F
:10C050009923B1F7E2EAF5E0949108C08091C0001D
:10C0600085FFFCCF9093C600319694919923B1F748
:10C070008091C00085FFFCCF8AE08093C6000E94BB
:10C08000154222C089ED96E00E9437D70E9476E3E0
:10C090006093B8087093B9088093BA089093BB086E
:10C0A0000E9476E36093D3087093D4088093D508F8
:10C0B0009093D608E4CF0E94DE9088E50E94164750
:10C0C000882309F0C6C8C8C86E960FB6F894DEBFBC
:10C0D0000FBECDBFCF91DF911F910F91FF90EF90D9
:10C0E000DF90CF90BF90AF909F908F907F906F9098
:10C0F0005F904F903F902F9008952F923F924F92D4
:10C100005F926F927F928F929F92AF92BF92CF92E7
:10C11000DF92EF92FF920F931F93DF93CF93CDB7F0
:10C12000DEB76E970FB6F894DEBF0FBECDBF80E6C8
:10C13000A82EB12CEDEEF7E084900AE0702EE3E635
:10C14000F8E094906624639434C22D3071F02A3361
:10C1500021F480918D0A882341F080918E0A90917C
:10C160008F0A8F3591050CF400C2E0918E0AF09190
:10C170008F0A309709F417C3A091900AB091910AE1
:10C18000AA9D9001AB9D300DBA9D300D1124E20F98
:10C19000F31FE85FF64F108280918D0A882309F023
:10C1A000DFC110928D0AAE5FB64F1C92690128E084
:10C1B00039E0C20ED31EC6016AE179E00E9408246C
:10C1C000892B39F4C6016EE470E00E944324009785
:10C1D00029F5C60167E179E00E940824892B09F45A
:10C1E00086C3C60164E179E00E9408248C01C6017F
:10C1F0006EE470E00E9443247C01081B190B093097
:10C2000011050CF074C3C60161E179E00E940824B5
:10C210008E199F09181619060CF069C3C6016EE441
:10C2200070E00E94432490930709809306090196C9
:10C2300060E070E04AE050E00E94AB226093920A16
:10C240007093930A8093940A9093950AC090CB08B8
:10C25000D090CC08E090CD08F090CE08A7019601D0
:10C260002F5F3F4F4F4F5F4F62177307840795074C
:10C2700009F446C38091900A9091910AFC01EA9DCD
:10C28000C001EB9D900DFA9D900D1124885F964F93
:10C290006CE079E00E940824892B09F031C3E7EEB5
:10C2A000F4E0949108C08091C00085FFFCCF90938A
:10C2B000C600319694919923B1F7E9EDF8E0949195
:10C2C00008C08091C00085FFFCCF9093C6003196D6
:10C2D00094919923B1F786E896E0B701A6012AE088
:10C2E00030E00E94BE3F8091C00085FFFCCF73C04C
:10C2F000FE264F5FFC01E40FF11DE85FF64FE08181
:10C30000EA32B1F73093070920930609C901019673
:10C3100060E070E00E944E210E9464EB2F2D30E01F
:10C320002617370709F45DC0E7EEF4E0949108C0E2
:10C330008091C00085FFFCCF9093C6003196949108
:10C340009923B1F7EAEBF8E0949108C08091C0001E
:10C3500085FFFCCF9093C600319694919923B1F755
:10C360004091CB085091CC086091CD087091CE08D7
:10C3700086E896E02AE030E00E94BE3F8091C0004F
:10C3800085FFFCCF28C0E7EEF4E0949108C08091CF
:10C39000C00085FFFCCF9093C600319694919923FD
:10C3A000B1F7E0E9F8E0949108C08091C00085FF02
:10C3B000FCCF9093C600319694919923B1F786E80B
:10C3C00096E0B701A6012AE030E00E94BE3F8091CE
:10C3D000C00085FFFCCF8AE08093C6000E945145D3
:10C3E00042C08091920A9091930AA091940AB091D0
:10C3F000950A8093CB089093CC08A093CD08B09376
:10C40000CE0836C0E7EEF4E0949108C08091C000F9
:10C4100085FFFCCF9093C600319694919923B1F794
:10C42000E6E6F8E0949108C08091C00085FFFCCF5B
:10C430009093C600319694919923B1F74091CB081F
:10C440005091CC086091CD087091CE0886E896E0B6
:10C450002AE030E00E94BE3F8091C00085FFFCCF03
:10C460008AE08093C60010928F0A10928E0A67C2EB
:10C470008091900A9091910A8A9D70018B9DF00C99
:10C480009A9DF00C11248701085F164FC80167E4DC
:10C4900070E00E9443249C01009709F44BC09093E4
:10C4A0000709809306092F5F3F4F201B310B2E0D8C
:10C4B0003F1DC901885F964F60E070E00E944E21E9
:10C4C0000E9464EB64307105A8F58091C008882350
:10C4D000C9F480918706882369F5992DE3E6F8E091
:10C4E00008C08091C00085FFFCCF9093C6003196B4
:10C4F00094919923B1F78091C00085FFFCCF709291
:10C50000C60018C0982DEDEEF7E008C08091C0007D
:10C5100085FFFCCF9093C600319694919923B1F793
:10C520008091C00085FFFCCF7092C60083EE97E03B
:10C530000E9437D78091900A9091910A019664E009
:10C5400070E00E94DAEE9093910A8093900A8091B5
:10C55000960A9091970A01969093970A8093960A6B
:10C5600010928F0A10928E0A24C02B3311F460921D
:10C570008D0A80918D0A8823E1F420918E0A3091F2
:10C580008F0A8091900A9091910A8A9DF0018B9D6B
:10C59000F00D9A9DF00D1124E20FF31FE85FF64FA6
:10C5A00080918C0A80832F5F3F4F30938F0A2093B6
:10C5B0008E0A8091820690918306209184063091A4
:10C5C0008506821B930B8F779070892B09F4B2C17B
:10C5D0008091960A9091970A04970CF0ABC186E877
:10C5E00096E00E94E23E282F80938C0A8A3009F060
:10C5F000ACCDBBCD80918E0A90918F0A892B09F426
:10C6000028C19DC14D3089F04A3321F480918D0AB3
:10C61000882359F080918E0A90918F0A8F35910569
:10C6200024F42F5F3F4F09F0EFC02091780830913C
:10C63000790840917A0850917B0880917008909118
:10C640007108A0917208B0917308281739074A073A
:10C650005B0708F4A1C0962DE0EDF7E008C08091DB
:10C66000C00085FFFCCF9093C6003196949199232A
:10C67000B1F78091C00085FFFCCF3092C6000E94C8
:10C6800076E36093BC087093BD088093BE089093D6
:10C69000BF082091B8083091B9084091BA0850916C
:10C6A000BB08621B730B840B950B28EE33E040E054
:10C6B00050E00E94EDEEF22EE32ED42EC52E2DB7C3
:10C6C0003EB7285030400FB6F8943EBF0FBE2DBF86
:10C6D0000DB71EB70F5F1F4FEDB7FEB7B282A18235
:10C6E000F801538242826F2D7E2D842F952F20E1F9
:10C6F0003EE040E050E00E94EDEEF80135832483F7
:10C700006F2D7E2D8D2D9C2D2CE330E040E050E0F0
:10C710000E94EDEECA01B9012CE330E040E050E0A8
:10C720000E94EDEEF801778366830E947224972DB4
:10C73000E1EEF4E02DB73EB7285F3F4F0FB6F89417
:10C740003EBF0FBE2DBF08C08091C00085FFFCCF4B
:10C750009093C600319694919923B1F7F50107C0E3
:10C760008091C00085FFFCCF31969093C6009081E8
:10C770009923B1F78091C00085FFFCCF3092C600AD
:10C78000C5010E9459D787E896E00E94802887E873
:10C7900096E061E00E94ED2E20918E0A30918F0A82
:10C7A0002115310519F410928D0AC9C08091900AA3
:10C7B0009091910A889DF001899DF00D989DF00D52
:10C7C0001124E20FF31FE85FF64F1082FC01EE5FC9
:10C7D000F64F20822091960A3091970A2F5F3F4FA3
:10C7E0003093970A2093960A019664E070E00E94C5
:10C7F000DAEE9093910A8093900A10928D0A10922B
:10C800008F0A10928E0A3AC04B3311F420928D0A8F
:10C8100080918D0A882391F520918E0A30918F0A9C
:10C820008091900A9091910A889DF001899DF00D68
:10C83000989DF00D1124E20FF31FE85FF64F8091F1
:10C840008C0A80832F5F3F4F30938F0A20938E0A8C
:10C8500015C010E6812E912C22242394E0EDF7E000
:10C860006490BAE03B2E5E010894A11CB11CACEBB5
:10C870004A2EA7E05A2EE1EEF4E074902091780859
:10C880003091790840917A0850917B088091700826
:10C8900090917108A0917208B09173082817390718
:10C8A0004A075B0708F04BC08091960A9091970A5F
:10C8B00004970CF044C080915D0890915E08A091AF
:10C8C0005F08B09160088093780890937908A093EE
:10C8D0007A08B0937B0885E598E00E94B8859C01B2
:10C8E000482F80938C0A8A3009F08CCE9ECEC601E8
:10C8F0006AE270E00E944324009709F4B9CD82CD2A
:10C900008091900A9091910A8A9D80018B9D100DD3
:10C910009A9D100D1124C801885F964F6AE270E05D
:10C920000E9443249C01009709F42DCDFF2440E090
:10C93000C801E0CC80918906882309F05BCE6E9611
:10C940000FB6F894DEBF0FBECDBFCF91DF911F9120
:10C950000F91FF90EF90DF90CF90BF90AF909F909E
:10C960008F907F906F905F904F903F902F900895A1
:10C97000CF93DF938091960A9091970A03970CF4D6
:10C98000BCDB87E896E060E00E94ED2E8091960A7D
:10C990009091970A892B09F469C0809187068823B2
:10C9A00009F44CC0209100093091010980E690E023
:10C9B000289FE001299FD00D389FD00D1124C85F1A
:10C9C000D64FCE0162E379E00E940824892BE1F47E
:10C9D00087E896E0BE010E94AA29809188068823F4
:10C9E00069F5EFE2F9E0949108C08091C00085FFFD
:10C9F000FCCF9093C600319694919923B1F7809122
:10CA0000C00085FFFCCF16C087E896E00E94912900
:10CA1000EDE1F9E0949108C08091C00085FFFCCF62
:10CA20009093C600319694919923B1F78091C000FC
:10CA300085FFFCCF8AE08093C60002C00E94A04818
:10CA40008091960A9091970A01979093970A809304
:10CA5000960A8091000990910109019664E070E0C6
:10CA60000E94DAEE90930109809300090E94129EC1
:10CA70000E949B420E94D0990E9417D8DF91CF91CB
:10CA80000895DF93CF930F920F92CDB7DEB70E9438
:10CA9000D441269A2E9886E896E040E052EC61E078
:10CAA00070E00E94AA3EECE2FAE0949108C0809106
:10CAB000C00085FFFCCF9093C600319694919923D6
:10CAC000B1F78091C00085FFFCCF8AE08093C6005B
:10CAD00041EE54E0FA01949108C08091C00085FFB6
:10CAE000FCCF9093C600319694919923B1F784B707
:10CAF000282F80FF15C0E4E2FAE0949108C08091ED
:10CB0000C00085FFFCCF9093C60031969491992385
:10CB1000B1F78091C00085FFFCCF8AE08093C6000A
:10CB200021FF15C0E4E1FAE0949108C08091C000B3
:10CB300085FFFCCF9093C600319694919923B1F76D
:10CB40008091C00085FFFCCF8AE08093C60022FF61
:10CB500015C0E3E0FAE0949108C08091C00085FF21
:10CB6000FCCF9093C600319694919923B1F78091B0
:10CB7000C00085FFFCCF8AE08093C60023FF15C06C
:10CB8000E3EFF9E0949108C08091C00085FFFCCFED
:10CB90009093C600319694919923B1F78091C0008B
:10CBA00085FFFCCF8AE08093C60025FF15C0E3EE29
:10CBB000F9E0949108C08091C00085FFFCCF90936C
:10CBC000C600319694919923B1F78091C00085FFFA
:10CBD000FCCF8AE08093C60014BEEBEDF9E094919F
:10CBE00008C08091C00085FFFCCF9093C6003196AD
:10CBF00094919923B1F7E5EDF9E0949108C0809103
:10CC0000C00085FFFCCF9093C60031969491992384
:10CC1000B1F78091C00085FFFCCF8AE08093C60009
:10CC2000FA019491E1EEF4E008C08091C00085FF24
:10CC3000FCCF9093C600319694919923B1F7E5EC1F
:10CC4000F9E0949108C08091C00085FFFCCF9093DB
:10CC5000C600319694919923B1F7EAE9F9E09491ED
:10CC600008C08091C00085FFFCCF9093C60031962C
:10CC700094919923B1F7EEE8F9E0949108C080917E
:10CC8000C00085FFFCCF9093C60031969491992304
:10CC9000B1F7E3E7F9E0949108C08091C00085FF07
:10CCA000FCCF9093C600319694919923B1F780916F
:10CCB000C00085FFFCCF8AE08093C600E8E6F9E07B
:10CCC000949108C08091C00085FFFCCF9093C6006E
:10CCD000319694919923B1F7ECE5F9E0949108C06D
:10CCE0008091C00085FFFCCF9093C600319694914F
:10CCF0009923B1F78091C00085FFFCCF8AE0809333
:10CD0000C600FA019491E1EEF4E008C08091C00001
:10CD100085FFFCCF9093C600319694919923B1F78B
:10CD2000EDE4F9E0949108C08091C00085FFFCCF4C
:10CD30009093C600319694919923B1F72091521B9C
:10CD40003091531BCE0101962115310519F48855F8
:10CD50009B4102C0821B930B9A83898369817A81EC
:10CD600086E896E04AE050E00E94F13FE6E3F9E011
:10CD7000949108C08091C00085FFFCCF9093C600BD
:10CD8000319694919923B1F786E896E060E17AE0D4
:10CD90004AE050E00E94F13F8091C00085FFFCCF47
:10CDA0008AE08093C6001092020910920309109243
:10CDB0000409109205090E943E3B0E949B9C0E9420
:10CDC000596F0E94D08F0E940DD980E197E220E92F
:10CDD00031E0F9013197F1F70197D9F7249A0E94D0
:10CDE0001A3E0F900F90CF91DF910895BC01809172
:10CDF000960A9091970A04970CF070C02091900ABF
:10CE00003091910A80E690E0AC01249FC001259FFB
:10CE1000900D349F900D1124885F964F0E94DA2365
:10CE2000E1EEF4E0949108C08091C00085FFFCCF52
:10CE30009093C600319694919923B1F7E4E3FAE018
:10CE4000949108C08091C00085FFFCCF9093C600EC
:10CE5000319694919923B1F72091900A3091910ADB
:10CE600080E690E0289FF001299FF00D389FF00D9B
:10CE70001124E85FF64F07C08091C00085FFFCCF0A
:10CE800031969093C60090819923B1F7E2E3FAE0DE
:10CE9000949108C08091C00085FFFCCF9093C6009C
:10CEA000319694919923B1F78091C00085FFFCCF12
:10CEB0008AE08093C600C901019664E070E00E9498
:10CEC000DAEE9093910A8093900A8091960A90915D
:10CED000970A01969093970A8093960A0895BC0149
:10CEE0008091960A9091970A04970CF070C0209157
:10CEF000900A3091910A80E690E0AC01249FC00135
:10CF0000259F900D349F900D1124885F964F0E94AD
:10CF10004E24E1EEF4E0949108C08091C00085FFBA
:10CF2000FCCF9093C600319694919923B1F7E1E438
:10CF3000FAE0949108C08091C00085FFFCCF9093E7
:10CF4000C600319694919923B1F72091900A3091BF
:10CF5000910A80E690E0289FF001299FF00D389F0C
:10CF6000F00D1124E85FF64F07C08091C00085FFE7
:10CF7000FCCF31969093C60090819923B1F7EFE3EF
:10CF8000FAE0949108C08091C00085FFFCCF909397
:10CF9000C600319694919923B1F78091C00085FF26
:10CFA000FCCF8AE08093C600C901019664E070E07E
:10CFB0000E94DAEE9093910A8093900A8091960AEB
:10CFC0009091970A01969093970A8093960A0895F4
:10CFD0002F923F924F925F926F927F928F929F9289
:10CFE000AF92BF92CF92DF92EF92FF920F931F9377
:10CFF000DF93CF93CDB7DEB7CD55D0400FB6F894C1
:10D00000DEBF0FBECDBF2F969FAF8EAF2F9761961D
:10D010007FAF6EAF61972A0162962FAF62976396DA
:10D020000FAF63976496EFAE64976896ACAEBDAEF3
:10D03000CEAEDFAE6897E22EFF24EE0CFF1CEE0CA6
:10D04000FF1C9A012E0D3F1D2D963FAF2EAF2D9741
:10D05000D9016D907D908D909C90FC01EE0DFF1D8F
:10D06000C401B30120813181428153810E941CEAB5
:10D0700069AF7AAF8BAF9CAF10E0000F111F000FAC
:10D08000111FF201E00FF11F2B96FFAFEEAF2B97B0
:10D09000A080B180C280D3802F96EEADFFAD2F97D8
:10D0A000E00FF11FC601B50120813181428153811A
:10D0B0000E941CEA6DAB7EAB8FAB98AF64962FAD30
:10D0C0006497E22FF0E0EE0FFF1FEE0FFF1F2F9689
:10D0D000AEADBFAD2F97AE0FBF1F4D915D916D915E
:10D0E0007C9129964CAF5DAF6EAF7FAF299761966B
:10D0F0006EAD7FAD6197E60FF71F60817181828110
:10D10000938129962CAD3DAD4EAD5FAD29970E9420
:10D110001BEA69AB7AAB8BAB9CAB6196AEADBFAD96
:10D1200061971C968D919D910D90BC91A02D259697
:10D130008CAF9DAFAEAFBFAF25972F96AEADBFAD55
:10D140002F971C962D913D914D915C911F972196A3
:10D150002CAF3DAF4EAF5FAF2197A4019301505864
:10D160002DA73EA74FA758ABB601A501705849A7F8
:10D170005AA76BA77CA761966EAD7FAD6197E60E4F
:10D18000F71ED7016D917D918D919C9129AD3AAD9E
:10D190004BAD5CAD0E941BEA3B014C016196EEADCC
:10D1A000FFAD61970E0F1F1FD8016D917D918D917D
:10D1B0009C912DA93EA94FA958AD0E941BEA5B0185
:10D1C0006C016DA57EA58FA598A9A60195010E9469
:10D1D000D5ED7B018C0169A57AA58BA59CA5A40141
:10D1E00093010E94D5ED9B01AC01C801B7010E94DB
:10D1F0001BEA1B012C016DA57EA58FA598A9A40192
:10D2000093010E94D5ED7B018C0169A57AA58BA5C0
:10D210009CA5A60195010E94D5ED9B01AC01C8011A
:10D22000B7010E941CEA9B01AC01C201B1010E943E
:10D230008FEA5B016C0120E030E040E050E00E94AA
:10D24000F5EA882354F4C601B5012BED3FE049EC23
:10D2500050E40E941CEA5B016C01E8968FADE897F0
:10D26000882351F0C601B5012BED3FE049EC50E4B5
:10D270000E941BEA5B016C01C601B501E7962CAD6B
:10D280003DAD4EAD5FADE7970E94D5ED29A93AA916
:10D290004BA95CA95F770E9410ED7B018C012FE602
:10D2A00032E143E85AE30E94F5EA87FDF4C1C80180
:10D2B000B7010E94D2EB0E9469EB78A76FA3672B9E
:10D2C00021F4E1E0F0E0F8A7EFA32FA138A5B90120
:10D2D00080E090E00E9495EB7B018C01C601B501D6
:10D2E000A80197010E94FCEA6BA37CA38DA39EA3D7
:10D2F00069A97AA98BA99CA9A80197010E94FCEAB7
:10D300006F8F78A389A39AA325966CAD7DAD8EAD62
:10D310009FAD259721962CAD3DAD4EAD5FAD2197CC
:10D320000E941BEAA80197010E94FCEA6B8F7C8F88
:10D330008D8F9E8F6BA17CA18DA19EA120E030E0FE
:10D3400040E05FEB0E94D5ED2BA13CA14DA15EA179
:10D350000E94D5ED20E030E040E85FE30E941CEA47
:10D360006F8B788F898F9A8F64963FAD6497E32F88
:10D37000F0E0EE0FFF1FEE0FFF1F9E012F5F3F4FEC
:10D38000E20FF31F29964CAD5DAD6EAD7FAD2997D1
:10D3900040835183628373832F96AEADBFAD2F97C9
:10D3A0001C964D915D916D917C911F974D875E8785
:10D3B0006F87788B41E050E05A8B498B66246296E8
:10D3C0007FAD6297672F70E0660F771F660F771F3C
:10D3D000C901860F971F6A969FAF8EAF6A976396B3
:10D3E000BFAD6397AB2FB0E0AA0FBB1FAA0FBB1F47
:10D3F00021E030E02C0F3D1F2A0F3B1F6C963FAF02
:10D400002EAF6C976E96FFAFEEAF6E9719C138E1F5
:10D4100036150CF446C06DA57EA58FA598A92BA145
:10D420003CA14DA15EA10E94D5ED7B018C0169A5B7
:10D430007AA58BA59CA52F89388D498D5A8D0E9480
:10D44000D5ED9B01AC01C801B7010E941CEA7B012C
:10D450008C016DA57EA58FA598A92F89388D498D42
:10D460005A8D0E94D5ED5B016C0169A57AA58BA54B
:10D470009CA52BA13CA14DA15EA10E94D5ED9B01D5
:10D48000AC01C601B5010E941BEA6DA77EA78FA75C
:10D4900098AB6394C701D80189A79AA7ABA7BCA78B
:10D4A00065C049895A89BA0180E090E00E9495EBF5
:10D4B0002BA13CA14DA15EA10E94D5ED7B018C0169
:10D4C000C8010E94F9EA6B8B7C8B8D8B9E8BB70118
:10D4D000C8010E9438EE3B014C012D96AEADBFADA8
:10D4E0002D97ED90FD900D911C9117FB109517F95C
:10D4F00010952B96EEADFFAD2B97208031804280AA
:10D500005380C801B7012B893C894D895E890E94EF
:10D51000D5ED5B016C01C201B101A40193010E9430
:10D52000D5ED9B01AC01C601B5010E941CEA6DA7B7
:10D530007EA78FA798ABC801B701A40193010E94F1
:10D54000D5ED7B018C01C201B1012B893C894D894C
:10D550005E890E94D5ED9B01AC01C801B7010E9414
:10D560001BEA69A77AA78BA79CA7662469AD7AAD49
:10D570008BAD9CAD2DA53EA54FA558A90E941CEAD8
:10D580006A96AEADBFAD6A976D937D938D939C9374
:10D5900013976DA97EA98FA998AD29A53AA54BA58A
:10D5A0005CA50E941CEA6C96EEADFFAD6C976083A3
:10D5B0007183828393836E96AEADBFAD6E976D918E
:10D5C0007D918D919C912F8D38A149A15AA10E94E6
:10D5D0001CEA6E96EEADFFAD6E9760837183828319
:10D5E00093836D857E858F8598892B8D3C8D4D8DA0
:10D5F0005E8D0E941CEA6D877E878F87988BCE0197
:10D6000001960E94C640CE010196BE016B5F7F4F1E
:10D61000AE01475F5F4F9E01235F3F4F6896ECACC2
:10D62000FDAC0EAD1FAD6897F8E7CF2ED12CCC0E18
:10D63000DD1E02D729893A892F5F3F4F3A8B298B0C
:10D6400049895A896FA178A54617570708F4DFCE94
:10D6500061964EAD5FAD6197485F5F4F61962EADAD
:10D660003FAD6197245F3F4F61968EAD9FAD61974F
:10D67000DC0114966196BFAFAEAF6197BD016896AD
:10D68000ECACFDAC0EAD1FAD6897E8E7CE2ED12C0B
:10D69000CC0EDD1ED1D6C35ADF4F0FB6F894DEBFD5
:10D6A0000FBECDBFCF91DF911F910F91FF90EF90F3
:10D6B000DF90CF90BF90AF909F908F907F906F90B2
:10D6C0005F904F903F902F9008953F924F925F92BE
:10D6D0006F927F928F929F92AF92BF92CF92DF9282
:10D6E000EF92FF920F931F93CF93DF938091080BDC
:10D6F000882309F4F6C08090B7049090B804A090F5
:10D70000B904B090BA04609191177091921788276C
:10D7100077FD8095982F0E9497EB20E030E040E065
:10D7200050E40E941CEAA50194010E94F5EA87FDDD
:10D73000D8C030901A150F2EF0E04F2EF0E05F2E7B
:10D74000F0E06F2EF0E07F2EF02DC1EAD0E058C05F
:10D75000232D30E02C9FF0012D9FF00D3C9FF00D0C
:10D760001124E75FF44F80819181A281B3810097FA
:10D77000A105B10581F484819581A681B7810097C7
:10D78000A105B10541F480859185A285B3850097F7
:10D79000A105B10591F12C9F60012D9FD00C3C9FFC
:10D7A000D00C112489E09BE0C80ED91EF6016485D7
:10D7B0007585868597850E9497EB7B018C01F60124
:10D7C00060897189828993890E9495EB9B01AC01E4
:10D7D000C801B7010E94FCEAF60122A133A144A1CD
:10D7E00055A10E94D5ED7B018C01A30192010E94FD
:10D7F00003ED181614F4270138013394FFE03F229B
:10D8000080911915381609F0A3CFC301B2012091F8
:10D81000BB043091BC044091BD045091BE040E94F1
:10D82000D5ED9B01AC01C501B4010E941CEA7B014E
:10D830008C01A50194010E94F5EA87FD02C0470111
:10D8400058011091B3040091B404F090B504E09035
:10D85000B604C501B401212F302F4F2D5E2D0E943B
:10D8600003ED181634F4812F902FAF2DBE2D4C01EF
:10D870005D0140902F1550903015609031157090DB
:10D880003215C301B201A50194010E9403ED1816DF
:10D89000C4F4C501B40120E037ED43EA5CE30E9423
:10D8A000D5ED7B018C01C301B20128E431EE4AE7DA
:10D8B0005FE30E94D5EDA80197010E941CEA4B018D
:10D8C0005C0180922F1590923015A0923115B09284
:10D8D0003215C501B4010E9464EB709392176093F6
:10D8E0009117DF91CF911F910F91FF90EF90DF90F3
:10D8F000CF90BF90AF909F908F907F906F905F90F0
:10D900004F903F9008958091191590911A15891B99
:10D910008F7008950F931F93CF93DF93C0E0D0E0F3
:10D920008E010851154FFE01E454F54F608171815D
:10D93000828193810E9495EBFE01E455F54F208191
:10D940003181428153810E94D5ED0E9469EBF8013B
:10D9500060837183828393832496C031D10501F75C
:10D96000DF91CF911F910F910895FC01608171812A
:10D97000828193812091B80A3091B90A4091BA0A04
:10D980005091BB0A0E94D5ED0E94A5ED6093040B57
:10D990007093050B8093060B9093070B84E09BE03C
:10D9A0000C9498908F929F92AF92BF92CF92DF92F9
:10D9B000EF92FF920F931F93FC018B015A014901D3
:10D9C00060817181828193812091AC0A3091AD0A8E
:10D9D0004091AE0A5091AF0A0E94D5ED0E94A5ED8C
:10D9E00038EFC32E3AE0D32E6093F80A7093F90A09
:10D9F0008093FA0A9093FB0AF80160817181828119
:10DA000093812091B00A3091B10A4091B20A5091AD
:10DA1000B30A0E94D5ED0E94A5ED24E0E22EF12C80
:10DA2000EC0CFD1C6093FC0AF701718382839383E5
:10DA3000F50160817181828193812091B40A3091D6
:10DA4000B50A4091B60A5091B70A0E94D5ED0E94DE
:10DA5000A5ED8601085F1F4F6093000BF8017183ED
:10DA600082839383F401608171818281938120910B
:10DA7000B80A3091B90A4091BA0A5091BB0A0E9483
:10DA8000D5ED0E94A5EDF6013C966093040B7183E1
:10DA900082839383C601B701A8019F010E945E9013
:10DAA00080E090E0A0E0B0E080931B1590931C15FF
:10DAB000A0931D15B0931E1580931F1590932015EC
:10DAC000A0932115B09322158093231590932415CC
:10DAD000A0932515B09326158093271590932815AC
:10DAE000A0932915B0932A1580932B1590932C158C
:10DAF000A0932D15B0932E151F910F91FF90EF90CD
:10DB0000DF90CF90BF90AF909F908F9008958F92AD
:10DB10009F92AF92BF92CF92DF92EF92FF920F93BC
:10DB20001F93CF93DF93EC016B01009709F45CC066
:10DB30008FA9882309F058C0EEA0FFA008A519A559
:10DB4000FB01B6A0A7A090A481A4C801B7012B2D0A
:10DB50003A2D492D582D0E94F5EA88230CF044C037
:10DB6000C801B701A80197010E94D5ED7B018C0186
:10DB70006AA97BA98CA99DA9905820E030E040E0DB
:10DB800050EC0E94D5ED2EA53FA548A959A90E94A9
:10DB9000D5ED9B01AC01C801B7010E941CEA0E94AF
:10DBA00042EE7B018C016B2D7A2D892D982D9701EA
:10DBB000A8010E94F5EA882324F4EB2CFA2C092D05
:10DBC000182D6B2D7A2D892D982D9701A8010E9473
:10DBD000F5EA882349F0C701D801F60186A397A387
:10DBE000A0A7B1A781E086ABDF91CF911F910F91E4
:10DBF000FF90EF90DF90CF90BF90AF909F908F906D
:10DC00000895EF92FF920F931F93CF93DF93F090BD
:10DC10001A1500E010E020E030E041EAE42E11C0E7
:10DC2000FE9CE0011124C75FD44FC901B801AE01C9
:10DC30006EDF8F2D8F5F803109F480E0F82E980120
:10DC40008E0180911915F81659F7C901B80140E005
:10DC500050E05DDFDF91CF911F910F91FF90EF902A
:10DC60000895AF92BF92CF92DF92EF92FF920F93FF
:10DC70001F93CF93DF93EB018A016115710509F4BE
:10DC800066C04115510509F462C0DAA4CBA4BCA456
:10DC9000ADA46EA17FA188A599A52D2D3C2D4B2D5E
:10DCA0005A2D0E94F5EA882309F451C08FA98823D0
:10DCB00009F043C0F801E6A0F7A000A511A56D2D5D
:10DCC0007C2D8B2D9A2DA80197010E9403ED18162B
:10DCD000A4F5C801B701A80197010E94D5ED7B0109
:10DCE0008C016AA97BA98CA99DA9905820E030E0FD
:10DCF00040E050EC0E94D5ED2EA53FA548A959A9BA
:10DD00000E94D5ED9B01AC01C801B7010E941CEA3D
:10DD10000E9442EE7B018C016D2D7C2D8B2D9A2D66
:10DD20009701A8010E94F5EA882324F4ED2CFC2C2D
:10DD30000B2D1A2DC701D80104C08D2D9C2DAB2DA4
:10DD4000BA2D8EA39FA3A8A7B9A781E08EABDF91C0
:10DD5000CF911F910F91FF90EF90DF90CF90BF90E8
:10DD6000AF900895CF92DF92EF92FF920F93DF93DF
:10DD7000CF930F920F92CDB7DEB7809119158FB761
:10DD8000F894F0901A158FBF8091191590E0409685
:10DD90008F1991098F7090700497FCF000911915FC
:10DDA00003500F70CC24DD2440E050E061EAE62E01
:10DDB00012C0802F002309F480E1082F01500E9D2E
:10DDC000C0011124875F944F9A838983B60149DF8C
:10DDD000A601C980DA800F1561F70F900F90CF91DF
:10DDE000DF910F91FF90EF90DF90CF900895CF9348
:10DDF000DF936091B60890911A15809119159817C4
:10DE000011F470E043C040911A15242F30E081EAEC
:10DE100090E0289FF001299FF00D389FF00D11240C
:10DE2000EF5AF44F608150E070E0C1EAD0E028C0C2
:10DE3000242F30E02C9FF0012D9FF00D3C9FF00D22
:10DE40001124E75FF44F80859185A285B385009703
:10DE5000A105B10509F05F5F2C9FF0012D9FF00D2A
:10DE60003C9FF00D1124E75FF44F84859585A685CE
:10DE7000B7850097A105B10509F07F5F4F5F4F702F
:10DE8000809119154817A1F6552341F49FB7F894CE
:10DE9000809108018160809308019FBF772309F476
:10DEA000129A89E070E00E9465E40FDCDF91CF9167
:10DEB00008951092191510921A1580E1E8EFFAE012
:10DEC000DF011D928A95E9F780E090E0A0E0B0E0E4
:10DED00080931F1590932015A0932115B0932215C0
:10DEE0008093231590932415A0932515B0932615A0
:10DEF0008093271590932815A0932915B0932A1580
:10DF000080932B1590932C15A0932D15B0932E155F
:10DF100080931B1590931C15A0931D15B0931E158F
:10DF200008952F923F924F925F926F927F928F92BD
:10DF30009F92AF92BF92CF92DF92EF92FF920F9398
:10DF40001F93DF93CF93CDB7DEB766970FB6F894E4
:10DF5000DEBF0FBECDBF9E8B8D8B6A017B0148015A
:10DF60005901DC01D8966D917D918D919C91DB9743
:10DF70000E9495EB698B7A8B8B8B9C8BA70196010A
:10DF80000E94D5ED0E94E2EA0E9469EB6D837E83D8
:10DF90008F83988769897A898B899C89A5019401E7
:10DFA0000E94D5ED0E94E2EA0E9469EB69837A83C0
:10DFB0008B839C832D813E814F8158852837310585
:10DFC0004105510540F448E750E060E070E04D83C2
:10DFD0005E836F83788769817A818B819C816837C2
:10DFE00071058105910540F488E790E0A0E0B0E07C
:10DFF00089839A83AB83BC83AD89BE89AC5BBF4FF9
:10E00000AD90BD90CD90DC901397A454B040BE8BE2
:10E01000AD8BDC966D917D918D919C91DF970E94E7
:10E0200095EB6D877E878F87988BC601B5010E941F
:10E0300097EB1B012C0120E030E040E050E00E9413
:10E04000F5EA882321F4E0E070E060E028C0698907
:10E050007A898B899C899B01AC010E94D5ED7B015B
:10E060008C016D857E858F8598899B01AC010E940E
:10E07000D5ED9B01AC01C801B7010E941BEA7B01F1
:10E080008C01C201B101A20191010E941CEA9B0115
:10E09000AC01C801B7010E94FCEAE62F692F2E2FC0
:10E0A000372F482F562FB901CA010E94E2EA0E9479
:10E0B00064EB3B014C01ED89FE89E05CFF4F608120
:10E0C0007181828193810E9495EB69877A878B8722
:10E0D0009C8766277727CB016A197B098C099D09E4
:10E0E0000E9497EB5B016C0120E030E040E050E0E3
:10E0F0000E94F5EA882321F4E0E070E060E028C0A7
:10E1000069857A858B859C859B01AC010E94D5ED44
:10E110007B018C0169897A898B899C899B01AC017F
:10E120000E94D5ED9B01AC01C801B7010E941BEA1A
:10E130007B018C01C601B501A60195010E941CEA74
:10E140009B01AC01C801B7010E94FCEAE62F692FD0
:10E150002E2F372F482F562FB901CA010E94D2EB1C
:10E16000ED89FE89A088B188C288D38886017501AF
:10E17000E618F708080919090E9464EBA80197013D
:10E18000261B370B480B590B57FF71C0C201B10159
:10E1900020E030E040E050E00E94F5EA882321F4DE
:10E1A000E0E070E060E044C0C201B101A201910171
:10E1B0000E941CEA7B018C01C601B5010E9495EB0F
:10E1C0009B01AC01C801B7010E94D5ED7B018C0118
:10E1D0006D857E858F8598899B01AC010E94D5ED68
:10E1E0009B01AC01C801B7010E941BEA7B018C01B5
:10E1F00069857A858B859C859B01AC010E94D5ED54
:10E200009B01AC01C801B7010E941CEA7B018C0193
:10E21000C201B10120E030E040E850E40E94D5EDB9
:10E220009B01AC01C801B7010E94FCEAE62F692FEF
:10E230002E2F372F482F562FB901CA010E94E2EA2C
:10E240000E9464EBAC01CB01DA013C014D0197FE69
:10E2500003C06624772443016A147B048C049D0464
:10E2600010F03501460120E030E040E050E09FB77B
:10E27000F8946D897E8960567F4FDB018C91A05A9E
:10E28000B040BE8BAD8B882321F5FD01648A758A71
:10E29000868A978A260D371D481D591D58962D933D
:10E2A0003D934D935C935B972D813E814F815885C3
:10E2B000DC962D933D934D935C93DF97A05CBF4F0D
:10E2C00029813A814B815C812D933D934D935C93E1
:10E2D00013979FBF66960FB6F894DEBF0FBECDBFF3
:10E2E000CF91DF911F910F91FF90EF90DF90CF9032
:10E2F000BF90AF909F908F907F906F905F904F9066
:10E300003F902F9008954F925F927F928F929F92AD
:10E31000AF92BF92CF92DF92EF92FF920F931F9333
:10E32000CF93DF9370901A15C0E0D0E071EA472ECA
:10E33000512C45C02097A9F18EA9882361F4849CB3
:10E34000F001859CF00D949CF00D1124E75FF44FD3
:10E3500086A9882331F1EAA0FBA00CA11DA16EA122
:10E360007FA188A599A5A80197010E94FCEA5B01FD
:10E370006C01849CF001859CF00D949CF00D11249F
:10E38000E75FF44F66A177A180A591A5A801970149
:10E390000E94FCEA8B019C01CE01B601A501C1DD02
:10E3A0001EAA739480E1781609F47724849CE00116
:10E3B000859CD00D949CD00D1124C75FD44F872C21
:10E3C000992487FC90948091191590E088169906FD
:10E3D00009F0B0CF2097E9F0EAA0FBA00CA11DA1A5
:10E3E0006EA17FA188A599A5A80197010E94FCEACA
:10E3F0005B016C016DEC7CEC8CE49DE3A801970162
:10E400000E94FCEA8B019C01CE01B601A50189DDC9
:10E410001EAADF91CF911F910F91FF90EF90DF9097
:10E42000CF90BF90AF909F908F907F905F904F90D4
:10E43000089598DCE6DB67CF2F923F924F925F9270
:10E440006F927F928F929F92AF92BF92CF92DF9204
:10E45000EF92FF920F931F93DF93CF93CDB7DEB769
:10E46000C859D0400FB6F894DEBF0FBECDBF5C01D7
:10E470004B013A012901CB56DF4FE882C559D04004
:10E48000CA56DF4FF882C659D040C956DF4F0883BD
:10E49000C759D040C856DF4F1883C859D040E796B7
:10E4A000DFAECEAEE797809119158F5F803109F40A
:10E4B00080E0282F332727FD309538AB2FA706C0E3
:10E4C0000E94129E0E949B420E9417D880911A15AA
:10E4D00090E04FA558A98417950791F36091AC0A75
:10E4E0007091AD0A8091AE0A9091AF0AE5966CAF3B
:10E4F0007DAF8EAF9FAFE597D5012D913D914D91A9
:10E500005C910E94D5ED0E94A5EDC158DF4F688354
:10E51000CF57D040C058DF4F7883C058D040CF5736
:10E52000DF4F8883C158D040CE57DF4F9883C25801
:10E53000D0402091B00A3091B10A4091B20A509176
:10E54000B30AE1962CAF3DAF4EAF5FAFE197CA0182
:10E55000B901D4012D913D914D915C910E94D5ED71
:10E560000E94A5EDCD57DF4F6883C358D040CC57EC
:10E57000DF4F7883C458D040CB57DF4F8883C558CE
:10E58000D040CA57DF4F9883C658D0402091B40A74
:10E590003091B50A4091B60A5091B70AAD962CAFAA
:10E5A0003DAF4EAF5FAFAD97CA01B901D3012D9119
:10E5B0003D914D915C910E94D5ED0E94A5EDC9570A
:10E5C000DF4F6883C758D040C857DF4F7883C8589B
:10E5D000D040C757DF4F8883C958D040C657DF4F58
:10E5E0009883CA58D0402091B80A3091B90A409116
:10E5F000BA0A5091BB0AA9962CAF3DAF4EAF5FAFA0
:10E60000A997CA01B901D2012D913D914D915C911B
:10E610000E94D5ED0E94A5EDC557DF4F6883CB580A
:10E62000D040C457DF4F7883CC58D040C357DF4F1A
:10E630008883CD58D040C257DF4F9883CE58D04002
:10E6400080911915E82FF0E0A596FFAFEEAFA597E2
:10E6500081EA90E09F01289FF001299FF00D389FEB
:10E66000F00D1124E75FF44FE056FF4F1082E05A9F
:10E67000F0404091F80A5091F90A6091FA0A7091BD
:10E68000FB0AA3964CAF5DAF6EAF7FAFA397C158A7
:10E69000DF4F288039804A805B80CF57D040241AD2
:10E6A000350A460A570A208231824282538257FE37
:10E6B0000BC088279927DC0182199309A409B509A1
:10E6C00080839183A283B3836091FC0A7091FD0AD9
:10E6D0008091FE0A9091FF0A6F966CAF7DAF8EAF6E
:10E6E0009FAF6F97CD57DF4F288139814A815B817A
:10E6F000C358D040261B370B480B590B6B962CAFD9
:10E700003DAF4EAF5FAF6B9781EA90E0A5964EADFF
:10E710005FADA597489FF001499FF00D589FF00D00
:10E720001124E75FF44F6B966CAD7DAD8EAD9FAD60
:10E730006B97648375838683978397FF0DC0DC0195
:10E74000CB01B095A095909581959F4FAF4FBF4F4E
:10E7500084839583A683B7838091000B9091010BEE
:10E76000A091020BB091030B67968CAF9DAFAEAF3B
:10E77000BFAF6797C957DF4F288139814A815B81D5
:10E78000C758D040281B390B4A0B5B0B63962CAF44
:10E790003DAF4EAF5FAF639781EA90E0A5964EAD77
:10E7A0005FADA597489FF001499FF00D589FF00D70
:10E7B0001124E75FF44F63966CAD7DAD8EAD9FADD8
:10E7C0006397608771878287938797FF0DC0DC010D
:10E7D000CB01B095A095909581959F4FAF4FBF4FBE
:10E7E00080879187A287B3878091040B9091050B56
:10E7F000A091060BB091070B2F968CAF9DAFAEAFDB
:10E80000BFAF2F97C557DF4F288139814A815B8180
:10E81000CB58D040281B390B4A0B5B0B2B962CAFE7
:10E820003DAF4EAF5FAF2B9740919E0450919F0438
:10E8300027965FAF4EAF27972B966CAD7DAD8EAD13
:10E840009FAD2B9797FF07C0909580957095619528
:10E850007F4F8F4F9F4F2796AEADBFAD27979D013E
:10E86000442737FD4095542F0E94A7EE24E630E060
:10E8700040E050E00E940FEF81EA90E0A5966EAD77
:10E880007FADA597689FF001699FF00D789FF00D0F
:10E890001124E75FF44FDF011C96248711963C9307
:10E8A000119712964C93129713965C93E080F18027
:10E8B000028113816480758086809780A084B184F2
:10E8C000C284D384C901DA019C01AD012A153B053C
:10E8D0004C055D0514F4A60195012615370548057C
:10E8E000590514F4A401930181EA90E0A596AEAD18
:10E8F000BFADA597A89FF001A99FF00DB89FF00D9F
:10E900001124E75FF44FDA01C9012E153F054007D6
:10E91000510714F4D801C701808B918BA28BB38B64
:10E9200081EA90E0A5962EAD3FADA597289FF00116
:10E93000299FF00D389FF00D1124E75FF44FE85B3D
:10E94000FF4F8091B6089091B708AA2797FDA09530
:10E95000BA2F80839183A283B383E854F04010A23E
:10E96000C158DF4F488159816A817B81CF57D040A0
:10E97000A3968CAD9DADAEADBFADA397481759071B
:10E980006A077B0714F481E080A3CD57DF4F28810D
:10E9900039814A815B81C358D0406F966CAD7DADA3
:10E9A0008EAD9FAD6F97261737074807590794F428
:10E9B00081EA90E0A596AEADBFADA597A89FF00106
:10E9C000A99FF00DB89FF00D1124E75FF44F80A1CF
:10E9D000826080A3C957DF4F288139814A815B81DA
:10E9E000C758D04067966CAD7DAD8EAD9FAD679733
:10E9F000261737074807590794F481EA90E0A5964F
:10EA0000AEADBFADA597A89FF001A99FF00DB89F2F
:10EA1000F00D1124E75FF44F80A1846080A3C557F7
:10EA2000DF4F288139814A815B81CB58D0402F96B6
:10EA30006CAD7DAD8EAD9FAD2F972617370748077C
:10EA4000590794F481EA90E0A596AEADBFADA597C5
:10EA5000A89FF001A99FF00DB89FF00D1124E75F6A
:10EA6000F44F80A1886080A381EA90E0A5962EAD46
:10EA70003FADA597289FF001299FF00D389FF00D1D
:10EA80001124E75FF44FE796AEADBFADE7978C91E9
:10EA900081A3208131814281538125962CAF3DAFE6
:10EAA0004EAF5FAF2597211531054105510509F09E
:10EAB0005F9881EA90E0A5964EAD5FADA597489F1F
:10EAC000F001499FF00D589FF00D1124E75FF44FBE
:10EAD000648075808680978061147104810491043C
:10EAE00009F08A9881EA90E0A5966EAD7FADA59772
:10EAF000689FF001699FF00D789FF00D1124E75F8A
:10EB0000F44FA084B184C284D384A114B104C1049D
:10EB1000D10441F09FB7F894809108018E7F8093D3
:10EB200008019FBF81EA90E0A596AEADBFADA59765
:10EB3000A89FF001A99FF00DB89FF00D1124E75F89
:10EB4000F44F84859585A685B7850097A105B10505
:10EB500011F112982091CC0A3091CD0A4091CE0A41
:10EB60005091CF0A29A73AA74BA75CA7CB56DF4FF6
:10EB70006881C559D040CA56DF4F7881C659D04008
:10EB8000C956DF4F8881C759D040C856DF4F98819A
:10EB9000C859D04024C04091E40A5091E50A6091E0
:10EBA000E60A7091E70A49A75AA76BA77CA7CB563C
:10EBB000DF4F6881C559D040CA56DF4F7881C659AA
:10EBC000D040C956DF4F8881C759D040C856DF4F63
:10EBD0009881C859D04029A53AA54BA55CA50E94AB
:10EBE000F5EA87FD18C0CB56DF4F8881C559D04064
:10EBF000CA56DF4F9881C659D040C956DF4FA88109
:10EC0000C759D040C856DF4FB881C859D04089A7EE
:10EC10009AA7ABA7BCA7C201B1010E9497EBE596EA
:10EC20002CAD3DAD4EAD5FADE5970E94FCEAEC9694
:10EC30006FAFEC97ED967FAFED97EE968FAFEE97B7
:10EC4000EF969FAFEF97AC01CB01DA0189839A83EE
:10EC5000AB83BC836B966CAD7DAD8EAD9FAD6B977A
:10EC60000E9497EBE1962CAD3DAD4EAD5FADE197C7
:10EC70000E94FCEAE8966FAFE897E9967FAFE997C4
:10EC8000EA968FAFEA97EB969FAFEB97AC01CB017B
:10EC9000DA018D839E83AF83B88763966CAD7DADBB
:10ECA0008EAD9FAD63970E9497EBAD962CAD3DADB9
:10ECB0004EAD5FADAD970E94FCEA562E472E382E22
:10ECC000292EAC01CB01DA0189879A87AB87BC87F3
:10ECD0002B966CAD7DAD8EAD9FAD2B970E9497EBC3
:10ECE000A9962CAD3DAD4EAD5FADA9970E94FCEA53
:10ECF0007B018C012796AEADBFAD2797BD0188275C
:10ED000077FD8095982F0E9497EB9B01AC01C8017D
:10ED1000B7010E94D5ED20E030E048EC52E40E94BB
:10ED2000FCEA9B01AC016D877E878F87988B2596C7
:10ED30006CAD7DAD8EAD9FAD2597663071058105BB
:10ED400091051CF576E06716710481049104ECF4DA
:10ED500086E0A816B104C104D104BCF481EA90E0B5
:10ED6000A596AEADBFADA597A89FF001A99FF00DE8
:10ED7000B89FF00D1124E75FF44FDA01C901BF77A6
:10ED800086A797A7A0ABB1AB4DC0EC962FADEC9783
:10ED9000ED963FADED97EE964FADEE97EF965FADEA
:10EDA000EF97B901CA010E948CEE3B014C01E89635
:10EDB0002FADE897E9963FADE997EA964FADEA9710
:10EDC000EB965FADEB97B901CA010E948CEE5B0137
:10EDD0006C01252D342D432D522DB901CA010E94FD
:10EDE0008CEE7B018C01C401B301A60195010E9448
:10EDF0001CEAA80197010E941CEA0E9442EE21EA47
:10EE000030E0A5964EAD5FADA597429FF001439FC0
:10EE1000F00D529FF00D1124E75FF44F66A777A71E
:10EE200080AB91AB81EA90E0A5966EAD7FADA597E2
:10EE3000689F8001699F100D789F100D1124075F56
:10EE4000144F065A1F4F609194057091950580915B
:10EE50009605909197050E9464EBD8016D937C9381
:10EE60000850104080919C0590919D05A0919E05B1
:10EE7000B0919F05F80180839183A283B3830550ED
:10EE800010408091A405D8018C938091A605F801CB
:10EE900082938F010C541040815056E5E52EF12CE1
:10EEA000E00EF11E823008F07EC0D8019E966D9172
:10EEB0007D918D919C91D1972091980530919905E4
:10EEC00040919A0550919B050E94D5ED0E9464EBFC
:10EED00097FF07C090958095709561957F4F8F4FF4
:10EEE0009F4FF70160837183828393836091F40560
:10EEF00070E067507040882777FD8095982F0E94BA
:10EF000097EB3B014C0140EBA42E45E0B42E81EA87
:10EF100090E0A5962EAD3FADA597289F6001299F53
:10EF2000D00C389FD00C112445E65BE0C40ED51EF2
:10EF3000D5016C9170E080E090E00E9495EBA40117
:10EF400093010E94D5ED20E030E04FE753E40E94AA
:10EF5000FCEA20E030E040EE50E40E941CEA7B0135
:10EF60008C0120E030E040EE50E40E94F5EA882376
:10EF700051F40F2EF0E0EF2EF0E0FF2EF0E00F2F17
:10EF8000F0E01F2FF02DC801B7010E9469EBF601D8
:10EF900061936F010894A11CB11CF4EFAF16F5E06A
:10EFA000BF0631F606C0D7011D921D921D921C921C
:10EFB000139781EA90E0A5962EAD3FADA597289FC7
:10EFC000F001299FF00D389FF00D1124E75FF44FF9
:10EFD000A080B180C280D380E480F5800681178153
:10EFE0006084718482849384248535854685578521
:10EFF000EA5AFF4F80819181A281B38182179307E2
:10F00000A407B50714F4DA01C90186159705A80508
:10F01000B90514F4D401C3019C01AD018E159F05FF
:10F02000A007B10714F4A80197012A153B054C0568
:10F030005D054CF05C016D018E159F05A007B107C1
:10F0400014F45701680181EA90E0A5964EAD5FADDA
:10F05000A597489FF001499FF00D589FF00D11248E
:10F06000E75FF44FA08AB18AC28AD38A8091AB0548
:10F07000882341F1E35BFF4F8081882319F1ECE4A1
:10F08000FAE0949108C08091C00085FFFCCF909376
:10F09000C600319694919923B1F7E2E5FAE0949194
:10F0A00008C08091C00085FFFCCF9093C6003196C8
:10F0B00094919923B1F78091C00085FFFCCF8AE03D
:10F0C0008093C60081EA90E0A5966EAD7FADA597CE
:10F0D000689FF001699FF00D789FF00D1124E75FA4
:10F0E000F44F86A597A5A0A9B1A98DA39EA3AFA310
:10F0F000B8A760E070E080E89FE32DA13EA14FA19A
:10F1000058A50E94FCEA9B01AC0169A57AA58BA5D4
:10F110009CA50E94D5ED2B013C0180911915909181
:10F120001A15A82FB0E05096A91BB109AF70B070A6
:10F13000BEA7ADA7A230B1050CF451C05D01CC242F
:10F14000B7FCC094DC2CC601B5010E9497EB20E00F
:10F1500030E040E051E40E94F5EA88230CF03FC023
:10F1600060E074E284E799E4A30192010E94FCEA62
:10F170000E94A5ED7B018C016091980A7091990A1B
:10F1800080919A0A90919B0AE616F70608071907DC
:10F1900030F56E197F09800B910B660F771F881F62
:10F1A000991FA60195010E94EDEECA01B9010E94C6
:10F1B00095EB0E94A5ED9B01AC012E0D3F1D401F5C
:10F1C000511FCA01B9010E9495EB9B01AC0160E09F
:10F1D00074E284E799E40E94FCEA2B013C0181EA95
:10F1E00090E0A596EEADFFADA597E89F8001E99F61
:10F1F000100DF89F100D1124075F144F6DA17EA113
:10F200008FA198A5A30192010E94D5EDD8019296F5
:10F210006D937D938D939C93959750966D917D9171
:10F220008D919C9153970E9495EBA30192010E94AE
:10F23000D5ED0E94E2EA0E9469EBF80160AF71AF80
:10F2400082AF93AFC157DF4F1882CF58D040C0571D
:10F25000DF4F1882C059D04020E8222E9FE3392E7C
:10F2600088249924E1E0F0E0EC0FFD1FE80DF91D82
:10F27000C301B20120813181428153810E94D5EDC9
:10F28000E1E1F0E0EC0FFD1FE80DF91D60837183F3
:10F29000828393835B016C01E894D7F8F401E45610
:10F2A000F54FE080F18002811381C601B501A8010C
:10F2B00097010E9403ED1816CCF4C801B701A6010E
:10F2C00095010E94FCEA6B017C01C157DF4F688108
:10F2D000CF58D040C057DF4F7881C059D040C101CE
:10F2E000A70196010E94F5EA88236CF4C157DF4F0D
:10F2F0008881CF58D040C057DF4F9881C059D04047
:10F30000D1016C017D0124E030E0820E931E30E1DA
:10F310008316910471F0D701C601C157DF4FC8822F
:10F32000CF58D040C057DF4F9883C059D0401D01FF
:10F3300099CFC701B60120E030E040E85FE30E94CA
:10F34000F5EA88230CF04CC08E010F5E1F4F81E25E
:10F35000A82EB12CAC0EBD1ED8016D917D918D9162
:10F360009C91A70196010E94D5EDF80161937193DC
:10F37000819391938F01EA15FB0571F781EA90E083
:10F38000A5962EAD3FADA597289F8001299F100D12
:10F39000389F100D1124075F144FD80192966D917C
:10F3A0007D918D919C919597A70196010E94D5ED35
:10F3B000F80162A373A384A395A360AD71AD82AD80
:10F3C00093AD0E9495EBA70196010E94D5ED0E9496
:10F3D00069EBD801D8966D937D938D939C93DB97C1
:10F3E00081EA90E0A596EEADFFADA597E89F80017C
:10F3F000E99F100DF89F100D1124075F144FD801DD
:10F4000050966D917D918D919C9153970E9495EBB3
:10F41000F80126A537A540A951A90E94FCEA1B01C5
:10F420002C01F80180819181A281B3810097A1050F
:10F43000B10549F584819581A681B7810097A10521
:10F44000B10509F580859185A285B3850097A10551
:10F45000B105C9F4C201B1012091D40A3091D50A95
:10F460004091D60A5091D70A0E94D5ED0E94E2EA57
:10F470000C5B1F4F0E9469EBD8016D937D938D93B8
:10F480009C93139771C1C201B1012091D00A3091B0
:10F49000D10A4091D20A5091D30A0E94D5ED0E9420
:10F4A000E2EA0E9469EB21EA30E0A596EEADFFADFD
:10F4B000A597E29F6001E39FD00CF29FD00C11242E
:10F4C00029E03BE0C20ED31EB4E46B2E712C6C0C11
:10F4D0007D1CD3016D937D938D939C9313978090A6
:10F4E000E80A9090E90AA090EA0AB090EB0A0E941C
:10F4F00095EB7B018C01F6016081718182819381A2
:10F500000E9497EB9B01AC01C801B7010E94D5EDA9
:10F510007B018C01D60150966D917D918D919C91CE
:10F5200053970E9495EB9B01AC01C801B7010E9463
:10F53000FCEA7B018C01C501B4010E9495EB9B01A3
:10F54000AC01C801B7010E9403ED18162CF4F301B9
:10F5500080829182A282B3828090EC0A9090ED0A20
:10F56000A090EE0AB090EF0A81EA90E0A5962EAD49
:10F570003FADA597289F6001299FD00C389FD00CE4
:10F58000112449E05BE0C40ED51EA4E46A2E712C60
:10F590006C0C7D1CD3016D917D918D919C910E948D
:10F5A00095EB7B018C01F6016481758186819781E1
:10F5B0000E9497EB9B01AC01C801B7010E94D5EDF9
:10F5C0007B018C01D60150966D917D918D919C911E
:10F5D00053970E9495EB9B01AC01C801B7010E94B3
:10F5E000FCEA7B018C01C501B4010E9495EB9B01F3
:10F5F000AC01C801B7010E9403ED18162CF4F30109
:10F6000080829182A282B3828090F40A9090F50A5F
:10F61000A090F60AB090F70A81EA90E0A5962EAD88
:10F620003FADA597289F6001299FD00C389FD00C33
:10F63000112449E05BE0C40ED51EF4E46F2E712C5A
:10F640006C0C7D1CD3016D917D918D919C910E94DC
:10F6500095EB7B018C01F601648575858685978520
:10F660000E9497EB9B01AC01C801B7010E94D5ED48
:10F670007B018C01D60150966D917D918D919C916D
:10F6800053970E9495EB9B01AC01C801B7010E9402
:10F69000FCEA7B018C01C501B4010E9495EB9B0142
:10F6A000AC01C801B7010E9403ED18162CF4F30158
:10F6B00080829182A282B3828090F00A9090F10AB7
:10F6C000A090F20AB090F30A81EA90E0A5962EADE0
:10F6D0003FADA597289F6001299FD00C389FD00C83
:10F6E000112449E05BE0C40ED51EE4E46E2E712CBB
:10F6F0006C0C7D1CD3016D917D918D919C910E942C
:10F7000095EB7B018C01F60160857185828593857F
:10F710000E9497EB9B01AC01C801B7010E94D5ED97
:10F720007B018C01D60150966D917D918D919C91BC
:10F7300053970E9495EB9B01AC01C801B7010E9451
:10F74000FCEA7B018C01C501B4010E9495EB9B0191
:10F75000AC01C801B7010E9403ED18162CF4F301A7
:10F7600080829182A282B38281EA90E0A5962EAD3A
:10F770003FADA597289F6001299FD00C389FD00CE2
:10F78000112449E05BE0C40ED51EF601EC5BFF4F8F
:10F7900060817181828193810E9495EB7B018C0154
:10F7A000A20191010E94FCEAD601D2966D937D934D
:10F7B0008D939C93D597C801B7012DEB37E346E0B5
:10F7C00051E40E94D5ED0E9464EBF601648F758FC1
:10F7D000868F978F6090D80A7090D90A8090DA0A45
:10F7E0009090DB0AC401B30120E030E040E05FE329
:10F7F0000E94D5ED5B016C01298D3A8D4B8D5C8D9E
:10F8000021962CAF3DAF4EAF5FAF21974091DC0A00
:10F810005091DD0A6091DE0A7091DF0A49AF5AAF5C
:10F820006BAF7CAFCB01BA0120E030E040E05FE39A
:10F830000E94D5ED7B018C0121966CAD7DAD8EAD26
:10F840009FAD21979F77A80197010E9403ED18169D
:10F8500044F4C601B501A80197010E94F5EA882386
:10F8600014F4860175016D8D7E8D8F8D98A16DAB21
:10F870007EAB8FAB98AF8091E00A9091E10AA091A6
:10F88000E20AB091E30A89AB9AABABABBCABBC016B
:10F89000CD0120E030E040E05FE30E94D5ED1B01A8
:10F8A0002C016DA97EA98FA998AD9F77A201910126
:10F8B0000E9403ED181644F4C801B701A20191019A
:10F8C0000E94F5EA882314F41701280181EA90E0E8
:10F8D000A596AEADBFADA597A89FF001A99FF00D6D
:10F8E000B89FF00D1124E75FF44F22A133A144A18A
:10F8F00055A129A33AA34BA35CA3C201B1010E9465
:10F90000F5EA87FD04C029A03AA04BA05CA04DA554
:10F910005EA5423051050CF407C150911B15CF561E
:10F92000DF4F5883C159D04060911C15CE56DF4F30
:10F930006883C259D04070911D15CD56DF4F788332
:10F94000C359D04080911E15CC56DF4F8883C459CF
:10F95000D040652FCE56DF4F7881C259D040CD566A
:10F96000DF4F8881C359D040CC56DF4F9881C459AE
:10F97000D04027E137EB41ED58E30E9403ED181624
:10F980000CF0D2C069897A898B899C8920911F15D6
:10F990003091201540912115509122150E941BEAAB
:10F9A0009B01AC010E94D5ED7B018C016D897E89A4
:10F9B0008F89988D2091231530912415409125151C
:10F9C000509126150E941BEA9B01AC010E94D5EDC7
:10F9D0009B01AC01C801B7010E941CEA0E9442EEE3
:10F9E0007B018C01A40193010E9403ED18165CF0C9
:10F9F0000F2EF0E06F2EF0E07F2EF0E88F2EFFE369
:10FA00009F2EF02D08C0C401B301A80197010E94E8
:10FA1000FCEA3B014C0121966CAD7DAD8EAD9FADF6
:10FA20002197209127153091281540912915509143
:10FA30002A150E941BEA7B018C01E89417F9C80182
:10FA4000B70129AD3AAD4BAD5CAD0E9403ED181680
:10FA500094F469AD7AAD8BAD9CADA80197010E947D
:10FA6000FCEA5B016C01C401B301A60195010E948F
:10FA7000F5EA882314F4640153016DA97EA98FA9C6
:10FA800098AD20912B1530912C1540912D1550914A
:10FA90002E150E941BEA7B018C01E89417F9C8011E
:10FAA000B70129A93AA94BA95CA90E9403ED181630
:10FAB00094F469A97AA98BA99CA9A80197010E942D
:10FAC000FCEA7B018C01C601B501A80197010E94E7
:10FAD000F5EA882314F48601750169A17AA18BA146
:10FAE0009CA1A80197010E94D5ED7B018C01CF5606
:10FAF000DF4F6881C159D040CE56DF4F7881C2595F
:10FB0000D040CD56DF4F8881C359D040CC56DF4F0F
:10FB10009881C459D040A80197010E94F5EA87FD59
:10FB200019C0D801C70102C0D201C101CF56DF4FB1
:10FB30008883C159D040CE56DF4F9883C259D040F8
:10FB4000CD56DF4FA883C359D040CC56DF4FB88382
:10FB5000C459D04081EA90E0A596AEADBFADA5975F
:10FB6000A89F8001A99F100DB89F100D1124075F59
:10FB7000144FCF56DF4F8881C159D040CE56DF4F4A
:10FB80009881C259D040CD56DF4FA881C359D0408B
:10FB9000CC56DF4FB881C459D040F80182A793A753
:10FBA000A4A7B5A762A973A984A995A9905820E034
:10FBB00030E040E050EC0E94D5EDD8019E962D91AA
:10FBC0003D914D915C91D1970E94D5ED2BE037EDA1
:10FBD00043E25BE30E941CEA0E9442EEF62EE72E0F
:10FBE000D82EC92ECF56DF4F6881C159D040CE568E
:10FBF000DF4F7881C259D040CD56DF4F8881C3593D
:10FC0000D040CC56DF4F9881C459D0402F2D3E2D87
:10FC10004D2D5C2D0E94F5EA87FD14C0CF56DF4FB5
:10FC2000F882C159D040CE56DF4FE882C259D04049
:10FC3000CD56DF4FD882C359D040CC56DF4FC88253
:10FC4000C459D04081EA90E0A596EEADFFADA597EE
:10FC5000E89F8001E99F100DF89F100D1124075FA8
:10FC6000144FCF56DF4F8881C159D040CE56DF4F59
:10FC70009881C259D040CD56DF4FA881C359D0409A
:10FC8000CC56DF4FB881C459D040F80186A397A362
:10FC9000A0A7B1A762A173A184A195A12F2D3E2D8C
:10FCA0004D2D5C2D0E94F5EA18162CF081E0D8014C
:10FCB000D7968C9302C0F80117AA81EA90E0A59626
:10FCC0002EAD3FADA597289FF001299FF00D389FDD
:10FCD000F00D1124E75FF44F81E086ABAFE1B5E1B1
:10FCE000FE01719680E101900D928150E1F781EA69
:10FCF00090E0A5964EAD5FADA597489F6001499FE6
:10FD0000D00C589FD00C112469E07BE0C60ED71EA2
:10FD1000D6019296ED90FD900D911C919597E092F1
:10FD20001B15F0921C1500931D1510931E15969629
:10FD30006D917D918D919C919997A80197010E9459
:10FD4000FCEA4B015C01C201B101A80197010E94CC
:10FD5000FCEA8B019C01C601B501A4010E94916FD0
:10FD6000BFA5B0931915C557DF4F288139814A8146
:10FD70005B81CB58D0402093040B3093050B40930C
:10FD8000060B5093070BC957DF4F488159816A8191
:10FD90007B81C758D0404093000B5093010B609378
:10FDA000020B7093030BCD57DF4F688179818A81F5
:10FDB0009B81C358D0406093FC0A7093FD0A8093E6
:10FDC000FE0A9093FF0AC158DF4F88819981AA816A
:10FDD000BB81CF57D0408093F80A9093F90AA09343
:10FDE000FA0AB093FB0A0E9419720E94CA8FC85681
:10FDF000DF4F0FB6F894DEBF0FBECDBFCF91DF91BE
:10FE00001F910F91FF90EF90DF90CF90BF90AF9038
:10FE10009F908F907F906F905F904F903F902F902A
:10FE20000895FF920F931F93CF93DF938B010E944E
:10FE300076E3EB01FF24FA9409C00E9476E36C1B81
:10FE40007D0B6017710710F080E008C0FEBC0DB498
:10FE500007FEFDCF8EB58F3F81F781E0DF91CF9117
:10FE60001F910F91FF900895FC014281242F30E0F3
:10FE7000C9019595879580658CBD40FF02C080E0E3
:10FE800004C080E0463009F081E08DBD808160E0F3
:10FE90000C94F6E5DF92EF92FF920F931F93CF93AE
:10FEA000DF93EC01D62E79018A01DEDFCE016CE210
:10FEB00071E0B7DF8D2D80648EBD0DB407FEFDCFE0
:10FEC00028E130E0D801C701022E04C0B695A795FD
:10FED000979587950A94D2F78EBD0DB407FEFDCF96
:10FEE000285030408FEF283F380761F7DD2011F4AC
:10FEF00085E906C088E0D81611F487E801C08FEFC5
:10FF00008EBD0DB407FEFDCF8CE0D81631F48FEF17
:10FF10008EBD0DB407FEFDCF8EB59FEF2FEF2EBD2A
:10FF20000DB407FEFDCF8EB587FF04C0992311F0F5
:10FF30009150F5CF8B83DF91CF911F910F91FF905F
:10FF4000EF90DF900895FC01808161E00C94F6E56C
:10FF5000DC016EBDFA0120E030E00DB407FEFDCFFC
:10FF600080818EBD0DB407FEFDCF81818EBD2E5FD9
:10FF70003F4F329682E02030380779F70DB407FE04
:10FF8000FDCF8FEF8EBD0DB407FEFDCF8FEF8EBD81
:10FF90000DB407FEFDCF8FEF8EBD0DB407FEFDCF74
:10FFA0008EB513968C9313978F71853011F481E081
:10FFB000089583E111968C931197CD01C4DF80E001
:10FFC0000895CF92DF92EF92FF920F931F93CF93FA
:10FFD000DF93EC017A018B0169018C81833039F068
:10FFE00059E0EE0CFF1C001F111F5A95D1F7CE01EE
:10FFF00068E1A80197014EDF882311F086E020C058
:020000021000EC
:10000000CE016EEFA601A4DF8823D9F0CE0168E50A
:1000100072E007DF882311F487E112C0CE016DE0A2
:1000200020E030E040E050E035DF882341F48FEFFE
:100030008EBD0DB407FEFDCF8EB5882371F086E12D
:100040008983CE0180DF80E0DF91CF911F910F91F6
:10005000FF90EF90DF90CF900895CE0174DF81E0A4
:10006000F3CFBF92CF92DF92EF92FF920F931F9345
:10007000CF93DF93EC016B017A010E9476E38B0151
:10008000BB24BA9409C00E9476E3601B710B6D52C9
:10009000714010F081E10BC0BEBC0DB407FEFDCF76
:1000A0008EB58B838F3F79F38E3F31F08FE089835C
:1000B000CE0149DF80E02EC0D7011197EF28D9F09B
:1000C0008FEF8EBD20E030E09FEF0BC00DB407FE38
:1000D000FDCF8EB5F601E20FF31F80839EBD2F5F2B
:1000E0003F4F2A173B0790F30DB407FEFDCF8EB5A7
:1000F000AC0DBD1D8C938FEF8EBD0DB407FEFDCFF3
:100100008EB58FEF8EBD0DB407FEFDCF8EB5CE013F
:100110001ADF81E0DF91CF911F910F91FF90EF9057
:10012000DF90CF90BF900895CF92DF92EF92FF9231
:100130000F931F93CF93DF93EC017A018B01690139
:100140008C81833039F0A9E0EE0CFF1C001F111FD9
:10015000AA95D1F7CE0161E1A80197019BDE882322
:1001600031F084E08983CE01EEDE80E005C0CE016F
:10017000B60140E052E075DFDF91CF911F910F9102
:10018000FF90EF90DF90CF900895BF92CF92DF92D3
:10019000EF92FF920F931F93CF93DF93EC01B62E54
:1001A0001C82198248830E9476E36B01888161E09A
:1001B0000E9443E5CE01C7DE82E360E00E9443E592
:1001C00083E361E00E9443E584E361E00E9443E54C
:1001D00085E361E00E9443E585E361E00E94F6E586
:1001E00085E08A8382E58CBD1DBC80E09FEF9EBDCB
:1001F0000DB407FEFDCF8F5F8A30C9F709C00E949A
:1002000076E36C197D09615D774010F081E059C09B
:10021000CE0160E020E030E040E050E03BDE182F0F
:100220008B83813061F7CE0168E02AEA31E040E05B
:1002300050E030DE82FF02C01C8311C080E02FEF4F
:100240002EBD0DB407FEFDCF9EB58F5F8430C1F784
:100250009B839A3A11F082E034C082E08C838C81D7
:10026000823021F0EE24FF2487010FC0E12CF12C15
:10027000012D00E4102F09C00E9476E36C197D095E
:10028000615D774010F08AE01CC0CE0167E320E09A
:1002900030E040E050E0FEDDCE0169E2A8019701C8
:1002A000F9DD8B83882341F78C81823019F5CE01EB
:1002B0006AE320E030E040E050E0ECDD882329F004
:1002C00088E08983CE013FDE20C08FEF8EBD0DB464
:1002D00007FEFDCF8EB5807C803C11F483E08C83DB
:1002E00080E09FEF9EBD0DB407FEFDCF2EB58F5F62
:1002F0008330C1F7CE0127DE86E08B1518F488E144
:10030000898303C0BA8281E001C080E0DF91CF9190
:100310001F910F91FF90EF90DF90CF90BF900895C5
:10032000CF93DF93EB01DC0190E020E03EE28C9183
:10033000803269F0283029F4FE01E90FF11D308385
:100340009F5FFE01E90FF11D8C9180839F5F2F5FFE
:1003500011962B3061F7C90FD11D1882DF91CF9113
:1003600008950F931F93CF93DF93DC01EB018A0174
:1003700080E090E020E2FE01E80FF91F2083019663
:100380008B309105C1F757E040E024C0622F2E3238
:1003900019F087E69AE007C05A3051F15AE048E078
:1003A00018C0321729F1FC01019634913323C9F7A3
:1003B0005417F0F02132E0F02F37D0F4822F81561D
:1003C0008A3110F4622F6052FE01E40FF11D608348
:1003D0004F5F11962C91222311F02F32B9F6F801BC
:1003E000B183A08390E08881803219F091E001C050
:1003F00090E0892FDF91CF911F910F9108956F9217
:100400007F928F929F92AF92BF92CF92DF92EF92A4
:10041000FF920F931F93CF93DF93EC017A018B012F
:100420002B81222309F480C089899A89AB89BC89F0
:1004300084179507A607B70708F476C085C0E114AE
:10044000F1040105110551F41C821D821E821F82D8
:10045000188619861A861B8681E067C0288539852B
:100460004A855B85E98DFA8D858590E00996215056
:1004700030404040504039014A01082E04C0969453
:100480008794779467940A94D2F72F5F3F4F4F4F2A
:100490005F4F0894E108F10801091109570168014B
:1004A00004C0D694C794B794A7948A95D2F70894B9
:1004B000E11CF11C011D111DA614B704C804D904C8
:1004C00028F0211531054105510549F48D899E8992
:1004D000AF89B88D8C839D83AE83BF8316C0A61869
:1004E000B708C808D90811C04C815D816E817F8131
:1004F000898D9A8D94010E94798D0894A108B10884
:10050000C108D108882331F40FC084E0882E912CD3
:100510008C0E9D1EA114B104C104D10429F7E886F4
:10052000F9860A871B8798CF80E0DF91CF911F91D2
:100530000F91FF90EF90DF90CF90BF90AF909F9082
:100540008F907F906F900895223009F078CFE7CF99
:10055000CF93DF93EC018C859D85AE85BF8540E010
:10056000611141E0BC01CD010E94538B882319F435
:1005700020E030E00AC08889282F30E095E0220F83
:10058000331F9A95E1F7275C3A4EC901DF91CF916D
:1005900008950F931F93CF93DF938C01FC01838108
:1005A0008823E9F1818187FF37C0C80161E0D0DF8E
:1005B000EC010097A1F18881853E89F1F8018381E2
:1005C000823040F481899289A389B4898C8F9D8F70
:1005D000AE8FBF8FF801858996899B8F8A8F858919
:1005E0009689A789B08DCD01AA27BB279D8B8C8BBF
:1005F000E0913315F0913415309751F0BE016A5EE9
:100600007F4FCE0148961995888D998D9B8B8A8B4B
:10061000F80181818F7781830E94188B04C081E06B
:10062000F801808380E0DF91CF911F910F910895B1
:100630000F931F938C01ADDFF80113821F910F916F
:100640000895FC018381882311F0CF01F1CF089533
:10065000CF93DF93FC01EB018381882381F08250EB
:10066000823020F48FE28883198207C0CF0160E0D6
:100670006FDF009721F0BE0153DE81E001C080E012
:10068000DF91CF9108956F927F928F929F92AF9258
:10069000BF92CF92DF92EF92FF920F931F93DF935F
:1006A000CF9300D00F92CDB7DEB77C015A016B011A
:1006B000DC0113968C911397813009F08EC011964E
:1006C0008C9181FF8AC09DC00097A105B10511F4EE
:1006D00081E084C0F7016084718482849384C701BF
:1006E000B601A5018CDE882309F477C0D70159969D
:1006F0008D919C915A97A114B104C104D10489F43D
:1007000055964D915D916D917C9158970E94EE8D1B
:10071000882309F462C0F701158A168A178A108E99
:1007200044C0D70114964D915D916D917C911797BE
:100730009E012F5F3F4F0E94798D882309F44DC0A1
:10074000D7015996ED91FC915A9749815A816B8155
:100750007C818789803149F4483FBFEF5B07B0E077
:100760006B07B0E07B0748F020C0483F8FEF580789
:100770008FEF68078FE07807C0F4CF010E94EE8DFD
:10078000882359F1D70114964D915D916D917C911B
:10079000179759968D919C915A970FEF1FEF2FEF56
:1007A0003FE00E94F38C8823C1F0F701A18AB28A4E
:1007B000C38AD48A818180688183C701EADE882365
:1007C00061F0B601A5016A147B048C049D0410F449
:1007D000B401A301C70113DE01C080E00F900F90A8
:1007E0000F900F90CF91DF911F910F91FF90EF909D
:1007F000DF90CF90BF90AF909F908F907F906F9041
:100800000895F70181899289A389B489841795078E
:10081000A607B70708F058CFE0CFCF93DF93EC01DE
:1008200040E050E060E070E02EDF882359F0CE0118
:1008300061E08EDEFC01009729F085EE80831B824B
:10084000F7D601C080E0DF91CF9108952F923F92BB
:100850004F925F926F927F928F929F92AF92BF92D0
:10086000CF92DF92EF92FF920F931F93CF93DF937C
:10087000EC012A018B81882309F4B5C0898180FFAE
:10088000B2C0C7C025014E185F083B0174E0272E97
:10089000312C2C0E3D1E4201A0C0288539854A8589
:1008A0005B856FEFA62E61E0B62EA222B3228B816C
:1008B00079018A0199E016950795F794E7949A953E
:1008C000D1F7E98DFA8D823049F4428D538D648DD4
:1008D000758D4E0D5F1D601F711F3FC0D480DA946F
:1008E000DE20A114B104D9F4DD20C9F421153105AD
:1008F0004105510549F48D899E89AF89B88D8C8356
:100900009D83AE83BF830BC04C815D816E817F81EF
:10091000CF0191010E94798D882309F464C0E98D8B
:10092000FA8D4C815D816E817F81425050406040E4
:100930007040058404C0440F551F661F771F0A943A
:10094000D2F786859785A089B189480F591F6A1FFC
:100950007B1F4D0D511D611D711D80E092E08A19B4
:100960009B0984018815990508F48C0182E0003008
:10097000180709F066C08091351590913615A09141
:100980003715B0913815481759076A077B0709F4DE
:1009900058C08091391790913A179301C5DB88238D
:1009A00049F421C09501275C3A4EC301B901A80161
:1009B0000E942F24600E711E980140E050E088854F
:1009C0009985AA85BB85820F931FA41FB51F8887B1
:1009D0009987AA87BB87801A910A8114910409F02C
:1009E0005CCFA20102C04FEF5FEFCA01DF91CF9150
:1009F0001F910F91FF90EF90DF90CF90BF90AF903D
:100A00009F908F907F906F905F904F903F902F902E
:100A10000895A988BA88CB88DC88E884F9840A8597
:100A20001B859A0140E050E0D601C5018E199F094F
:100A3000A00BB10B281739074A075B0708F022CF34
:100A400024CFCB01BA0140E02ED6882309F0AACFEB
:100A5000CACFCF92DF92EF92FF920F931F93CF9363
:100A6000DF937C01EB018A01FC018381823008F471
:100A70006EC080859185A285B3858F719070A070BE
:100A8000B0700097A105B10509F061C06CC0F80114
:100A90001082EDE0CE2ED12CC701BE0140E250E025
:100AA000D5DE9C018032910521F0009709F04FC0FE
:100AB00050C04881442309F44CC0453E69F34E328E
:100AC00059F38B858F738F30E9F501151105D1F13D
:100AD0008A8D9B8D892BB1F5842F90E08F7190705A
:100AE000009781F1833091056CF58C9D90018D9D6F
:100AF000300D9C9D300D11242D503040F801E20F37
:100B0000F31F898180838B8181838D8182838F8193
:100B10008383898584838E858583888986838A8972
:100B200087838C8980878E898187888D82878C8D49
:100B300083878E8D8487888186FF04C0F801E20F49
:100B4000F31F15868B8583FDA7CF822F03C08FEF00
:100B500001C080E0DF91CF911F910F91FF90EF9046
:100B6000DF90CF9008954115510509F090CF91CFB6
:100B7000DF93CF930F92CDB7DEB7BE016F5F7F4F8C
:100B800041E050E063DE019719F02FEF3FEF03C023
:100B90008981282F30E0C9010F90CF91DF9108950E
:100BA000EF92FF920F931F93CF93DF93EC018B8112
:100BB000823030F1E884F9840A851B85CE01D8DFC4
:100BC00097FD1EC088859985AA85BB854F96A11D76
:100BD000B11D88879987AA87BB87A5E016950795D9
:100BE000F794E794AA95D1F72E2D30E02F7030704E
:100BF000F5E0220F331FFA95E1F7275C3A4E02C069
:100C000020E030E0C901DF91CF911F910F91FF905B
:100C1000EF9008950F931F93CF93DF93EC018B0117
:100C20008B81882309F040C0FB018789803109F05E
:100C300041C082E08B831D8A1E8A1F8A188E808D98
:100C4000918DA0E0B0E045E0880F991FAA1FBB1F5F
:100C50004A95D1F7898B9A8BAB8BBC8B13C083E001
:100C60008B83F801428D538D648D758D4D8B5E8B1A
:100C70006F8B788F9E012F5E3F4FC8010E944A8E76
:100C8000882391F01A8F098F81E089831C821D824D
:100C90001E821F82188619861A861B861C861D8650
:100CA0001E861F86188A01C080E0DF91CF911F91B8
:100CB0000F9108958032C1F7D2CF1F93CF93DF9366
:100CC000EC01142F262F30E0F90175E0EE0FFF1F25
:100CD0007A95E1F7E75CFA4E8385817121F0842FE4
:100CE000827109F066C08091351590913615A091FA
:100CF0003715B09138158C879D87AE87BF87688B75
:100D0000F90165E0EE0FFF1F6A95E1F7E75CFA4E27
:100D100084899589A0E0B0E0DC01992788278D8B34
:100D20009E8BAF8BB88F228D338DA90160E070E070
:100D3000482B592B6A2B7B2B4D8B5E8B6F8B788FBF
:100D4000838590E088719070009751F4848D958D23
:100D5000A68DB78D898B9A8BAB8BBC8B81E00BC03A
:100D6000409739F59E012F5E3F4F898D9A8D92D71E
:100D70008823F9F084E08B83812F8F7089831C8214
:100D80001D821E821F82188619861A861B8614FFF2
:100D900016C0CE0140E050E060E070E074DC8823D3
:100DA00071F409C049895A896B897C89CE0127DB96
:100DB00002C01B8280E0DF91CF911F91089515FD45
:100DC000F1CF81E0F8CFCF93DF93EC019C012C5F52
:100DD0003F4F898D9A8D41E050E060E070E0C5D7CB
:100DE0008823A1F08D899E89AF89B88D0097A105D0
:100DF000B10559F48C819D81AE81BF818D8B9E8B15
:100E0000AF8BB88F89818068898381E0DF91CF9132
:100E100008952F923F924F925F927F928F929F926E
:100E2000AF92BF92CF92DF92EF92FF920F931F93F8
:100E3000DF93CF9300D000D0CDB7DEB76C01162F73
:100E4000072F5E834D83DC0113968C9113978130BD
:100E500009F069C111968C9181FF65C182C1F601CB
:100E6000418952896389748980859185A285B3857A
:100E700084179507A607B70729F0C601C0DA8823AB
:100E800009F451C1812F902F9C0119014D805E8082
:100E90000FC1D6015996ED91FC915A97DA01C9011B
:100EA00049E0B695A795979587954A95D1F77480AF
:100EB0007A9478228FEF882E81E0982E82229322D6
:100EC000772009F051C08114910409F04DC0D6017A
:100ED00014964D915D916D917C9117974115510537
:100EE0006105710581F455968D919D910D90BC9190
:100EF000A02D0097A105B10559F1F60184839583D2
:100F0000A683B78331C0CF019E012F5F3F4FF1D53C
:100F1000882309F408C129813A814B815C81D6017B
:100F20005996ED91FC915A978789803149F4283F71
:100F3000BFEF3B07B0E04B07B0E05B0770F008C0C5
:100F4000283FEFEF3E07EFEF4E07EFE05E0728F098
:100F5000C60139DF882341F4E6C0D60114962D93EB
:100F60003D934D935C93179780E092E0881999091F
:100F700052018415950508F45C01D6015996ED914E
:100F8000FC915A971496ED90FD900D911C91179736
:100F90008EEF9FEFAFEFBFEFE80EF91E0A1F1B1F8A
:100FA000058404C0EE0CFF1C001F111F0A94D2F729
:100FB00086859785A089B189E80EF91E0A1F1B1F37
:100FC000E70CF11C011D111D90E0A91692E0B90675
:100FD00039F58091351590913615A0913715B0915E
:100FE00038158E159F05A007B10771F410923B17B5
:100FF0008FEF9FEFAFEFBFEF8093351590933615CE
:10100000A0933715B09338158091391790913A17FE
:10101000B801A70191010E94E17F8823A9F583C04F
:101020008114910411F5D60118962D913D914D91A1
:101030005C911B9751968D919D910D90BC91A02D27
:10104000281739074A075B0780F0F2D2882309F492
:101050006AC081E080933B17E0923515F092361517
:10106000009337151093381507C0C801B70141E048
:101070001AD3882309F457C09401275C3A4EC9015A
:10108000B101A5010E942F24950140E050E0F60136
:1010900080859185A285B385820F931FA41FB51FFC
:1010A00080879187A287B3872A0C3B1C4A185B086C
:1010B000D60118962D913D914D915C911B9741144D
:1010C000510409F0E6CE51968D919D910D90BC9101
:1010D000A02D82179307A407B50748F4F601218BCA
:1010E000328B438B548B81818068818311C08091C6
:1010F000331590913415892B59F08D819E81892B60
:1011000039F0D60111968C911197806811968C93C5
:10111000F601818183FF04C0C6013BDA882319F000
:101120004D815E8105C081E0D6018C934FEF5FEF6A
:10113000CA0126960FB6F894DEBF0FBECDBFCF9181
:10114000DF911F910F91FF90EF90DF90CF90BF90B4
:10115000AF909F908F907F905F904F903F902F9097
:10116000089582FD7CCE8ECEDF92EF92FF920F9398
:101170001F93CF93DF93EC0189899A89AB89BC894E
:10118000805E9F4FAF41B04008F06FC0CE011BDEC4
:10119000882309F46AC04CD2882309F466C0E98D1B
:1011A000FA8DEC80FD800E811F818EEF9FEFAFEFF7
:1011B000BFEFE80EF91E0A1F1B1F058404C0EE0CCA
:1011C000FF1C001F111F0A94D2F786859785A089FE
:1011D000B189E80EF91E0A1F1B1F81E080933B179F
:1011E000E0923515F09236150093371510933815A7
:1011F00080E092E0E9E3F5E1DF019C011D922150DE
:101200003040E1F7DD24D39411C0B801A7014D0DA2
:10121000511D611D711D8091391790913A1729E375
:1012200035E10E94E17F882301F1D394E98DFA8DA5
:101230008481D81650F320E032E040E050E005848D
:1012400004C0220F331F441F551F0A94D2F7898907
:101250009A89AB89BC89820F931FA41FB51F898B04
:101260009A8BAB8BBC8B81E001C080E0DF91CF918A
:101270001F910F91FF90EF90DF9008958F929F92B2
:10128000AF92BF92CF92DF92EF92FF920F931F9394
:10129000CF93DF936C01EB01942E852EA22E898DC6
:1012A0009A8DD6015A969C938E935997CB0140E024
:1012B00050E060E070E0A3D8BB2437C0CE0170DC02
:1012C000FC01009709F48FC055E016950795F79437
:1012D000E7945A95D1F71E2D1F708081882311F055
:1012E000853EC9F4BB2099F420913515309136150F
:1012F0004091371550913815D6011C962D933D938A
:101300004D935C931F9750961C93BB24B39480819C
:10131000882359F418C0892D982DBF014BE050E067
:101320000E942224009709F46CC0E884F9840A859D
:101330001B8589899A89AB89BC89E816F9060A0751
:101340001B0708F4BBCFA6FE4EC0A1FE4CC0BB20BD
:1013500049F0F6011089C60161E0FAD8EC01009766
:1013600061F441C08B81823009F43DC0CE01FCDEC6
:101370008823C9F110E0C9E3D5E180E2DE011D92C6
:101380008A95E9F7DE01292D382DC901FC018BE092
:1013900001900D928150E1F7E0913315F0913415F1
:1013A000309739F0BE01625F7F4FCE0140961995AC
:1013B00008C081E298E2998B888B80E098E09F8753
:1013C0008E87888999899B8B8A8B998F888F8E8548
:1013D0009F859F8B8E8B2CD1882329F0C601612F8E
:1013E0004A2D6BDC01C080E0DF91CF911F910F91FE
:1013F000FF90EF90DF90CF90BF90AF909F908F9035
:101400000895A7FEEBCFEFCF2F923F924F925F92BE
:101410006F927F928F929F92AF92BF92CF92DF9204
:10142000EF92FF920F931F93DF93CF93CDB7DEB769
:10143000C654D0400FB6F894DEBF0FBECDBF3C01FE
:101440006B01DE01AE5BBF4F11965C934E93259608
:101450002FAF25971C861F861FA21AA6611571053E
:1014600009F47CC0FC018381882309F077C0FA016C
:1014700080818F32F1F08601ECE0EE2EF12CEC0E43
:10148000FD1E72E4A72EB12CAC0EBD1E4E010894B9
:10149000811C911C2796FFAEEEAE279767E2262EA1
:1014A000312C2C0E3D1E270123C01196B183A08341
:1014B00001C0FD01A081B1818C918F32B1F3D601C1
:1014C00013968C91139782508230A8F28E01095D99
:1014D0001F4F59966D917C915A97C8019BDB8823C9
:1014E00059F63CC0342D252D8701832F922F7C0186
:1014F000F50180819181B401A5010E94B181882309
:1015000029F42CC03196D501ED93FC93D501ED91D2
:10151000FC9180818F32B1F38823B9F0C701B80103
:10152000A40121E0ABDE8823C9F00C151D0511F0E4
:10153000C8017ED82796EEADFFAD2797EE16FF06C1
:1015400089F6C101322D292FCFCFC301B801A401E3
:1015500025962FAD259792DE182F01C010E0CE0101
:1015600087966FD8CE010C966CD8812FCA5BDF4F5F
:101570000FB6F894DEBF0FBECDBFCF91DF911F91A4
:101580000F91FF90EF90DF90CF90BF90AF909F9022
:101590008F907F906F905F904F903F902F90089525
:1015A0000F931F93DF93CF93CDB7DEB76B970FB633
:1015B000F894DEBF0FBECDBF9C01AB0119821C8227
:1015C0008E010F5F1F4FC801B90122E01DDF882384
:1015D00011F410E003C0C80120D9182FCE010196E4
:1015E00030D8812F6B960FB6F894DEBF0FBECDBFFB
:1015F000CF91DF911F910F910895DB010D90002095
:10160000E9F71197A61BB70B0496AD0102CCDF9347
:10161000CF930F92CDB7DEB769830496BE016F5F9B
:101620007F4F41E050E0F5DB0F90CF91DF910895BF
:1016300080913B17882399F14091351550913615CB
:1016400060913715709138158091391790913A173C
:1016500029E335E10E94E17F882319F140913C178D
:1016600050913D1760913E1770913F1741155105FC
:101670006105710591F08091391790913A1729E32E
:1016800035E10E94E17F882361F010923C171092AF
:101690003D1710923E1710923F1710923B1781E0B2
:1016A000089580E00895DF92EF92FF920F931F93C9
:1016B0007B018C01D42E8091351590913615A09127
:1016C0003715B09138158E159F05A007B107B9F0F1
:1016D000AFDF8823E1F08091391790913A17B80174
:1016E000A70129E335E10E949480882381F0E092EC
:1016F0003515F09236150093371510933815DD2007
:1017000011F481E005C081E080933B1701C080E0C7
:101710001F910F91FF90EF90DF9008958F929F920D
:10172000AF92BF92CF92DF92EF92FF920F931F93EF
:10173000CF93DF936C01142F70933A17609339178E
:10174000FC01178A82E090E0A0E0B0E08083918302
:10175000A283B38310923B1710923C1710923D174F
:1017600010923E1710923F178FEF9FEFAFEFBFEF32
:101770008093351590933615A0933715B09338158F
:10178000442321F48824992454013FC0453008F0B3
:101790001CC160E070E080E090E040E084DF8823DE
:1017A00009F413C1C12FD0E02197FE0174E0EE0FC0
:1017B000FF1F7A95E1F7E75CFA4EE254FE4F808115
:1017C000EE5BF14090E08F779070892B09F0FDC0BF
:1017D000E653FE4F80819181A281B38184369105C9
:1017E000A105B10508F4F1C064E0CC0FDD1F6A95D6
:1017F000E1F7C150D94E88809980AA80BB808114BE
:101800009104A104B10409F4E0C0C501B40140E0B1
:101810004ADF882309F4D9C0809144159091451579
:101820008050924009F0D1C020914915222309F43B
:10183000CCC08091471590914815892B09F4C5C0FB
:1018400080914615882309F4C0C0F601228B80914F
:1018500046158483158661E070E007C04F5FF6018E
:1018600045874150483008F0B0C0F6014585848175
:1018700090E09B01042E02C0220F331F0A94E2F76E
:101880008217930759F720914F1530915015211564
:10189000310519F040E050E008C020915D1530910D
:1018A0005E1540915F1550916015F60125833683D2
:1018B00047835087E0904715F090481500E010E00E
:1018C000E80CF91C0A1D1B1DE38AF48A058B168B94
:1018D00080914A1590914B15918F808F6091491599
:1018E00070E080E090E00E94A7EE6E0D7F1D801FEB
:1018F000911FF601628F738F848F958F20914A1507
:1019000030914B1555E0220F331F5A95E1F72150C6
:101910003E4F232F3327269540E050E0260F371FF8
:10192000481F591F26873787408B518B80914C1554
:1019300090914D15009719F0A0E0B0E008C080919B
:10194000591590915A15A0915B15B0915C158501C0
:101950007401E21AF30A040B150BA8019701280F72
:10196000391F4A1F5B1FF601058404C05695479531
:10197000379527950A94D2F7218732874387548772
:10198000253FFFE03F07F0E04F07F0E05F0720F45E
:101990008CE0F601878B19C0255F3F4F40405040D7
:1019A00018F480E1F6010EC08091651590916615DE
:1019B000A0916715B0916815F601828F938FA48F5F
:1019C000B58F80E2878B81E001C080E0DF91CF910D
:1019D0001F910F91FF90EF90DF90CF90BF90AF904D
:1019E0009F908F9008956F927F928F929F92AF9267
:1019F000BF92CF92DF92EF92FF920F931F93CF93FC
:101A0000DF93EC015A016B01380149014230510565
:101A10006105710508F45DC089859A85AB85BC8533
:101A20000196A11DB11D84179507A607B70708F4F5
:101A300050C08F89803129F4E52EF62E072F11270B
:101A40000CC0803209F045C07A018B0187E0169501
:101A50000795F794E7948A95D1F78B899C89AD898E
:101A6000BE89E80EF91E0A1F1B1FC801B70141E01D
:101A70001ADE882371F18F89803149F4F501F07005
:101A8000EE0FFF1FE75CFA4E718260820DC0F50118
:101A9000EF77F070EE0FFF1FEE0FFF1FE75CFA4EBF
:101AA00060827182828293828A89823080F08D8105
:101AB0009E81AF81B885E80EF91E0A1F1B1FE092B8
:101AC0003C17F0923D1700933E1710933F1781E0AB
:101AD00001C080E0DF91CF911F910F91FF90EF90B7
:101AE000DF90CF90BF90AF909F908F907F906F903E
:101AF0000895CF92DF92EF92FF920F931F93CF93AF
:101B0000DF93EC017A018B01690189859A85AB85A8
:101B1000BC850196A11DB11D84179507A607B707BF
:101B200008F452C08F89803129F45527412F302F76
:101B30002F2D0CC0803209F047C09A01AB0167E03D
:101B400056954795379527956A95D1F78B899C8946
:101B5000AD89BE89280F391F4A1F5B1F809135153B
:101B600090913615A0913715B0913815281739077F
:101B70004A075B0731F0CA01B90140E094DD8823D0
:101B800019F18F89803159F4F701F070EE0FFF1FC2
:101B9000E75CFA4E80819181A0E0B0E00EC0F701D1
:101BA000EF77F070EE0FFF1FEE0FFF1FE75CFA4EAE
:101BB00080819181A281B381BF70F601808391837E
:101BC000A283B38381E001C080E0DF91CF911F91B8
:101BD0000F91FF90EF90DF90CF900895AF92BF925A
:101BE000CF92DF92EF92FF920F931F93DF93CF93E9
:101BF00000D00F92CDB7DEB76C017A018B0182E085
:101C000090E0A0E0B0E0F60180839183A283B383EB
